:020000040800F2
:1040000008F50020B9420008C1DC00082595000829
:104010009DBB0008A9570008657101080000000059
:10402000000000000000000000000000CD4100087A
:104030007B6600080000000055420008A542000809
:10404000D3420008D3420008D34200089DFD000877
:10405000D3420008D3420008D3420008D3420008EC
:10406000D3420008D3420008D3420008D3420008DC
:10407000D3420008D342000855640008D342000828
:10408000D34200085D640008D3420008D342000810
:10409000D3420008D3420008D3420008C968000890
:1040A000D3420008D3420008D3420008D34200089C
:1040B000D3420008D3420008D3420008D34200088C
:1040C000D3420008D3420008D3420008D34200087C
:1040D000D34200089D640108D964010815650108F0
:1040E000D3420008ADFC0008D342000800000000E5
:1040F00000000000000000000000000000000000C0
:104100000000000000000000D3420008D342000875
:10411000D3420008D3420008D3420008D34200082B
:10412000D3420008D3420008D3420008D34200081B
:10413000D3420008D3420008D3420008D34200080B
:10414000D3420008D3420008D3420008D3420008FB
:10415000DFF80CD000F0A6FC0048004725870108D6
:1041600008F5002080F309887047EFF30980704755
:10417000684680F3098804480078C00714BF02200D
:10418000032080F3148870477CA10108DFF818C071
:10419000EFF305831B0618BF6047EFF31483DB07BB
:1041A00008BF604700DF7047F5910108DFF818C0CD
:1041B000EFF305831B0618BF6047EFF31483DB079B
:1041C00008BF604700DF70479D930108EFF3098047
:1041D000816911F8021C39BB90E80F10E047EFF33A
:1041E000098C194B93E80600914218D059B10CB4D0
:1041F0004FF0010381F826302CE9F00FC1F82CC0F4
:1042000015F0E6FA0CBC1A60D2F82CC0BCE8F00F2E
:1042100092F826308CF309881BB192F82500CCF86F
:1042200000006FF0020E704710B5084A1268914204
:1042300009D8074C54F8214090E80F10A047EFF33D
:10424000098C8CE80F0010BD940400203C4B000842
:104250003C4B000815F08AF9114B93E80600914297
:104260001BD00CB44FF0000381F82630EFF3098C1B
:104270002CE9F00FC1F82CC015F0AAFA0CBC1A609A
:10428000D2F82CC0BCE8F00F8CF3098892F82630E5
:104290001BB192F82530CCF800306FF0020E704759
:1042A0009404002015F064FBD6E7000014F024FC11
:1042B00015F05EFBD0E7000006488047064800473F
:1042C000FEE7FEE7FEE7FEE7FEE7FEE7FEE7FEE7C6
:1042D000FEE7FEE7653A01085141000840EA0103A4
:1042E0009B0703D009E008C9121F08C0042AFAD2AC
:1042F00003E011F8013B00F8013B521EF9D2704770
:10430000D2B201E000F8012B491EFBD27047002217
:10431000F6E710B513460A4604461946FFF7F0FFC4
:10432000204610BD421E12F8013F002BFBD111F8B0
:10433000013B02F8013B002BF9D1704730B505462F
:104340002A460B4612F8010B13F8014B08B1A042A4
:10435000F8D01CB1002802D06D1CF1E7284630BD12
:1043600010B5044604E00B7800F8013B03B1491C8A
:10437000521EF8D2204610BD421C10F8011B002925
:10438000FBD1801A704710B5002200E0521C835CFC
:104390008C5CA34201D1002BF8D1D8B2E1B2401A13
:1043A00010BD30B504460020034600E05B1C93427C
:1043B00003D2E05CCD5C401BF8D030BD034611F861
:1043C000012B00F8012B002AF9D11846704730B5AF
:1043D00005460020034600E05B1C934205D2EC5CDE
:1043E000C85C201A01D1002CF6D130BD2DE9F04770
:1043F00091460F4680460446002614F8015B2DB115
:1044000000F070FA0068405DC007F6D12B2D02D095
:104410002D2D18D0641E4A463946204600F066FA13
:1044200027B13968A14201D1C7F8008071054FF06A
:1044300002040BD54042002803DD13F0CBF90460E1
:10444000A007BDE8F08746F48066E4E70028F8DAC4
:1044500013F0C0F904606FF00040F2E770B5064653
:1044600013F0B8F9046805460A2200213046FFF728
:10447000BDFF2C6070BD70B5064613F0ABF9046843
:1044800005460A2200213046FFF7B0FF2C6070BDC0
:104490002DE9FE4F804681EA0300C00F0C460090D4
:1044A00021F0004123F00045B8EB0200A94105D2FC
:1044B0004046214690461C460B46024623F00040EB
:1044C000104347D0270DC7F30A00C3F30A510290E7
:1044D000401A019040286BDAC3F3130040F4801BAC
:1044E0000098924620B10023D2EB030A63EB0B0B3A
:1044F00001985946C0F14002504600F0C2F9064604
:104500000D4650465946019A00F0DAF910EB0800C2
:104510006141002487EA115284EAE7731A4340D0CC
:10452000009A62B3019A012A4FEA075215DC001B78
:1045300061EB02014FF0004202EA0752CDE900426E
:10454000001C41F5801132462B4600F02DFA03B0D5
:10455000BDE8F08F40462146F9E7001B61EB020100
:10456000001C41F5801300185B412018A2F50017CC
:1045700047EB030140EAD570B6196D4111E06D08B3
:104580004FEA360645EAC0754FEA0752001B61EB59
:104590000201001C41F5801149084FEA3000001962
:1045A000514132462B4603B0BDE8F04F00F0EDB963
:1045B0000098012240000023D0EB020263EBE0737D
:1045C000009821464FEAE074B8EB000061EB04016B
:1045D000E9E783F000435BE781F0004158E72DE90C
:1045E000FE4F81EA030404F0004421F000410094EE
:1045F0004FF0000B23F0004350EA01045ED052EA72
:1046000003045BD0C3F30A54C1F30A552C44A4F24B
:10461000F3340194A0FB0254C1F3130141F480115F
:10462000C3F3130343F4801301FB024400FB034E66
:10463000840A970A44EA815447EA8357A4FB07682F
:1046400002958D0A05FB07854FEA932C04FB0C5459
:104650002705029D4FEA065847EA1637B5EB0805CD
:104660006EEB070C870E920E47EA811742EA83121F
:10467000A7FB0201B6EB0B0164EB00042B0D43EA30
:104680000C335E1844EB1C50DA465146E7FB02013E
:10469000C5F313044FEA0B3343EA14534FEA0432D1
:1046A000019C43EA0603A4F10C040294009CCDE9AA
:1046B00000B400F079F903B0BDE8F08F00200146A6
:1046C000F9E72DE9F04D81EA030404F0004B21F0F5
:1046D000004514464FF0000A23F0004150EA05025D
:1046E00020D054EA01021DD0C5F30A570246C5F393
:1046F0001303C1F31300C1F30A5640F4801543F4C9
:104700008013A7EB0608101BD64608F2FD3873EBA2
:10471000050002D308F1010801E092185B41B8F1ED
:10472000000F03DA00200146BDE8F08D00204FF4B1
:104730008011064684460EE0171B73EB050705D370
:10474000121B63EB050306434CEA010C49084FEAD0
:10475000300092185B4150EA0107EDD152EA0300A4
:1047600012D082EA040083EA0501084305D0101B39
:10477000AB4106D20122002306E000224FF00043A5
:1047800002E06FF0010253101AEB06004CEB0851E7
:1047900010EB0A0041EB0B01BDE8F04D00F0F5B85D
:1047A0000EB5C10F80EAE0700844CA07002140F24C
:1047B00033438DE80E000A460B4600F0F5F803B0CF
:1047C00000BDC1F30A5210B5C1F3130140F2FF332B
:1047D00041F480119A4201DA002010BD40F23343C7
:1047E0009A42A2F2334203DC524200F059F810BD63
:1047F000904010BD30B50B46014600202022012418
:1048000009E021FA02F59D4205D303FA02F5491B9E
:1048100004FA02F52844151EA2F10102F1DC30BDB4
:104820002DE9F05F0546002092469B4688460646E5
:10483000814640241BE0284641464746224600F078
:104840002FF853465A46C01A914110D311461846C4
:10485000224600F016F82D1A67EB01084F46224653
:104860000120002100F00DF817EB00094E41201E39
:10487000A4F10104DFDC484631462A464346BDE840
:10488000F09F202A04DB203A00FA02F10020704752
:104890009140C2F1200320FA03F31943904070477E
:1048A000202A04DB203A21FA02F00021704721FA85
:1048B00002F3D040C2F120029140084319467047EC
:1048C000202A06DBCB17203A41FA02F043EAE073D4
:1048D00006E041FA02F3D040C2F1200291400843C1
:1048E000194670470048704750B201082DE9F05F43
:1048F00082460078002715468B460AF10104B94626
:10490000302801D09DB113E014F8010B012778285D
:1049100003D0582801D045B10AE00DB1102D07D1C0
:104920000027102514F8010B02E0082500E00A25F5
:104930000026B0460EE005FB080005FB06F1012746
:1049400001EB10461FFA80F8B6F5803F00D3B94658
:1049500014F8010B294600F0B7F80028EBDABBF198
:10496000000F05D00FB1641E00E05446CBF80040A4
:10497000B9F1000F06D012F02DFF02210160C81E10
:10498000BDE8F09F48EA0640FAE710B5141E73F13F
:10499000000408DA401C41F1000192185B411A43FF
:1049A00001D120F0010010BD2DE9F04D92469B464B
:1049B00011B1B1FA81F202E0B0FA80F220329046F1
:1049C000FFF75FFF04460F4640EA0A0041EA0B0189
:1049D00053465A46084313D0114653EA010019D0F2
:1049E000C8F140025046FFF75BFF05460E465046B1
:1049F00059464246FFF745FF084305D0012004E031
:104A000020463946BDE8F08D0020054346EAE076B1
:104A10002C4337430A986305E40AA0EB0800002200
:104A2000FD0A44EA47540A3002D500200146E9E76E
:104A3000010510196941DDE9084500196941BDE822
:104A4000F04DA2E7C1F30A52C1F3130140F2FF3364
:104A500041F480119A4202DA00200146704740F288
:104A600033439A42A2F2334202DC5242FFF718BFAC
:104A7000FFF707BF30B5041E71F1000404DB4FF0EF
:104A80000044404264EB0101141E73F1000405DB95
:104A90001C464FF00043524263EB0403994208BFA7
:104AA000904230BD064C074D06E0E06840F001033F
:104AB00094E8070098471034AC42F6D3FFF74CFB5C
:104AC0002CB701084CB701083A2800D2303820F042
:104AD0002002412A01D3A2F13700884201D34FF0CE
:104AE000FF30704770B58C1810F8015B15F00703A4
:104AF00001D110F8013B2A1106D110F8012B03E077
:104B000010F8016B01F8016B5B1EF9D12B0705D47E
:104B10000023521E0DD401F8013BFAE710F8013BC7
:104B2000CB1A921C03E013F8015B01F8015B521EE3
:104B3000F9D5A142D8D3002070BD000000000000CC
:104B400000B587B0012148020AF0A4FF0121082026
:104B50000AF0A0FF0120ADF8040048208DF80700FE
:104B600001A9194802F08CFD642001F087FD0020A6
:104B70008DF8070001A9144802F082FDC82001F059
:104B80007DFD002002908DF80C008DF80D004FF493
:104B9000602004900020059001208DF8180002A9E3
:104BA0000A4800F02DF8002301221946074800F0BA
:104BB0004FF80121054800F00BF80121034800F0EF
:104BC000A3F807B000BD0000000801400024014028
:104BD00021B1826842F00102826003E0826822F023
:104BE0000102826070470146C86C80B2704702467D
:104BF000002013680B400BB1012000E0002070473B
:104C000030B502460020002350680F4C20400D793B
:104C10000C6844EA05242043506090680B4C204007
:104C2000D1E902542C434D7944EA45042043906075
:104C3000D06A20F470000C7C641EE4B2234340EA86
:104C40000350D06230BD0000FFFEF0FFFDF7F1FF22
:104C5000F0B504460D4600200021092D11DDE06865
:104C6000A5F10A0606EB4607072606FA07F1884370
:104C7000A5F10A0606EB460603FA06F10843E060D2
:104C80000CE0206905EB4507072606FA07F1884383
:104C900005EB450603FA06F108432061072A0FDAFF
:104CA000606B561E06EB86071F2606FA07F188433F
:104CB000561E06EB860605FA06F10843606322E0FD
:104CC0000D2A0FDA206BD61F06EB86071F2606FA81
:104CD00007F18843D61F06EB860605FA06F108435E
:104CE000206310E0E06AA2F10D0606EB86071F269E
:104CF00006FA07F18843A2F10D0606EB860605FACF
:104D000006F10843E062F0BD21B1826842F4A002DE
:104D1000826003E0826822F4A00282607047000093
:104D200070B505460C480068B0F1FF3F01D1002086
:104D300070BD03F0FBFB09480468601C632808DBB6
:104D400007A00DF095FFC82009F0DCF8022010F054
:104D500057F90120ECE70000180200201C02002097
:104D6000B5E7BBB0C8DDC1BFB2BBD7E300000000F0
:104D7000F0B504460A4625460CE003F00F071E1165
:104D8000304600F02FF802F8010B384600F02AF800
:104D900002F8010B15F8013B002BEED1002010703A
:104DA000F0BD2DE9F04706460C4637464FF00408A3
:104DB00011E017F8015B05F00F0A4FEA2519484684
:104DC00000F010F804F8010B504600F00BF804F85E
:104DD000010BA8F10108B8F1000FEAD10020207002
:104DE000BDE8F087002805DB092803DC00F130016D
:104DF000C8B208E00A2805DB0F2803DC00F15701E0
:104E0000C8B200E0FF2070472DE9F8430746884606
:104E10003846FFF7B1FA0646304606EBD071491026
:104E2000A6EB410111B10020BDE8F883002546E062
:104E300017F815008DF800006800401C385C8DF8EC
:104E4000010000242DE01DF8040030280ADB1DF8C5
:104E50000400392806DC1DF804003038C0B20DF813
:104E600004001CE01DF8040061280ADB1DF80400A2
:104E7000662806DC1DF804005738C0B20DF804009F
:104E80000DE01DF80400412809DB1DF80400462848
:104E900005DC1DF804003738C0B20DF80400601CB2
:104EA000C4B2022CCFDB9DF80000F02101EA001013
:104EB0009DF80110084308F80500681CC5B206EB10
:104EC000D671B5EB610FB3DB2846ADE7F0B5A3B003
:104ED00004465022F9490EA8FFF700FAF8A120462F
:104EE00008F0BAFA78B9E07B2C2806D004F10F005C
:104EF000FFF7B4FAF549086005E004F11000FFF788
:104F0000ADFAF2490860F2A1204608F0A5FA30B9DE
:104F1000204602F06DFD074612F0C4F8FDE2EEA156
:104F2000204608F099FA30B9204602F067FD07469E
:104F300012F0B8F8F1E2EAA1204608F08DFA90B933
:104F400004F10B00FFF78AFAE84908600846E8A276
:104F50002821036803A812F015FC012203A90020F0
:104F60000EF0A2FAD9E2E8A1204608F075FA68B975
:104F7000204603F0EFF8E7494870084640780228D9
:104F8000CCD10020887001F09DF9C6E2E2A1204654
:104F900008F062FA00BB02AA22A9204604F012FB24
:104FA0009DF88800012802D0022814D10EE09DF857
:104FB0000800D849887008468078022805D1D94869
:104FC000007820F01000D749087004E09DF8080030
:104FD00001F08CF900BFA0E2D3A1204608F03CFA12
:104FE000002857D101200346B7A20D21009020468A
:104FF00001F038FF0546B0F1FF3F8FD06019FFF791
:105000002DFAC0B2229001200346CAA20D210090C1
:10501000204601F027FF0546B0F1FF3F8AD0601916
:10502000FFF71CFA86B202200123C2A20D210090D4
:10503000204601F017FF0546B0F1FF3F92D09DF8E2
:105040008800012802D0022823D118E0605D7E2864
:105050000FD1A819401E205C7E280AD1711E6A1C3F
:10506000A01814F09BF886B26019314606F082F859
:1050700004E00122B0A100200EF016FA09E001229E
:10508000B2A100200EF010FA6019314601F04CF97F
:1050900000BF42E2B3A1204608F0DEF900289AD012
:1050A000B3A1204608F0D8F9002894D0B4A1204636
:1050B00008F0D2F990B9A07A3038C0B222909DF8A9
:1050C0008800012802D0022807D103E0022091497C
:1050D000887002E001F0F6F800BF1EE2ABA12046A6
:1050E00008F0BAF9D0BB04F10800FFF7B7F9A949F5
:1050F000087004F10B00FFF7B1F9A749087004F13B
:105100000E00FFF7ABF9A549087004F11100FFF795
:10511000A5F90830A249087008460078182803DB72
:10512000084600781838087004F11400FFF796F963
:105130009C49087004F11700FFF790F99A4908702C
:105140000846027897480178954800780DF00AF8EB
:10515000012296A100200EF0A7F9DEE1FFE796A15B
:10516000204608F079F9002846D1A079202803D1FB
:10517000E0798DF8340002E0A0798DF834009DF8D4
:1051800034308FA250210EA812F0FCFA9DF83400A2
:1051900030380A2824D2DFE800F005230A0F14195A
:1051A0002323231E89A10EA8FFF7BCF81DE08AA1C6
:1051B0000EA8FFF7B7F818E08AA10EA8FFF7B2F81B
:1051C00013E089A10EA8FFF7ADF80EE08AA10EA8A2
:1051D000FFF7A8F809E08AA10EA8FFF7A3F804E0FA
:1051E00088A10EA8FFF79EF800BF00BF01220EA9FC
:1051F00000200EF059F990E184A1204608F02CF926
:10520000002859D183A1601D08F026F918B90120A2
:1052100011F098FF81E181A1601D08F01DF918B916
:10522000022011F08FFF78E17FA1601D08F014F9D2
:1052300018B9022011F086FF6FE17DA1601D08F012
:105240000BF918B9022011F07DFF66E17AA1601D0B
:1052500008F002F918B9032011F074FF5DE179A19B
:10526000601D08F0F9F830B9002078490870042072
:1052700011F068FF51E176A1601D08F0EDF848B922
:1052800004F10900FFF7EAF870490870042011F0F2
:1052900059FF42E170A1601D08F0DEF818B9062040
:1052A00011F050FF39E16EA1601D08F0D5F820B96A
:1052B000072011F047FF30E1E1E0D7E030A201081C
:1052C0005E535953494E464F3A0000009003002068
:1052D0002B434353513A00002B4353513A000000F3
:1052E0002B4D4F444F445245583A00008C03002048
:1052F0004D6F646F647265785F4E657476616C752E
:10530000653D25640D0A00002B504F435F505050FF
:105310003A000000000100202B54435053544154E4
:1053200055533A00041F00202B5443505245435616
:105330003A0000002C000000556E6B6E6F776E20F7
:1053400050726F746F636F6C00000000636F6C6F5E
:105350006E7920636F6D696E672E2E2E2E2E2E2E87
:105360002E2E2E002B5443504F50454E3A00000035
:105370002B544350434C4F53453A4F4B00000000D1
:105380002B544350434C4F53453A00002B43434C5E
:105390004B3A000004000020050000200600002019
:1053A000030000200100002002000020557064610D
:1053B000746554696D6500005E4D4F44453A0000C8
:1053C0005B4D6F64652025635D0000004E6F2073A8
:1053D000657276657200000043444D41204D6F6454
:1053E0006500000047534D0054442D5343444D4144
:1053F0002F4556444F0000005743444D41000000E4
:105400004C544500556E6B6E6F7700005E4D5347F0
:105410003A0000005265616479000000687474709D
:105420003A657272000000005665724572720000A3
:105430007665723A657272006E6F6E657776657228
:10544000000000006C6F6164696E6700CE0200208E
:105450004842443A00000000446F6E6500000000BE
:10546000496E7374616C6C65640000002CA1601D52
:1054700007F0F2FF18BB052011F064FE4DE02AA1F1
:10548000204607F0E9FF38B901212A4880F8B9120F
:1054900000202949087240E028A1204607F0DCFFDF
:1054A00070B9284890F89C00022804D0254890F84C
:1054B0009C00032831D10121204612F073FE2CE01C
:1054C00021A1204607F0C8FF70B91E4890F89C0043
:1054D000022804D01B4890F89C0003281DD100210D
:1054E000204612F05FFE18E019A1204607F0B4FF35
:1054F00018B9A01D02F02CF80FE017A1204607F004
:10550000ABFF10B912F05CFF07E016A1204607F0D0
:10551000A3FF10B9601D03F037F823B0F0BD000001
:10552000776765743A0000002B504F433A5354415B
:105530005254000040390020402900202B474749A1
:10554000503A0000AB5600202B475049503A00001B
:105550002B464F54413A00002B504F433A57414B92
:10556000455550002B5544503A00000010B5012419
:105570001B48007830B1012808D002280AD003283F
:105580001DD118E017A007F023FE18E019A007F0BE
:105590001FFE14E01B48007830B100201949087044
:1055A00019A007F015FE05E001201649087019A0A2
:1055B00007F00EFE03E01AA007F00AFE00BF00BFCE
:1055C0001A480078012800D1032405480078401CBF
:1055D000C0B203490870A04201DD0020087010BD70
:1055E0002204002041542B4D4F444F445245583F14
:1055F0000D0A000041545E535953494E464F0D0A5F
:10560000000000002304002041542B474749503F2D
:105610000D0A000041542B475049503F0D0A00002D
:1056200041542B5544503F0D0A0000002800002033
:1056300010B59AB001220BA100200DF035FF072014
:1056400000900D48D0F81D100C4B4FF4817201A84A
:105650000EF096FB84B2224601A9012005F064FDFC
:105660001AB010BD52652D41757468656E7469631A
:105670006174696F6E210000C4150020A4590020D8
:105680002DE9F04707468846DFF8D890B8F1000FBB
:1056900033D1B86A00F58055334E002411E04FF441
:1056A00080622946484614F0F9FA4FF48062314688
:1056B000484614F069FB05F5806506F58066601CB8
:1056C000C4B2042CEBDBBD6A4FF4FF16002411E0DA
:1056D0004FF480622946484614F0E0FA4FF48062A5
:1056E0003146484614F050FB05F5806506F58066A6
:1056F000601CC4B2042CEBDB32E01B4DB86A00F531
:105700008056002411E04FF480622946484614F088
:10571000C5FA4FF480623146484614F035FB05F572
:10572000806506F58066601CC4B2042CEBDB4FF488
:10573000FF15BE6A002411E04FF4806229464846F6
:1057400014F0ACFA4FF480623146484614F01CFB6A
:1057500005F5806506F58066601CC4B2042CEBDBA1
:10576000BDE8F087C0C1002000F01F0008B501218E
:1057700005200AF08FF90220ADF8000018208DF8FE
:10578000030003208DF802006946054801F078FF08
:10579000202107200AF008FE00200249086008BD09
:1057A00000080140300000200448026804480188D5
:1057B00004A011F0D7FF00BFFEE700006800002042
:1057C000640000200D0A5B4246485D463D25642C7E
:1057D0004C3D25640000000010B504462CB303F0D6
:1057E0003DFB012111A00DF007F9012314229F2197
:1057F000002003F0D7FB104800680F49C98850F813
:105800002130302226210D4808F0A6FA0B4808F076
:1058100018FB012368229F21002003F0C3FB012312
:1058200007A26E21002003F029FE10BDC9BEB3FD02
:10583000BAC5C2EB00000000584700201C4B0020F6
:105840005B4D5DC8B7B6A820205B455849545DCD77
:10585000CBB3F6002DE9F041074602F067FE15488C
:10586000D0F8008014480068B0F1FF3F01D1BDE8D6
:10587000F0810026002515E00C2000FB067405EBE6
:10588000850000EBC50123460B220B4800680AF097
:1058900041FB0020E07209A12046FEF774FD00B133
:1058A000761C6D1C642DE7DB002020606060A0602A
:1058B00000BFDCE71C02002018020020303030302E
:1058C000303030303030300010B50B4800680B49B4
:1058D000884208D10AA00DF0CBF90C4800F0A4FFD3
:1058E00008200FF08DFB044800680949884202D166
:1058F00008200FF085FB10BDB80000202A04EC0042
:10590000C7EBC9D4BAF22E2E2E0000001F4B002088
:105910002A04F40010B50F4808F03AFA0E4800685F
:105920000E4988420CD10E4909680D4AD28851F8B7
:1059300022000849C91C00F0D9FA08200FF060FBCA
:10594000054800680749884202D108200FF058FB3B
:1059500010BD00001C4B0020B80000202A04EC0001
:10596000584700202A04F40010B504462CB303F075
:1059700075FA012111A00DF03FF8012314229F2197
:10598000002003F00FFB104800680F49C98850F849
:105990002130302226210D4808F0DEF90B4808F0AE
:1059A0002DFA012368229F21002003F0FBFA012336
:1059B00007A26E21002003F061FD10BDD0DEB8C447
:1059C000BAC5C2EB00000000584700201C4B002065
:1059D000205BC9CF5DB8C4D6B5205BCFC25DD3D242
:1059E000D2C6200010B50C4808F0D2F90B48006868
:1059F0000B49884206D108200FF002FB0648C01C64
:105A0000FFF78EF9054800680649884202D1082050
:105A10000FF0F6FA10BD00001C4B0020B80000206B
:105A20002A04EC002A04F40010B50446002C22D00D
:105A300003F014FA012110A00CF0DEFF0123142260
:105A40009F21002003F0AEFA0EA330222621104839
:105A500008F082F90E4808F0D1F9012368229F214D
:105A6000002003F09FFA00200A49088001230AA2BF
:105A70006E2103F003FD10BDD0C2D4F6BAC5C2EB4F
:105A800000000000313131313131313131313100FB
:105A90001C4B00204C020020205BC9CF5DB8C4D64F
:105AA000B5205BCFC25DD3D2D2C6200010B513485B
:105AB00006F0B8F804461248844214D10F484079E1
:105AC00020B1012806D002280CD107E00A200FF0EF
:105AD00097FA07E00B200FF093FA03E00C200FF089
:105AE0008FFA00BF08E0074800680749884203D1E1
:105AF000064948780FF084FA10BD000080020020AB
:105B00002A04EC00B80000202A04F400540100200C
:105B100010B504460CB303F0A1F901210FA00CF05D
:105B20006BFF012314229F21002003F03BFA012385
:105B300068229F21002003F035FA0B490B4806F03C
:105B400045F8012368229F21002003F02BFA01234E
:105B500007A26E21002003F091FC10BDB5E7BBB099
:105B6000D1A1CFEE000000003C0200208002002006
:105B70005B4D5DC8B7B6A820205B455849545DCD44
:105B8000CBB3F60010B50E4804F046FF04460D48AE
:105B9000204450B1B0F5002F03D0B0F5402F0CD108
:105BA00007E002200FF02CFA08E011200FF028FA8D
:105BB00004E009200FF024FA00E000BF00BF10BD90
:105BC00058470020D6FB13FF38B50546002D40D0BE
:105BD00000202149088003F041F901211FA00CF0A9
:105BE0000BFF012314229F21002003F0DBF91E4844
:105BF000FFF730FE002408E004EB44001A4901EBF3
:105C000080001A4941F82400641C642CF4DB184815
:105C10000068012808DD1748174B0022134900903F
:105C2000164804F027FE07E01248134B00221449DF
:105C30000090124804F01EFE012368229F210020DC
:105C400003F0B0F901230FA26E21002003F016FC2F
:105C500038BD00BFFCE7000022020020B5E7BBB062
:105C6000B9DCC0ED00000000384B0020E84F0020F8
:105C70001C020020785100202402002058470020F8
:105C80002C020020205B4D5DBAF4BDD02020205BAB
:105C9000535DD1A1CFEE200010B500200849088047
:105CA00004F098FA074800680749884206D00120A6
:105CB0000FF0A6F90120054981F8750010BD00001C
:105CC000A4020020B80000202A04FC00041F0020C9
:105CD000FEB50446142619A5012C2ED103F0BEF8FA
:105CE00000222946012005F021FF012120A00CF00F
:105CF00083FE012314229F21002003F053F9282161
:105D00001DA00CF079FE2048007800901F48037811
:105D10001FA2082101A811F035FD3C2101A80CF0BB
:105D20006BFE012368229F21002003F03BF9012331
:105D30001AA26E21102003F0A1FBFEBD443546449B
:105D40004434444142354533433346424133414371
:105D5000433745424230423443384345443245326A
:105D6000424346434338423743384346000000002D
:105D7000B5E3C3FB00000000B1BEB4CEB5E3C3FB86
:105D8000CAB1BCE4000000000100002003000020B4
:105D9000253032643A25303264000000B0B4C8CEF9
:105DA000D2E2BCFCCDEAB3C9B5E3C3FB00000000FE
:105DB00010B504462CB303F051F801211DA00CF0DE
:105DC0001BFE012314229F21002003F0EBF81C4846
:105DD00000681B49C98850F8213030222621194813
:105DE00007F0BAFF174808F02CF8012368229F211A
:105DF000002003F0D7F8012313A26E21002003F046
:105E00003DFB16480078022813D115A007F0E0F9F1
:105E100008200FF0F5F80020104908700120124901
:105E20000861002011490871C8704FF480700E4954
:105E3000486110BDB2A6B4F2B5E7BBB000000000E7
:105E4000584700201C4B00205B4D5DB2A6B4F220E9
:105E5000205B455849545DB9D2B6CF0020020020DE
:105E60004154480D0000000000100140402900206E
:105E700010B513A00CF0FCFE03F0E4FB6420DFF887
:105E80004CC000DF08200FF0BBF811480068114932
:105E9000884213D110A007F09BF908200FF0B0F84A
:105EA00000200F49087001200E49086100200E49AA
:105EB0000871C8704FF480700A49486110BD000035
:105EC000D4DDB2BBD6A7B3D60000000049930108C9
:105ED000B80000202A04F4004154480D00000000DE
:105EE00020020020001001404029002070B5054626
:105EF0000E4609480068B0F1FF3F01D1002070BD97
:105F0000284600F00BF80446B4F1FF3F01D1002011
:105F1000F5E70120F3E70000180200203EB5054632
:105F2000002414E004EB840000EBC4016B460B2258
:105F30000948006809F0EEFF00208DF80B00694663
:105F40002846FEF720FA08B920463EBD641C642CA2
:105F5000E8DB4FF0FF30F8E71802002010B5002012
:105F60000B4908700B48006844F63821884208DD68
:105F7000012007490870012207A100200DF094FAC2
:105F800004E0012206A100200DF08EFA10BD0000F1
:105F900028000020F8000020706F632D6F776E00DE
:105FA000706F632D7869616E0000000010B50446C3
:105FB000B4F5A07F17DA012214A100200DF074FAC5
:105FC0000120DFF860C000DF17484079012801D1C7
:105FD00012F070F9002014494871042013494861F7
:105FE0000DF004FA10E0B4F5A57F0ADA1048007845
:105FF000401CC0B20E4908701E2805DD0020087044
:1060000002E000200A49087010BD00005662617469
:10601000206C6F772173687574646F776E206E6F74
:106020007721000049930108402900200010014019
:106030008C00002000B585B0012306A2142168461B
:1060400011F0A0FB684607F0C3F8022006498870EB
:1060500005B000BD41542B544350434C4F53453D74
:1060600025640D0A000000000001002000B585B085
:106070000F48007820B1012807D002280FD109E08D
:106080000CA1684611F092FB0BE00DA1684611F0DF
:106090008DFB06E00DA1684611F088FB01E005B01C
:1060A00000BD00BF684601F0AFFA00BFF7E700008F
:1060B00024040020455652435F48414C46000000EE
:1060C000414D524E422D313232000000455652436E
:1060D0005F46554C4C0000002DE9F0479AB0002770
:1060E000B84646A001F0FCFEC7B2781C48B946A0ED
:1060F00011F038FB002049490870401E1AB0BDE875
:10610000F087384601F008FF06462EB944A011F08A
:1061100029FB6FF00100F1E710AB0E220021384699
:1061200009F0F8FE05460DAA42A110A802F0B2F946
:1061300005462DB941A011F015FB6FF00100DDE718
:106140000DA8FEF78BF935490870084600786428D9
:1061500009DD084601783DA011F004FB00202F491D
:106160000870C01ECAE72D4801783DA011F0FAFA68
:1061700000243CE0C4EBC40000EB400000F10E0141
:1061800010AB1522384609F0C5FE05462A4610A96F
:106190006846FEF7A3F800200DF80500E1B20AAB4F
:1061A0000DAA684601F0B4FC48B9012230A10020D4
:1061B0000DF07AF9002019490870001F9EE70AA81F
:1061C000FEF74CF91FFA80F90DA8FEF747F900F029
:1061D000FF0A4946504607F013F800F0FF08B8F1EF
:1061E000000F03D0414627A011F0BCFA641C0B48F5
:1061F0000078A042BEDC002080E70000636F646589
:10620000632E696E690000004E6F20636F646563E2
:106210002E696E692066696C650D0A007C0200209B
:10622000636F6465632E696E6920656D7074790DA6
:106230000A0000005245475F4E554D004E6F202723
:106240005245475F4E554D270D0A00005245475FA6
:106250004E554D204F5645523A25640D0A00000018
:106260005245475F4E554D3A25640D0A0000000027
:1062700063616E742066696E6420696E6465780D72
:106280000A00000053455420436F646563457272F1
:106290006F416464723D253032780D0A00000000C1
:1062A00000B50246012A00DD00BD0548007862F312
:1062B00000000349087000F005F800BFF4E7000093
:1062C000625600200848007820F002000649087055
:1062D000002081F833000846007820F004000870A0
:1062E00000204874887470476256002000B5034649
:1062F000012B01D1012200E000220A480078C0F3FE
:10630000800090420DD0012A03D1002005498874F5
:1063100001E0FFF7D7FF0348007862F382000149EC
:10632000087000BD625600207047000010B504469A
:1063300024B1012C26D0022C6CD147E0012236A1D9
:1063400000200DF0B1F80A20DFF8D8C000DF364891
:106350000470002240F22551344810F043F9012224
:1063600040F22441314810F03DF9002240F225511D
:106370002F4810F037F9012240F224412C4810F048
:1063800031F947E001222BA100200DF08DF80A2001
:10639000DFF890C000DF24480470012240F225514C
:1063A000224810F01FF9002240F224411F4810F04B
:1063B00019F9012240F22551214810F013F9002269
:1063C00040F224411E4810F00DF923E001221DA1E6
:1063D00000200DF069F80A20DFF848C000DF1248FD
:1063E0000470012240F22551104810F0FBF8002201
:1063F00040F224410D4810F0F5F8012240F22551F9
:106400000B4810F0EFF8002240F22441084810F049
:10641000E9F800BF00BF10BD434F4D3C2D2D3E4D50
:1064200043552100499301080C0000200038014029
:1064300000440040434F4D3C2D2D3E47505321001A
:1064400000480040434F4D3C2D2D3E4D6F64656D1F
:106450002100000010B510F025F810BD10B510F0A7
:106460003FF810BD00F0805111B10349086001E010
:1064700002494860704700000404024000000240E6
:1064800000F0805111B10349086001E00249486001
:1064900070470000040402400000024021B102687D
:1064A00042F00102026004E002684FF6FE731A40F7
:1064B0000260704701684FF6FE72114001600021D2
:1064C000016041608160C1604B49884208D14A49FE
:1064D0000839496841F00F01474A083A51608AE09B
:1064E00045491431884208D143490839496841F087
:1064F000F001414A083A51607DE03F492831884225
:1065000008D13D490839496841F470613A4A083A6E
:10651000516070E038493C31884208D13649083929
:10652000496841F47041344A083A516063E03249A5
:106530005031884208D130490839496841F4702106
:106540002D4A083A516056E02B496431884208D1FF
:1065500029490839496841F47001274A083A5160CD
:1065600049E025497831884208D1234908394968EA
:1065700041F07061204A083A51603CE01F4988426E
:1065800006D1011F096841F00F01021F116032E0BE
:106590001A491431884208D11849091F096841F085
:1065A000F001164A121F116025E014492831884273
:1065B00008D11249091F096841F470610F4A121F7E
:1065C000116018E00D493C31884208D10B49091F80
:1065D000096841F47041094A121F11600BE0074934
:1065E0005031884207D10549091F096841F47021DB
:1065F000024A121F1160704708000240080402405E
:1066000001460020002201F0805313B1054B1A68A7
:1066100001E0054B1A6802EA01030BB1012000E01A
:106620000020704700040240000002401AB10368D5
:106630000B43036002E003688B430360704710B5AF
:106640000022026847F6F0739A430C6A8B68234372
:106650000C6923434C6923438C692343CC6923434E
:106660004C6A23438C6A23431A430260CB6843601D
:106670000B6883604B68C36010BD704710B54FF462
:106680002F73002109E0002201E000BF521C03F536
:106690009654A242F9D34C1CA1B28142F3DB10BD47
:1066A00001461CE000BF00BF00BF00BF00BF00BF2D
:1066B00000BF00BF00BF00BF00BF00BF00BF00BFE2
:1066C00000BF00BF00BF00BF00BF00BF00BF00BFD2
:1066D00000BF00BF00BF00BF00BF00BF00BF0A1E59
:1066E000A1F1010399B2DDD17047000070B586B009
:1066F00002AC02AE4A48C1884A4800EB81000068FB
:10670000009010222046009913F0C8FA9DF8090065
:10671000012812D143481638808870B14148163894
:106720008088401E3F49163988800846808820B9F5
:106730000846007820F0010008703A481638408872
:1067400030B1384816384088401E364916394880DE
:10675000344816380078C0F3800060B131481638EC
:1067600000788008401E2F491639097860F38201AD
:106770002C48163801702B481638D0F806000099BE
:1067800088420FD005AD049800F10C010422284680
:1067900013F0FAFA04AD059800F108010422284626
:1067A00013F0F2FA00200190012201A8009913F0E1
:1067B000EBFA1C481638D0F806000099884228D019
:1067C00018481638D0F806101022204613F066FA42
:1067D00014481638D0F8060000F108010422684673
:1067E00013F0D2FA049800F10C010422684613F069
:1067F000CBFA009800F10801042204A813F0C4FAAF
:10680000009800F10C0104220648103813F0BCFA7D
:1068100004E0044916390598C1F8060006B070BDB9
:10682000584700206A5200203EB5054619480068C6
:10683000B0F1FF3F01D100203EBD2846FFF76EFBBF
:106840000446B4F1FF3F01D10020F5E700208DF8A8
:106850000B0019E0052094FBF0F100FB114008B992
:1068600002F0F0FE601C00EB800202EBC0016B4600
:106870000B220848006809F04DFB641C06A168461D
:10688000FDF781FD00B901E0632CE3DB00BF0120CF
:10689000D2E7000018020020303030303030303085
:1068A0003030300028B10021054A1170054A1160CE
:1068B00004E00121024A1170024A11607047000091
:1068C00040040020A002002010B54FF4007000F03A
:1068D00023F801280DD107480078012805D10420AC
:1068E000054908610120054908704FF4007000F067
:1068F00007F810BD3C000020001001403D000020C2
:106900000149086070470000140401400149086013
:10691000704700001404014001460020034A126839
:106920000A400AB1012000E0002070471404014031
:10693000002123498279002A3AD00A461268036866
:106940009A430B461A600A1D126803689A430B1D8E
:106950001A60027911440A6803681A430A60184AE7
:106960000832126803689A43154B08331A601A1DDF
:10697000126803689A43124B0C331A604279102A4A
:106980000ED11A1F126803681A430D4B08331A60A0
:106990001A1D126803681A43094B0C331A600DE084
:1069A0000749427911440A6803681A430A6005E0FE
:1069B000027911440A6803689A430A60704700002C
:1069C0000004014010B50C240020FFF769FC0020F2
:1069D000174908700CF08EFE21464FF47A7009F0CA
:1069E00039FF2046DFF84CC000DF0CF083FE214663
:1069F0004FF4FA7009F02EFF2046DFF838C000DFB0
:106A00000CF078FE21464FF47A7009F023FF012044
:106A1000094908700FF0D2FE012003F027FE08207C
:106A20000AF02CFC012205A100200CF03DFD10BD58
:106A300034010020499301080D0000205B456E746D
:106A4000657254784D6F64655D00000010B50020DC
:106A500000F03AFD06200EF0D3FA10BD30B5044622
:106A600004254FF4302000F06FF80546042D17D1AF
:106A70000C48006940F002000A4908610846446178
:106A8000006940F0400008614FF4302000F05CF8ED
:106A900005460448006941F6FD7108400149086156
:106AA000284630BD0020024004200B49C96801F08F
:106AB000010109B101200EE00749C96801F0040194
:106AC00009B1022007E00449C96801F0100109B1C9
:106AD000032000E0042070470020024003480069C2
:106AE00040F080000149086170470000002002402A
:106AF00070B504460D460426F00200F025F806465F
:106B0000042E11D10948006940F0010007490861CD
:106B10002580F00200F018F806460448006941F6A6
:106B2000FE71084001490861304670BD00200240F6
:106B3000024803494860034848607047230167459D
:106B400000200240AB89EFCD00B502460423FFF7D9
:106B5000ABFF034603E0FFF7A7FF0346521E012BDE
:106B600001D1002AF7D102B90523184600BD10B59E
:106B700000F002F810BD00002DE9F0418CB04FF09C
:106B800000084FF478617A48FDF7C1FB0024002625
:106B900042E030223146684613F080F875490B9880
:106BA000884232D104EB440101EBC4027049083140
:106BB00001EB820014226946FDF790FB04EB4401CF
:106BC00001EBC4026A49083101EB820101F11400B2
:106BD000102205A9FDF782FB04EB440000EBC40280
:106BE0006348083000EB82000999416204EB4400DD
:106BF00000EBC4015E48083000EB81008662641C33
:106C00000A9808B10A9E07E009E05B490B988842A0
:106C100000D104E006F5805658488642B9DB00BF33
:106C200053484460012C06DA55A010F09BFD01206A
:106C30000CB0BDE8F08156484D490860042549680C
:106C4000491E01EB410202EBC1024949083101EB47
:106C5000820050A1FDF797FB70B945494968491E6C
:106C600001EB410202EBC1024149083101EB820113
:106C7000886A11F0AFFC054604274FF4FF1011F0AD
:106C8000A9FC07462DB943A144A010F06BFD0020DC
:106C9000CEE7002F64D1042D05D13EA141A010F014
:106CA00061FD002604E03BA143A010F05BFD01263E
:106CB00030224FF4FF11684612F0F0FF04EB44015C
:106CC00001EBC4022A49083101EB82001422694613
:106CD000FDF704FB04EB440101EBC4022449083135
:106CE00001EB820101F11400102205A9FDF7F6FA6B
:106CF00004EB440000EBC4021D48083000EB8200A6
:106D000009994162601E801B00EB400202EBC00249
:106D10001748083000EB8200816A3022684612F082
:106D2000BDFF04EB440000EBC4021148083000EB47
:106D300082000A998162A11B01EB410202EBC102B0
:106D40000B49083101EB82000121FEF799FC042D6B
:106D500004D107484068401C05494860002067E7A7
:106D60003B462A460BA11AA010F0FCFC02205FE76C
:106D700040B20020311B200812EFCDABFFDF1F0017
:106D80004E6F207265732066696C65730D0A000092
:106D9000F8DEBC8A7379732E696E69002573206FE3
:106DA0006B0D0A002573206C6F73742C2072656361
:106DB0006F7665720D0A0000257320696E76616C2E
:106DC00069642C207265636F7665720D0A0000009D
:106DD0002573206572726F722C20737461747573E1
:106DE0003A25642C25640D0A000000002DE9F04FBF
:106DF0000146C1F3074CC1F3072801F0FF09DFF892
:106E00005CA00020002224E09300DFF854B01BF8BF
:106E1000035003F1010E1BF80E6003F1020E1BF884
:106E20000E40A9EB0505002D00DA6D42A8EB060621
:106E3000002E00DA7642ACEB0404002C00DA644247
:106E400005EB060B0BEB0407574501DABA46104673
:106E5000521CFF2AD8DDBDE8F08F00003F420F0032
:106E6000405E00202DE9F04704460E4617461D46B9
:106E7000DDF820A04FF00008C14615E02A4639464B
:106E80002046FDF78EFA50B909F1010000F0FF0924
:106E9000D14504D108EB050000B2BDE8F087641CC1
:106EA00008F101001FFA80F82078B042E6D14FF0D7
:106EB000FF30F2E710B502F0C5FB3748007800B9A3
:106EC00010BD36484078F0B134480078A8B934484D
:106ED0000078C0EB0010840030484089401C80B22C
:106EE0002E494881A0421BDD0020488101222DA1AE
:106EF0000CF0DAFA09F01AF912E00020274948816B
:106F00002F4908700CE025484089401C80B2234975
:106F10004881B0F5616F03DD0020488109F006F972
:106F20001E484079012816D11C48007A10B900206B
:106F3000244908701948007A401CC0B217490872E9
:106F4000282808DD0120087201221FA100200CF072
:106F5000ABFA09F0EBF82448007800F001000028B3
:106F600018DD22480068A8B11F484078401CC0B214
:106F70001D4948700A280DDD0020487001221CA11F
:106F80000CF092FA00F05EFC01F016FF0FF034FFF7
:106F90000CF0C4FE00BF93E734010020402900201C
:106FA0005D000020506F634C6F737454696D656FA2
:106FB0007574215265736574204D6F64656D210091
:106FC0008D0000208E0000204D6F64656D5265635A
:106FD0007654696D656F7574215265736574204DC3
:106FE0006F64656D21000000041F0020A0020020D6
:106FF000475053207265626F6F742D2D0D0A00008B
:10700000F0B585B054239F222C21002001F080FF91
:10701000012042238022322100901D2001F0D9FF5F
:1070200000252048D0F8067001AE00242CE0102284
:107030003946304612F032FE9DF80400012807D18F
:1070400000208DF8040001223946304612F09CFEE3
:10705000049F0A2094FBF0F100FB114008B902F0F4
:10706000F1FA0A2094FBF0F100FB114050B9012025
:1070700005F11D02034640210090342001F0D5FFA8
:10708000681CC5B2601C84B2B4F57A7FCFDB0020E7
:107090000449488088800846007820F00100087084
:1070A00005B0F0BD545200202DE9F04F95B00746D1
:1070B000CCA1384606F0D0F9A0B90321384600F03B
:1070C0006BFF8346BBF1010F03D10120C849087053
:1070D00005E0BBF1020F02D10020C549087015B0D0
:1070E000BDE8F08FC3A1384606F0B6F950B9B87ABA
:1070F000332807D10020BE4908700122C0A10CF03E
:10710000D3F9ECE7BA48007800B9E8E702F09AFA58
:107110000323BFA23C2106A810F034FB0B2206A9D2
:107120003846FDF754F900B1D9E707F10B00FDF738
:1071300095F985B2052D00DAD1E70A2D02DA07F1BB
:107140000D0412E0642D02DA07F10E040DE0B5F52E
:107150007A7F02DA07F10F0407E042F210708542ED
:1071600002DA07F1100400E0B9E7AD48007830BB5F
:107170002078AB2805D00122AAA100200CF094F9B8
:10718000ADE7A0788DF81500E0788DF81400BDF813
:107190001460301D85420DDA2A462146A348FDF7CA
:1071A0009DF8A348058001209D490870301DA14924
:1071B000088094E7301D854200D128E08FE79C4885
:1071C000008828449B490988884217D1994800883B
:1071D00040F20B4188420BD89449954A128888188E
:1071E0002A462146FDF77AF8904C924805880EE031
:1071F000012291A100200CF057F970E7012291A122
:1072000000200CF051F900208549087067E72078CC
:10721000AB2805D001228DA100200CF045F95EE7D6
:1072200060780290A0788DF81500E0788DF8140051
:10723000BDF81460301D854205D0012285A10020D3
:107240000CF032F94BE700200190814608E014F879
:10725000090001994840019009F101001FFA80F9E5
:10726000F01C8145F3DB215C0198814205D00122AD
:107270007AA100200CF018F931E702986B2802D0AF
:107280007B2842D15AE000205949488004F1040883
:10729000283108F10200FDF776F828B1012271A12A
:1072A00000200CF001F91AE7D8F8160004909DF8B8
:1072B00013008DF80C009DF812008DF80D009DF85C
:1072C00011008DF80E009DF810008DF80F00484950
:1072D0000398086198F80000087398F80100487353
:1072E000102208F11A0142481830FCF7F7FF404815
:1072F000006958B903203E49C87201225DA10020EF
:107300000CF0D2F8C22006F01FFD67E03848007C80
:1073100000F0010020B1012258A100200CF0C4F8B7
:10732000252006F011FD00203149486101208871B7
:1073300048694FF4806102F017FA4FE000202C49B1
:10734000488020798DF8130060798DF81200A079BB
:107350008DF81100E0798DF81000DDF810A0207A8A
:107360008DF81500607A8DF81400BDF81450E81DF2
:10737000864204D0012246A110460CF095F80AF589
:1073800000102A4604F10A0102F076F90AEB050022
:1073900017490969884208D3012244A100200CF052
:1073A00083F8472006F0D0FC17E0012002F0B0F887
:1073B0000F4843A23C21436906A810F0E3F90122DB
:1073C00006A900200CF070F80AEB05000849486196
:1073D00048694FF4806102F0C7F900BF00BF00BFE9
:1073E0007DE600002B5443505354415455533A000A
:1073F000E05900202B544350434C4F53453A000072
:10740000466F74612054435020636C6F7365640051
:107410002B544350524543563A25642C000000003B
:107420004C0400204845727231000000285A0020A8
:10743000480400204A0400204275666665724F7653
:1074400065720000574C656E457272004845727255
:10745000320000006C656E457272000053756D4518
:107460007272000046696C654E616D6520657272CE
:107470006F7221004E6F2066696C6500464C656E28
:10748000206973206E6F74206576656E21000000A0
:10749000526563762066696C652064617461206C56
:1074A000656E206572726F7221000000446F776C08
:1074B0006F616420636F6D706C6563746564210037
:1074C0004842443D2564000010B590B0044674B1B4
:1074D00042F2B1300FA1032312A2CDE900103221F4
:1074E00003A810F04FF92046FFF7DCF908E003236A
:1074F00012A2322103A810F045F92046FFF7D2F975
:1075000003A805F065FE002203A910460BF0CCFF8E
:1075100010B010BD3132302E37372E36362E313284
:107520003900000041542B5443504F50454E3D25E7
:10753000642C25733A25640D0A00000041542B5435
:107540004350434C4F53453D25640D0A0000000055
:1075500010B5044620783038052830D2DFE800F036
:107560002203090D1100A01CFCF778FF15490860E3
:1075700025E015A000F048F821E016A000F044F83E
:107580001DE017A000F040F80121184880F8B9125A
:10759000012017490870DFF85CC000DF96301649FB
:1075A00008600CE015A000F02FF8012010490870C9
:1075B000DFF840C000DF96300F49086000BF00BF11
:1075C00010BD000028040020D5FDD4DAC9FDBCB6EA
:1075D0002E2E2E00D5FDD4DAB0B2D7B02E2E2E002E
:1075E000D5FDD4DAD6D8C6F42E2E2E004039002090
:1075F0002C040020B199010830040020CAA7B0DC97
:10760000CDCBB3F60000000070B505460122294637
:1076100000200BF049FF2846FCF7AEFEA021A1EBAD
:10762000C0004608402421461023A022002001F07B
:1076300029FC2146B0B201232A4601F01FFF70BD8C
:1076400030B500228B071C0F0F2303FA04F20B4BFB
:107650008C1053F824309343084C8D1044F8253097
:1076600023468C1053F824308C07240F00FA04F4BE
:107670002343024C8D1044F8253030BD08000140F2
:107680002DE9F041024600250026002000230024B9
:10769000002791F803C00CF00F0591F803C00CF01F
:1076A000100CBCF1000F03D091F802C04CEA0505A4
:1076B00091F800C0BCF1000F31D0146800202BE01D
:1076C0004FF0010C0CFA00F3B1F800C00CEA03060D
:1076D0009E4220D183004FF00F0C0CFA03F7BC43FD
:1076E00005FA03FC4CEA040491F803C0BCF1280F2E
:1076F00006D14FF0010C0CFA00FCC2F814C00AE0ED
:1077000091F803C0BCF1480F05D14FF0010C0CFA01
:1077100000FCC2F810C0401C0828D1D31460B1F896
:1077200000C0BCF1FF0F34DD546800202EE000F1F2
:10773000080C4FF0010808FA0CF3B1F800C00CEA8D
:1077400003069E4221D183004FF00F0C0CFA03F781
:10775000BC4305FA03FC4CEA040491F803C0BCF1F5
:10776000280F05D100F1080C08FA0CF8C2F81480B3
:1077700091F803C0BCF1480F07D100F1080C4FF09D
:10778000010808FA0CF8C2F81080401C0828CED373
:107790005460BDE8F0810000F0B50A4600230024E3
:1077A0000021002500F00046B6F1004F02D11D4E29
:1077B000F16901E01B4E7168C0F3034583B200F428
:1077C0004016B6F5401F08D121F07061154E76685D
:1077D00026F07066134F7E6012E000F48016B6F556
:1077E000801F06D1032606FA05F4A14341F070611B
:1077F00006E0460D360103FA06F6B14341F070612A
:1078000022B1460D360103FA06F6314300F0004678
:10781000B6F1004F02D1034EF16101E0014E7160FB
:10782000F0BD0000000001400246002093680B40BC
:107830000BB1012000E000207047416170470161F9
:107840007047000008B510208DF8030003208DF864
:1078500002004FF40070ADF8000069460448FFF7DD
:107860000FFF012203A100200BF01EFE002008BD27
:10787000001001405B31335D475053496E69742EEF
:107880002E2E000010B515480078022800D110BD3A
:10789000134800681349884217D11048007840B94E
:1078A0000020114908700D480078401C0B490870F1
:1078B00012E00D48007803280EDDFFF783F8074833
:1078C0000078401C0549087006E00448007801284B
:1078D00002D100200149087000BFD8E77B000020DA
:1078E000B80000202A04B400BD0000202DE9F041BA
:1078F00094B004466079382874D1A079302871D1C9
:1079000004F11D00FCF738FD801EC6B2482E00DBD6
:107910004826324604F11D0101A8FCF7DFFC0020D7
:1079200001A9885560771022694604F11900FCF717
:107930005DFD87B2002060761022694604F11100D7
:10794000FCF754FD8046002060741022694604F163
:107950000D00FCF74BFD85B2642D03DB012014B054
:10796000BDE8F0811DB901201F49086704E01E48E9
:10797000006F401C1C49086705EB450000EBC50182
:107980001A4840F8218005EB450000EBC501174877
:1079900000EB810087809DF8040090B9202105EB61
:1079A000450000EBC502114800EB82008171002107
:1079B00005EB450000EBC5020C4800EB8200C171ED
:1079C0000AE005EB450000EBC502084800EB820029
:1079D000811D01A80BF014FF0120034981F86D00FF
:1079E000BDE7FFE70020BAE740290020BC2A0020BD
:1079F00010B50446E01DFCF731FD10BD10B504467E
:107A0000A01DFCF72BFD10BD0146024850F82100D7
:107A100070470000100300202DE9F04F8BB0804626
:107A20008B4691463448834503D200200BB0BDE815
:107A3000F08F4846FCF7A0FC07460E2F07D00F2F0B
:107A400005D04B462DA2102108A80FF09BFE5B46E7
:107A50002CA20C2108A80FF095FE08A8FCF78CFCBE
:107A600000900025A7F10A0405E019F8040004A914
:107A700048556D1C641CBC42F7DB0026B24600244E
:107A800007E008A8005D464004A8005D80EA0A0AF5
:107A9000641C0A2CF5DB86EA0A061C4810F806A0CE
:107AA00000240CE008A8005D80EA0A0604A8005D36
:107AB000704001A90855154810F806A0641C0A2C4E
:107AC000F0DB002504240FE001A8005D0A2190FBF3
:107AD000F1F201FB120008F8050018F8050030303B
:107AE00008F805006D1C641C0A2CEDDB002088F8EA
:107AF000060001209AE700002058F20825303135B1
:107B00006C750000253031306C750000909F0108C5
:107B10002DE9F0479CB082460F4690461E464FF036
:107B20000009781CC7B23B462EA20F2118A80FF0FF
:107B300029FE002218A910460BF0B6FC08AA18A9C5
:107B4000504600F0A7FCC4B21CB900201CB0BDE830
:107B5000F08700250CE008A8405D2C2806D1681CA1
:107B600000F0FF09002008A948552546681CC5B249
:107B7000A542F0DB08A8FCF7FFFBC4B21E2C00DD19
:107B80001E24224608A94046FCF7A8FB002008F85E
:107B90000400424616A168460FF008FE002269461E
:107BA00010460BF081FC08A901EB0900FCF7E4FB8F
:107BB000C4B21E2C00DD1E2408A800EB09012246D9
:107BC0003046FCF78BFB00203055324608A1684652
:107BD0000FF0ECFD0122694600200BF065FC01204E
:107BE000B4E70000434F44454325303364000000B0
:107BF0003D3D3D25730000002DE9F14FA0B0002070
:107C0000159003F055FF16A99848FDF7CAF8002013
:107C10001490002404E016A8005D14A90855641C03
:107C2000032CF8DB14A8FCF719FC82460020119005
:107C30001290002405E016A9E01C085C11A9085563
:107C4000641C062CF7DB11A8FCF708FC83464FF4F4
:107C50007A709BFBF0F00590FCF7A2FDCDE90C01DA
:107C60000022834BDDE90C01FCF72BFDCDE90C0173
:107C70004FF47A709BFBF0F100FB11B0C0EB0010E9
:107C800080000590FCF78CFDCDE90A010022794BBC
:107C9000DDE90A01FCF715FDCDE90A01DDE90A235A
:107CA000DDE90C01FCF7F4FB05460E460022724BA1
:107CB00028463146FCF793FCCDE902016F490AFBE7
:107CC00001F0FCF76DFDCDE90001DDE90223FCF7D1
:107CD000DFFBCDE90401FCF774FD6949486615A98D
:107CE0006248001FFDF75DF8002404E015A8005D60
:107CF00013A90855641C032CF8DB13A8FCF7AEFB92
:107D00008146002405E015A9E01C085C0FA9085570
:107D1000641C062CF7DB0FA8FCF7A0FB0E904FF4B9
:107D20007A710E9890FBF1F00590FCF739FDCDE9E2
:107D3000080100224E4BDDE90801FCF7C2FCCDE949
:107D400008014FF47A710E9890FBF1F201FB1200DA
:107D5000C0EB001080000590FCF722FDCDE9060184
:107D60000022444BDDE90601FCF7ABFCCDE906013E
:107D7000DDE90623DDE90801FCF78AFB07468846B2
:107D800000223D4B38464146FCF729FCCDE9020173
:107D90003A4909FB01F0FCF703FDCDE90001DDE9FB
:107DA0000223FCF775FBCDE90401FCF70AFD344919
:107DB00088662098002856D10022324B384641462A
:107DC000FCF70DFCCDE90201FCF7FBFC05902EA3AE
:107DD0002EA21E21CDE9009018A80FF0D3FC01239C
:107DE00018AA1821002001F049FB0022254B284643
:107DF0003146FCF7F4FBCDE90201FCF7E2FC05900B
:107E000027A328A21E21CDE900A018A80FF0BAFCD4
:107E1000012318AA2821002001F030FB1848437CD8
:107E200025A21E2118A80FF0ADFC012318AA3821A5
:107E3000002001F023FB124890F87400012812D1B1
:107E40000F48006F6421B0FBF1F0C01C03461FA275
:107E50001E21059018A80FF095FC012318AA4821AF
:107E6000002001F00BFB21B0BDE8F08F145400207E
:107E700000004E4040774B4180842E4140420F002D
:107E8000041F0020006AF8405300000020CEB3B663
:107E9000C82025733A20252E33642E253035640002
:107EA0005700000020BEADB6C82025733A202564D7
:107EB0002E2530356400000020CEC0D0C7CAFD3A60
:107EC000202530326420B8F600000000BFAABBFABB
:107ED000B6A8CEBBCAB1BCE43A256420530000006A
:107EE00070B5054600240DE004EB440101EBC4022B
:107EF000084901EB82002946FCF745FA08B92046FB
:107F000070BD641C034808384068A042ECD84FF0AC
:107F1000FF30F5E748B200200246002A01DA0020CF
:107F2000704702EB420000EBC203064800EB8300FF
:107F3000416A002902DB0448814201DD0020EFE7AD
:107F40000846EDE748B20020FFCF1F002DE9F047BB
:107F500004460D461646A02C01DBA02D02DA0020B7
:107F6000BDE8F087A4F1A000C7B2A5F1A00000F021
:107F7000FF09A9F10100791E5E2202FB01004FEA10
:107F800040180449334620224868414607F0C2FFA2
:107F9000E6E70000345E00202DE9F04104460D467E
:107FA000022604F10B00FCF759FAC7B2607B3128B6
:107FB00001D1012603E0607B302800D10226AF42C8
:107FC00002D13046BDE8F0810020FBE710B53D4806
:107FD0000078401CC0B23B490870022801DD002037
:107FE00008703848007820B902F0E2F83649086095
:107FF00003E002F0DDF83549086033480068334992
:108000000968884201D0002010BD314800682E491F
:108010000968884219D02C4800682D490860084634
:1080200000682C49884206D001202B4908700020A6
:108030002A49087009E02648016829A00FF092FB40
:10804000002025490870294908702348007858B352
:108050002748007888B1274800781F490978884266
:1080600009D01D4800782349087019480068224942
:1080700008600120C8E70020C6E7174800781D49BE
:1080800008701E48007840B90F4800681A49086017
:1080900064201A4908700120B6E718480078401E8D
:1080A000164908700020AFE70020144908701148F5
:1080B000007820B100200F490870401EA4E700207E
:1080C000A2E70000CD000020D4000020D80000204E
:1080D000D00000202A04FC00CE000020BD000020BB
:1080E0004B45593D256C780D0A000000BC0000206E
:1080F000BF000020CF000020B8000020CC000020EE
:1081000000B589B00B480C49097800EB81000B4998
:1081100091F8F612435C0AA21E2101A80FF032FB6F
:10812000012201A900200BF0BFF901A805F050F8C9
:1081300009B000BDAEA101083F010020AB560020F0
:1081400041542B4D4F444F445245583D25640D0A30
:10815000000000000146487A312801D10120704713
:108160000220FCE72DE9F74F90B00546BB48408858
:10817000052802DB4FF0050902E0B84890F80290AC
:108180004FF0000B002009904FF47A780DF1280A87
:108190001198012812D1B148D0F80600AF49C1F8B2
:1081A00012000846D0F806101022504611F076FD55
:1081B000AA490C98C1F80E000020119000241298D2
:1081C00064287CD176E0A548D0F812701022394698
:1081D000504611F063FD082207F110010EA811F0BE
:1081E0005DFD9DF8280001284DD1BBF1000F07D19E
:1081F0000BF1010000F0FF0B98490C98C1F80E003C
:10820000DDF82A00C0F344400090DDF82A10C1F3E5
:1082100083534FF03F0C0CEA916204EBC40C05F160
:10822000DE0101EB4C008EA10FF0C0FA04EBC4029A
:1082300005F1DE0101EB42000EA9FCF773F89DF891
:108240002900012808D1002104EBC40205F1DE0059
:1082500000EB4200417407E0012104EBC40205F188
:10826000DE0000EB420041747C490D98C1F8120019
:1082700001F1160000EB84000760601CC4B24C459D
:1082800008DB264617E07548D0F806007349C1F8A8
:1082900012000FE0A8F101001FFA80F8B8F1000FFA
:1082A00007D1012272A100200BF0FEF8264602E061
:1082B00005E000BF87E700BF0020E880BEE072E075
:1082C0006648D0F80E7010223946504611F0E6FC90
:1082D000082207F110010EA811F0E0FC9DF828001B
:1082E00001284CD1099838B90998401CC0B20990AE
:1082F0005A490D98C1F81200DDF82A00C0F3444035
:108300000090DDF82A10C1F383534FF03F0C0CEAC4
:10831000916204EBC40C05F1DE0101EB4C0057A1A6
:108320000FF044FA04EBC40205F1DE0101EB420058
:108330000EA9FBF7F7FF9DF82900012808D10021BD
:1083400004EBC40205F1DE0000EB4200417407E0DB
:10835000012104EBC40205F1DE0000EB4200417490
:108360003E490C98C1F80E0001F1160000EB8400A4
:108370000760601CC4B24C4506DB264614E0374952
:108380000C98C1F80E000EE0A8F101001FFA80F869
:10839000B8F1000F06D101223BA100200BF084F8B8
:1083A000264601E000BF8BE700BF0DF1100A304602
:1083B00006EBD071C1F347010391002438E004EBD0
:1083C000C40105F1DE0000EB41000290701E001BAD
:1083D00000EBC00105F1DE0000EB4100019012222C
:1083E00050460299FBF77AFF1222DDE90110FBF7F4
:1083F00075FF122251460198FBF770FF174816309F
:1084000000EB84000768701E011B1448163000EB57
:10841000810001681148163000EB84000160701E75
:10842000011B0E48163000EB81000760601CC4B2CF
:1084300003988442C3DBA9F10100E880AE800020EC
:1084400085F83E01B5F83A11B5F83C0102F09CFA06
:10845000284602F09BFD13B0BDE8F08F5452002077
:10846000253032642F253032642F253032642000CD
:108470005B534D535D6572723100000025642F25FA
:10848000642F2564200000005B534D535D657272BC
:10849000320000002DE9F04F87B082460E461746A5
:1084A0004FF000090024A3469AF8000008B1307884
:1084B00018B9002007B0BDE8F08F0FE058460BF167
:1084C000010B01A901F80080B8F13D0F02D0B8F10D
:1084D0003B0F01D10020EDE7761C641C96F800806C
:1084E000B8F1000F01D0142CE8DB3D222046641CBB
:1084F00001A90A54002008555046FBF71FFF054606
:10850000254405E0287838706D1C7F1C09F10109AD
:108510002878202805DD28783B2802D0B9F1500FB3
:10852000F0DD002038704846C4E700003EB500206A
:1085300010490860002417E004EB840000EBC4013C
:108540006B460B220C48006807F0E4FC00208DF815
:108550000B000AA16846FBF716FF20B1054800682A
:10856000401C04490860641C642CE5DB0148006879
:108570003EBD00001C0200201802002030303030C8
:1085800030303030303030002DE9F04105460227E0
:1085900043E0E85D2C283ED1A81CFBF75FFF0646B0
:1085A000E919481CFBF75AFF0446052E0BD1192C7C
:1085B00009D1224890F82F03012804D001201F4937
:1085C00081F82F0330E0052E0BD1372C09D11B4841
:1085D00090F82F03022804D00220184981F82F03B5
:1085E00022E0052E0AD1052C08D1144890F82F035B
:1085F00020B10020114981F82F0315E0192C0AD071
:10860000372C08D0052C06D00526052400200B4960
:1086100081F82F0308E0781C07B22846FBF7ACFE70
:10862000B842B6D8BDE8F081044991F82F0304F0B0
:108630004BFE002005F0B8F900BFF3E7AB56002071
:108640000021064A00BF05E013780370401C521C4D
:108650004B1CD9B20C29F7DB70470000E8F7FF1F6D
:10866000024600210CE04D2B03D101F1100081B234
:1086700002E001F1080081B29F2901DD9F2103E0A2
:1086800012F8013B002BEED100BFC8B270470000CA
:10869000F0B589B0074617B9002009B0F0BD06A8AB
:1086A000FFF7CEFF1BA00FF05DF8002406E006A840
:1086B000015D1BA00FF056F8601C04B20C2CF6DB19
:1086C00019A00FF04FF8052408E0300240EA1566C3
:1086D0002D0206A8005D0543601E04B2002CF4DAEA
:1086E000B6B22A46334611A00FF03CF813A210216F
:1086F00002A8CDE900560FF045F8002404E002A8D6
:10870000005D3855601C04B20F2CF8DB0020F873B4
:108710000120C2E753544D33322049443D3D00000F
:1087200025303278000000000D0A000074656D707D
:108730003D253031356C6C750D0A00002530313522
:108740006C6C75002DE9F0438FB001213348FCF7C4
:10875000DBFA00BF02213148FCF749FA0028F9D0C2
:108760002E48FCF740FA0646642E0ADAB6F5805F1A
:1087700007DB2BA00EF0F6FF4FF0FF300FB0BDE887
:10878000F0832A482A49096840F82160284800688F
:10879000401C27490860092801DD002008600024EA
:1087A00006E0224850F8240005A941F82400641C82
:1087B0000A2CF6DB002419E000204DF824000025E7
:1087C0000DE005A850F825005DF82410884205DD6D
:1087D00005A850F825004DF824002F466D1C0A2DE1
:1087E000EFDB002005A941F82700641C042CE3DB23
:1087F000DDE9010100EB01080298C82802DA4FF018
:10880000FF30BBE74FF4987108FB01F0C11700EB94
:1088100011514FEA21394846B0E7000000240140D9
:1088200056444143204F564552000000DC1E0020B4
:108830008800002070B588B000268348007803289F
:108840001DDD8248007820F0040080490870002077
:108850007D49087001237EA21E2168460EF092FF1A
:10886000684604F0B5FC02207D49887000207649F6
:1088700008707648007820F0040074490870794840
:108880000068632808D076488078012804D16F48B2
:108890000078C0F3800038B90020734908600F20C9
:1088A0007249087008B070BD6848416B8163016B04
:1088B0004163C16A0163816AC162C06963498862B8
:1088C000002404E06148283050F82450641C052C32
:1088D000F8DB0520B5FBF0F55C4845620078C0F395
:1088E000001048BB61480078401CC0B25F49087066
:1088F0005F49097888421EDB00205C4908705A49AC
:1089000008605C480078B0B15B480078401CC0B299
:10891000594908705649497888420ADB002056496F
:1089200008700320524948700F20087007F0DEFBE2
:1089300001E0FCF77DFEB5E74348007820B9002050
:108940004A490870404908704C480078401CC0B241
:108950004A4908703C2807DD4948007820B90020C2
:10896000087001200FF0C8FB464801780078401CD1
:10897000444A10700F290ADD344890F87500012828
:1089800005D10FF0E7FB0020304981F875002F4832
:108990004068401C2D49486008460078C0F34000FC
:1089A000F8B139480068E0B108464068374991F8A5
:1089B000F812374A32F81110884205D300202349B3
:1089C00048600120334908700FF05CFEB0B13148B7
:1089D000007898B100202F4908700BF095FA012615
:1089E0000CE01A4840683C2808D30FF04BFE28B131
:1089F0000020164948600BF059FC012626480088E3
:108A0000401C80B224490880B42808DD3EB90FF02C
:108A100039FE20B10BF028FC00201F4908801F48B8
:108A20000078401CC0B21D4908701E2809DB0020D8
:108A300008701548006820B9012219A100200AF029
:108A400033FD00BF2EE7000000000020041F0020BF
:108A500041542B544350434C4F53453D25640D0026
:108A60000001002008010020200100200E0100204C
:108A700010010020402900201201002016010020D2
:108A80000F01002017010020A0020020AB5600209B
:108A900094A101081C0100201A01002018010020E7
:108AA00047505320636C6F73650000002DE9F0435D
:108AB00095B004463CB1002086490860864908709C
:108AC00015B0BDE8F0838548008828B1844810F0CF
:108AD0000FFB002081490880DFF808C200DF7D49D4
:108AE0000968884200D2EBE7DFF8F8C100DF6430A4
:108AF00078490860FFF79EFE7B488078032817D1ED
:108B00007A480078401CC0B2784908700A2812DD03
:108B10000020087076490870FDF78CFA002074492F
:108B200008707448007820F004007249087002E070
:108B300000206E49087068480078401CC0B2664941
:108B40000870042801DD00200870634800780028C0
:108B50003CD169480078012806D100206649087098
:108B600066A004F035FB05E001206349087066A0AB
:108B700004F02EFBDFF86CC100DF81466548006819
:108B8000FBF70EFE07460022634BFBF79AFD0546F6
:108B90000E466248016857484068CDE9036902956E
:108BA000CDE9050153480078C0F3400000905148DA
:108BB0000078C0F300135AA2372107A80EF0E2FD97
:108BC000012207A900200AF06FFC81E042480078EA
:108BD000012803D15EA004F0FBFA79E03E4800785A
:108BE000022818D14D480068632800D168E73E4844
:108BF0004078012809D1012359A2372107A80EF096
:108C0000C1FD07A804F0E4FA62E0012259A10020A6
:108C10000AF04AFC5CE03048007803283FD13F4826
:108C20000068632800D14BE73248007800F001006B
:108C300090B92D48C078322809DA2B48C078401CFA
:108C4000C0B22949C870022801DB0A20C87001227D
:108C50004CA100200AF028FC23488078012837D056
:108C600021484078012833D12248007820F00400C0
:108C7000204908704848B0F82D034849012348A20C
:108C8000CDE90010372107A80EF07CFD002207A9CE
:108C900010460AF009FC07A804F09AFA18E00E48FA
:108CA0000078042814D11D480068632800D107E724
:108CB0000D48807801280BD10E480078C0F3800061
:108CC00030B90C48007820F00400001D09490870F4
:108CD00000BFF5E6A0030020A40300201800002038
:108CE000980F0020B199010800010020A503002081
:108CF00000000020041F00209403002041542B4357
:108D000053510D0A0000000041542B434353510DB1
:108D10000A00000040000020000059400801002027
:108D20005B4154485D25642C5B4750535D25642CA2
:108D30005B4241545D25302E32662C5B5449434BD7
:108D40005D25642C25642C5B4353515D2564000034
:108D500041542B504F435F5050500D0A000000000B
:108D600041542B5443505354415455533D25640DA5
:108D70000A0000005761697420504F435F50505003
:108D800000000000475053206D6F64656D206E6FCA
:108D90007420776F726B2100AB56002030470020A3
:108DA00041542B5443504F50454E3D25642C257360
:108DB0003A25640D0A00000010B5194890F8F80231
:108DC000184931F8100068B14FF400701649486135
:108DD000134890F8F81215A00EF0C4FC01201849B1
:108DE00008601BE00E4890F8F81216A00EF0BAFCCE
:108DF0004FF400700C4908610020114908601548C3
:108E0000007820F00100134908700846007820F02F
:108E100002000870002048700F49088010BD000053
:108E2000AB56002094A10108001001406770734FF9
:108E300070656E696E673D3D3D25640D0A0000005A
:108E4000A0020020677073446F776E3D3D3D3D2565
:108E5000640D0A00041F00201800002010B5074808
:108E600002784FF4A0410648FBF74AFA8023A0227B
:108E70000021084605F026FA10BD000088040020F5
:108E8000406200202DE9F05F04460D4617469846E3
:108E9000A02C01DA802D01DBBDE8F09FE019A028AD
:108EA00002DBC4F19F0087B205EB0800802803DBDA
:108EB000C5F17F001FFA80F800261AE0A8191FFAF2
:108EC00080FA4FF0000910E004EB09001FFA80FB64
:108ED0000D4800780AEB8A010C4A02EB411101F8B7
:108EE0000B0009F101001FFA80F9B945ECDB701C99
:108EF00086B24645E2DB43463A462946204605F01F
:108F0000E1F900BFC8E700008804002040620020AB
:108F10002DE9FC5F04460D4616461F46B44201DCAF
:108F2000BD4201DDBDE8FC9FA02E00DB9F26802F07
:108F300000DB7F27301B401C1FFA80FB781B401C86
:108F40001FFA80FA4FF000081EE005EB080080B21F
:108F500001904FF0000911E004EB090080B200908D
:108F60000E480178019800EB80000D4A02EB401298
:108F70000098115409F101001FFA80F9D945EBDB83
:108F800008F101001FFA80F8D045DEDB53465A464F
:108F90002946204605F096F900BFC3E78804002063
:108FA00040620020F8B507460D4616461C4604B937
:108FB000F8BDBD4200DAFBE7601EC4B2002000909D
:108FC000301983B22A463146384600F049F800BFCE
:108FD000EEE72DE9F84306460C4617461D46DDF838
:108FE0002080BE4201DCAC4201DDBDE8F88343468F
:108FF000224639463046FFF7D5FF43462A463946D2
:109000003046FFF7CFFF0120434632462946009005
:10901000204600F00AF8012043463A4629460090CF
:10902000204600F002F800BFDFE72DE9F8430546CF
:109030000E4617461C46DDF820800CB9BDE8F883C3
:10904000AE4200DAFAE7601EC4B2381982B2334683
:1090500029463846CDF8008000F002F800BFEDE761
:109060002DE9FC5F04460D4616461F46B44201DC5E
:10907000BD4201DDBDE8FC9FA02C01DA802D00DBA4
:10908000F8E7A02E00DB9F26802F00DB7F27301B18
:10909000401C80B20190781B401C1FFA80FA4FF0F0
:1090A00000083AE005EB08001FFA80FBBBF17F0FD8
:1090B00001DD4FF07F0B4FF0000927E004EB0900C2
:1090C00080B2009000989F2801DD9F2000900C98AE
:1090D00001280CD0022809D1154801780BEB8B0030
:1090E000144A02EB4012009811540AE000BF1248E3
:1090F00001780BEB8B000F4A02EB401200981154E1
:1091000000BF00BF09F101001FFA80F901988145F5
:10911000D4DB08F101001FFA80F8D045C2DB5346CA
:1091200029462046019A05F0CDF800BFA2E70000CD
:1091300086040020406200208704002010B50AA0A9
:1091400000F008FA18B908A109A00EF00BFB10A056
:1091500008F0CAFB4FF47F026FF07F418B2000F0D4
:1091600075F8FFF77BFE10BD485A4B313600000002
:1091700043616E27742066696E64207468652048B8
:109180007A6B46696C6528257329210D0A00000059
:109190006C6F676F2E626D70000000002DE9F05F4C
:1091A00004460D4691469A4604EB0900A02803DBCD
:1091B000C4F19F001FFA80F905EB0A00802803DB49
:1091C000C5F17F001FFA80FA00262EE0A81987B2A9
:1091D0004FF0000B25E004EB0B001FFA80F807EBC3
:1091E0008700174901EB401010F80800154909786D
:1091F000884209D11448007807EB8701104A02EB36
:10920000411101F8080008E00E48007807EB8701DB
:109210000B4A02EB411101F808000BF101001FFAA3
:1092200080FBCB45D7DB701C86B25645CEDB534660
:109230004A462946204605F045F8BDE8F09F000063
:1092400040620020880400208704002070B5064694
:109250000C4615463046FDF7C9FD07490870204603
:10926000FDF7C4FD054908702846FDF7BFFD044918
:1092700008700DF0A5FE70BD870400208804002052
:10928000860400202DE9F84F05460E4617469846FD
:1092900008F00F0908F0F00AB9F1010F09D0B9F18F
:1092A000020F21D0B9F1030F39D0B9F1040F6CD1FD
:1092B00050E0002415E0012006EB040C1FFA8CF3AB
:1092C00005EB040C1FFA8CF2A6EB040C1FFA8CF1D0
:1092D00005EB040C00901FFA8CF0FFF77AFE601C7F
:1092E00084B2BC42E7DB51E0002415E0012006EB2C
:1092F000040C1FFA8CF3A5EB040C1FFA8CF2A6EBFE
:10930000040C1FFA8CF1A5EB040C00901FFA8CF0F2
:10931000FFF75FFE601C84B2BC42E7DB36E000244E
:1093200015E0012006EB040C1FFA8CF305EB040C8E
:109330001FFA8CF206EB040C1FFA8CF1A5EB040C5F
:1093400000901FFA8CF0FFF744FE601C84B2BC4210
:10935000E7DB1BE0002415E00120A6EB040C1FFA5C
:109360008CF305EB040C1FFA8CF2A6EB040C1FFA2D
:109370008CF1A5EB040C00901FFA8CF0FFF729FE8E
:10938000601C84B2BC42E7DB00E000BF00BFBDE868
:10939000F88F00002DE9F04FADB081460F469046A2
:1093A0004046FEF79DFD83465846FEF7B5FD8246D2
:1093B000BAF1000F02D12DB0BDE8F08F2CAB022224
:1093C0001C21584606F0A6FDBDF8B000082800D0C4
:1093D000F1E72BAB04221221584606F09BFD2AAB85
:1093E00004221621584606F095FD2B98A02802D895
:1093F0002A98802800D9DEE729AB04220A215846A2
:1094000006F088FD1C4B4FF480623621584606F06A
:1094100081FD2B9800F00304002C07DD2B9800F051
:109420000300C0F104002B99451800E02B9D2A98F9
:10943000461E002413E0299805FB060101AB58469F
:109440002B9A06F067FD01A800902B9882B238197C
:1094500081B20123484605F06BF8761E641C2A98F9
:109460008442E8D32A9883B22B9882B23946484680
:1094700004F028FF00BF9EE7405E00202DE9FF4F6B
:1094800083B0814693461F4607F0F0000290029891
:1094900028B94FF0020801264FF0100A04E04FF0FF
:1094A000030801264FF0180A5C46002523E02078C7
:1094B0009F280DDD00976378227809EB050188B2BB
:1094C000049904F071FF05EBC80085B2A41C12E0FA
:1094D0000097237809EB050188B20022049904F073
:1094E00063FF029818B905EBC60085B202E005EBF0
:1094F000061085B2641C20780028D8D153462A462D
:109500004846049904F0DEFE07B0BDE8F08F000085
:1095100003494A694A640A690A6481F83C00704751
:10952000E0590020044802680448018804A00EF0B5
:1095300019F900BFFEE70000680000206400002069
:109540000D0A5B4846485D463D25642C4C3D25642C
:109550000000000070B505461848406808B90020B2
:1095600070BD174800210160416081602846FEF708
:10957000B7FC0446002C01DA0020F1E71020104966
:109580000870487009780E4A527801FB02F0C11742
:1095900000EB5171C1F3C701094A91701046446054
:1095A00004EB440000EBC4010448083000EB8100E8
:1095B000406A114688600120D2E7000040B20020D6
:1095C000345E00202DE9F04104460D4616464FF06A
:1095D000020804F10B00FAF741FFC7B2607B3128A3
:1095E00002D14FF0010804E0607B302801D14FF038
:1095F00002082F7086F80080BDE8F08110B504469F
:109600000121C80206F036FA7D2006F023FB08B1DE
:1096100006F050FA45F2555000F028F8062000F008
:1096200019F8A0B200F01CF800F00CF800F002F8F5
:1096300010BD00004CF6CC400149086070470000A6
:10964000003000404AF6AA20014908607047000037
:109650000030004001494860704700000030004081
:1096600001498860704700000030004001490860EF
:10967000704700000030004070B504460D461646A5
:1096800032462146284610F07FFB70BD2DE9F74F8A
:10969000ADF58E6D82460E4600200190012E01D15F
:1096A000804609E0022E02D14FF4001804E00120A8
:1096B0000DF27C4DBDE8F08FDDF8780408B901208B
:1096C000019000250027AB460DF5816001F0D6FF23
:1096D00000BF24480069401BB0F5806F02D34FF4EF
:1096E000806906E01F48008A401B1FFA80F94FF08E
:1096F000010B08EB07014A4602A810F0CFFA0198C7
:1097000060B90198401CC0B2019000208DF808009B
:109710008DF809008DF80A008DF80B004D444F4478
:109720004A4602A90DF5816001F0BAFFBBF1000FB6
:10973000CFD00DF5816001F039FF002409E01AF85F
:1097400004100DF58C60005D814200D003E0601CC8
:1097500084B2102CF3DB00BF102C01DA0120A7E744
:109760000020A5E7E059002070B58AB004460D46F8
:1097700000200C4908702A46214601A804F0C2FCCA
:109780000646232E06D9012207A1002009F08CFEEF
:109790000AB070BD324601A9032001F0C5FC00BF2C
:1097A000F6E700004C0400207478627566206F763E
:1097B0006572210010B588B000200B49087068461A
:1097C00004F01AFD04461D2C06D9012207A1002031
:1097D00009F06AFE08B010BDA2B26946032001F08C
:1097E000A3FC00BFF6E700004C040020747862750B
:1097F00066206F76657221007FB54248407860B977
:10980000414801780078401C3F4A107021B901227C
:109810003EA1002009F048FE7FBD4048007800B11D
:10982000FAE738480078C0F3400000B9F4E735485B
:10983000007820F0020033490870012238A100208E
:1098400009F032FE022009F053FE2E480078C0F3E2
:10985000800000B1E0E70AF0E7F86C4601208DF8DF
:1098600000008DF8010032480078800631490978FF
:1098700040EA81503049097840EA41402F4909784F
:1098800040EA01302E49097840EA81102D490978D3
:109890000843CDF802002148B0F89601ADF8060063
:1098A0001848D0F80A100822204610F06DFA1B4D17
:1098B00008351448D0F80A0000F110014FF4C872BE
:1098C000284610F061FA0F48007820F00100401C93
:1098D0000C49087008464088401C4880084680882B
:1098E000401C88800846D0F80A00C1F806000846E7
:1098F000D0F806001449C1F88C00002004F054F898
:1099000000BF89E754520020740200205B534D537E
:109910005D496E76616C6964000000006A3D00205C
:109920005B534D535D53746F726520534D5300006C
:109930000400002005000020060000200300002095
:109940000100002002000020AB56002009480078EA
:10995000FF2804DA07480078401C064908700648CA
:109960000078FF2804DA04480078401C0249087097
:1099700070470000BC000020BD00002010B54D481D
:1099800000684D49884205D04A4800684A4918395C
:10999000884227D1012249A1002009F085FD00203D
:1099A0004D4908704D48007800281AD14C4800787D
:1099B00000287CD1DFF82CC100DF4B4909688842C0
:1099C00009D8DFF820C100DF474909680C1AA0B2A6
:1099D000DFF818C100DF46A003F0FAFB0020484979
:1099E000087064E033480068464988420BD1012280
:1099F00045A1002009F058FD0020414908700120D0
:109A00004549086053E02B4800682B49891D88426E
:109A100007D100203A490870012240A109F044FD15
:109A200045E0244800684149884205D1012240A10F
:109A3000002009F039FD10BD1E48006841498842E8
:109A400005D1012240A1002009F02EFDF3E71948BD
:109A500000684349884207D100202F49086001224D
:109A600040A109F021FDE6E7124800684349884219
:109A70001DD0104800684249884218D00D4800683F
:109A80004049884207D100200A49086001223EA1CE
:109A900009F00AFD0BE0074800684149884206D1F9
:109AA00000204049087001223FA109F0FDFC00BFE1
:109AB000C1E70000B80000202204FC005B4B4559C0
:109AC0005F5050542F4B45595F5050545F4D4943A0
:109AD00020467265655D0000C0000020480000203F
:109AE00020020020B199010870000020499301086C
:109AF00041542B504F433D3043303030300D0A003D
:109B0000BF0000202A047C005B4B45595F55502064
:109B1000467265655D000000580000205B4B4559AA
:109B20005F444F574E20467265655D002A00FC0079
:109B30005B4B45595F50414E454C5F4F4B20467241
:109B400065655D002A04EC005B4B45595F50414E52
:109B5000454C5F4D454E5520467265655D000000E1
:109B60002A04F4005B4B45595F50414E454C5F451C
:109B700058495420467265655D0000002A04DC00E7
:109B80002A04BC002A04B4005B4B45595F45584980
:109B9000545F444F574E5F475420467265655D00E1
:109BA0002A04F800490000205B4B45595F4F505490
:109BB000494F4E20467265655D00000008B50121E1
:109BC000084605F067FF01213248FDF7E5FD012158
:109BD0001C2005F05FFF48208DF8030003208DF85E
:109BE00002000820ADF8000069462B48FDF748FD4B
:109BF0002020ADF8000069462848FDF741FD4020CF
:109C0000ADF8000069462548FDF73AFD8020ADF823
:109C1000000069462148FDF733FD1020ADF8000033
:109C200069461E48FDF72CFD0820ADF80000694686
:109C30001A48FDF725FD0420ADF8000069461748D5
:109C4000FDF71EFD0220ADF8000069461248FDF741
:109C500017FD4FF48060ADF8000069460E48FDF72F
:109C60000FFD2020ADF8000069460B48FDF708FD08
:109C700010208DF803000001ADF800006946074888
:109C8000FDF7FEFC0020064908704D210E2006F06D
:109C90008BFB08BD0002300000100140000C0140A9
:109CA000BF00002000B589B0C748007808B90CF0A3
:109CB00043F8C6480068C64A811A904270D017DC43
:109CC000C44AA0EB020190426BD00ADCC2490844AE
:109CD00000283CD0B0F5401F73D0B0F5601F35D1DF
:109CE0003EE1B1F5001F6DD0B1F5401FF7D106E19F
:109CF000BA4A881A914211D00BDCB1F5802F76D088
:109D0000B7480844002873D0B64908440028E6D173
:109D1000BAE0182803D01E28E1D16AE000BF012074
:109D2000B14908700122B1A1002009F0BDFBA6488D
:109D3000007858B9B448007840B9DFF8D0C200DFE5
:109D40001430B3490860B3A003F042FA38E10120AF
:109D5000A54908700122B3A1002009F0A5FBB54870
:109D60008078012830D19848007860BBA6480078F8
:109D700048BBB1480078012826D1B048007828B9FE
:109D80000022AFA1012001F0D1FE2FE0A948D0F8B8
:109D9000070038B90022AEA1012001F0C7FE25E07E
:109DA000CCE0D7E00120B0490870A248D0F80730D5
:109DB000AEA21E2101A80DF0E5FC01A803F008FAEF
:109DC00014E0D9E0C0E0FFE77F48007870B98E4822
:109DD000007858B998480078012807D1974800784A
:109DE00020B1A7A003F0F4F909F008FEE8E0C9E00B
:109DF000BCE001207C4908700122A6A1002009F0E6
:109E000053FB8C48807801282BD16F48007840BBE9
:109E10007D48007828BB88480078012821D18748F0
:109E2000007828B9002286A1012001F07FFE2AE0F7
:109E30008048D0F80B0028B9002285A1012001F04C
:109E400075FE20E00120884908707A48D0F80B3070
:109E500086A21E2101A80DF095FC01A803F0B8F917
:109E600011E05948007870B96748007858B97248CD
:109E70000078012807D17148007820B18AA003F04A
:109E8000A7F909F0BBFD9BE06A48807801282BD137
:109E90004D48007840BB5C48007828BB6648007895
:109EA000012821D16548007828B9002264A1012049
:109EB00001F03CFE22E05F48D0F8030028B9002200
:109EC00063A1012001F032FE18E00120664908700C
:109ED0005848D0F8033065A21E2101A80DF052FCAD
:109EE00001A803F075F909E053480078012805D16D
:109EF0007248007810B904200BF082F860E06F48D7
:109F00000078A8B100206D4908706D4B6DA21E212C
:109F100001A80DF037FC01A803F05AF96EA26B21DD
:109F2000012008F0F5FC002201A9104609F0BCFA56
:109F300001226BA1002009F0B7FA41E001226EA1D5
:109F4000002009F0B1FA3BE0012271A1002009F0E4
:109F5000ABFA35E0012274A1002009F0A5FA2FE048
:109F6000012277A1002009F09FFA29E001227BA1BC
:109F7000002009F099FA23E001227FA1002009F0D6
:109F800093FA1DE082480078401C8149087081489E
:109F90000078C0F3001068B127480078012809D183
:109FA0007D480078012805D108460078032801D1B2
:109FB0000AF09EF9012279A1002009F075FA00BF8C
:109FC00000BF09B000BD000048000020B80000201C
:109FD0002A04F4002A04BC00D6FB83FFE0FF07003C
:109FE000FCFBFBFF0408FCFFBF0000205B4B455956
:109FF0005F5050542F4B45595F5050545F4D49436B
:10A000002050726573735D0020020020B199010831
:10A010007000002041542B504F433D3042303030CF
:10A02000300D0A005B4B45595F55502050726573E7
:10A03000735D0000AB560020540100204029002031
:10A040004345423442354337433242430000000027
:10A050004338424144374539434542344339453812
:10A0600044364333000000005C00002041542B5074
:10A070004F433D303930303030253038780D0A00CC
:10A0800041542B504F433D31303030303030370D5C
:10A090000A0000005B4B45595F444F574E205072F9
:10A0A0006573735D0000000041542B504F433D31F8
:10A0B000303030303030380D0A0000006C000020A5
:10A0C000EC3B002041542B504F433D303930303071
:10A0D0003025730D0A000000B2CBB5A500000000CA
:10A0E0005B4B45595F50414E454C5F4D454E5520A9
:10A0F00050726573735D00005B4B45595F50414E74
:10A10000454C5F455849542050726573735D00009B
:10A110005B4B45595F50414E454C5F555020507246
:10A120006573735D000000005B4B45595F50414E05
:10A13000454C5F444F574E2050726573735D00006D
:10A140005B4B45595F455849545F444F574E5F47F5
:10A15000542050726573735D000000005B4B4559DD
:10A160005F50315F50335F55504441544520507229
:10A170006573735D000000005B4B45595F4F4B5F9B
:10A18000444F574E5F4750532050726573735D00C4
:10A1900049000020041F0020340100205B4B45597A
:10A1A0005F4F5054494F4E2050726573735D0000ED
:10A1B0000648016801F0FC0109040548826840F284
:10A1C0002A40024041EA020070470000080C0140AA
:10A1D0000010014010B504463CB180200749486199
:10A1E00041000748FDF729FB06E08020034908618C
:10A1F00041000348FDF723FB10BD000000100140A3
:10A20000000C01402DE9F04F04460D4616461F464E
:10A21000A046B146AA46BB462A2000F085F94FEA7F
:10A22000282000F0AFF908F0FF0000F0ABF94FEA8A
:10A23000292000F0A7F909F0FF0000F0A3F92B2076
:10A2400000F072F94FEA2A2000F09CF90AF0FF00B2
:10A2500000F098F94FEA2B2000F094F90BF0FF0082
:10A2600000F090F92C2000F05FF9BDE8F08F0000BD
:10A27000F0B50E48008806120C4807787F239F220D
:10A2800000210846FFF7BEFF00240BE0002506E092
:10A29000304600F077F9384600F074F96D1CA02DB7
:10A2A000F6DB641C802CF1DBF0BD00008204002092
:10A2B00010B500F0FFF880207D494861402008611A
:10A2C0000120FCF7DBF94020794948610120FCF7C7
:10A2D000D5F94020764908617820FCF7CFF91120A4
:10A2E00000F022F97820FCF7C9F9B12000F01CF940
:10A2F000052000F047F93C2000F044F93C2000F034
:10A3000041F9B22000F010F9052000F03BF93C20A3
:10A3100000F038F93C2000F035F9B32000F004F9E2
:10A32000052000F02FF93C2000F02CF93C2000F033
:10A3300029F9052000F026F93C2000F023F93C2003
:10A3400000F020F9B42000F0EFF8032000F01AF933
:10A35000C02000F0E9F8282000F014F9082000F0EF
:10A3600011F9042000F00EF9C12000F0DDF8C02042
:10A3700000F008F9C22000F0D7F80D2000F002F933
:10A38000002000F0FFF8C32000F0CEF88D2000F090
:10A39000F9F82A2000F0F6F8C42000F0C5F88D2066
:10A3A00000F0F0F8EE2000F0EDF8C52000F0BCF869
:10A3B0001A2000F0E7F8362000F0B6F8A02000F0F0
:10A3C000E1F8E02000F0B0F8042000F0DBF82220F3
:10A3D00000F0D8F8072000F0D5F80A2000F0D2F8F5
:10A3E0002E2000F0CFF8302000F0CCF8252000F02F
:10A3F000C9F82A2000F0C6F8282000F0C3F826206B
:10A4000000F0C0F82E2000F0BDF83A2000F0BAF8B5
:10A41000002000F0B7F8012000F0B4F8032000F0AD
:10A42000B1F8132000F0AEF8E12000F07DF8042030
:10A4300000F0A8F8162000F0A5F8062000F0A2F819
:10A440000D2000F09FF82D2000F09CF8262000F051
:10A4500099F8232000F096F8272000F093F82720A1
:10A4600000F090F8252000F08DF82D2000F08AF8FB
:10A470003B2000F087F8002000F084F8012000F075
:10A4800081F8042000F07EF8132000F07BF83A20D9
:10A4900000F04AF8052000F075F8292000F044F893
:10A4A0004FF6FF71002000F09BF8FFF7E1FE10BDB2
:10A4B0000010014008B50121182005F0EBFA032037
:10A4C0008DF8020010208DF8030000021449086086
:10A4D0008020144908614FF47040ADF800006946CF
:10A4E0000F481038FDF7CCF84FF480500C49086045
:10A4F0004000086080000860401008604020094962
:10A50000086180200861C020ADF800006946054858
:10A51000FDF7B6F84020034908618020086108BDB6
:10A52000100C01400010014010B501464FF480535B
:10A53000134C23609B002360002018E0802343FA23
:10A5400000F29B010E4C236001EA020323B14FF499
:10A550000043241F236003E04FF40043084C2360B2
:10A560004FF40053064C241F2360431CD8B2082824
:10A57000E4DB4FF48053024C241F236010BD000025
:10A58000140C014010B501464FF48053134C236066
:10A590009B00241F2360002018E0802343FA00F270
:10A5A0009B010E4C236001EA020323B14FF40043E8
:10A5B000241F236003E04FF40043084C23604FF452
:10A5C0000053064C241F2360431CD8B20828E4DB48
:10A5D0004FF48053014C241F236010BD140C014024
:10A5E000024A1080024A1180704700008404002053
:10A5F0008204002008B50121084605F04BFA01212C
:10A600001648FDF7C9F801213C2005F043FA102057
:10A610008DF8030003208DF802004FF40050ADF8D0
:10A62000000069460E48FDF72BF80420ADF8000045
:10A6300069460C48FDF724F84FF48070ADF800002F
:10A6400069460948FDF71CF84FF4005004490861B9
:10A65000042004491031086008BD000000023000E9
:10A660000010014000140140000C014010B50446E8
:10A6700094210C2005F098FE0CB300206B49086073
:10A680006B4908706B4908706B490870FF206B4973
:10A6900008706B49087000206A4908706A490870A0
:10A6A0006A490870FF206A4908706A4908704FF4C7
:10A6B00000506949486104206849086010BDDFF80E
:10A6C000A0C100DF59490968884200D2F6E7DFF8E7
:10A6D00090C100DF0F30554908606248007820B90A
:10A6E0004FF400505C49486149E05F48007820B968
:10A6F0004FF400505849086141E0504800785949EA
:10A700000978884205D14E4800785749097888422F
:10A7100019D00020464908704A490870514800780D
:10A720004649087050480078454908704D480078FF
:10A730004006000E4049087041480078097801EB56
:10A7400040003C4908703A480078401CC0B2384983
:10A75000087038490978884202DD002034490870C1
:10A760003348007834490978884204DA4FF40050BD
:10A770003949086103E04FF40050374948613B48CC
:10A78000007818B904203549086048E03848007856
:10A7900020B904203149091F086040E02C480078A6
:10A7A00032490978884205D12A4800783049097829
:10A7B000884219D000201E490870224908702B4891
:10A7C0000078234908702A480078224908702748F1
:10A7D00000784006000E1D4908701E480078097870
:10A7E00001EB40001849087016480078401CC0B2C0
:10A7F0001449087014490978884202DD0020114983
:10A8000008701048007811490978884204DA042059
:10A810001249091F086002E0042010490860D32192
:10A820000C2005F0C1FD00BF48E70000A800002093
:10A83000AC000020AD000020AE000020AF000020E2
:10A84000B0000020B1000020B2000020B3000020C2
:10A85000B4000020B5000020001001401414014095
:10A86000B1990108A0000020A1000020A200002052
:10A87000A30000202DE9F0470446884691461E4675
:10A88000DDF820A0C4F80080002507E0206850F81B
:10A890002500077807B903E0681CC5B2C82DF5DBB1
:10A8A00000BF681EC5B2681CA080052095FBF0F0B3
:10A8B00060816089052190FBF1F201FB120010B16B
:10A8C0006089401C60810025C4F8D8600AE006B9A0
:10A8D0000AE0D4F8D80050F82500077807B903E05B
:10A8E000681CC5B2C82DF2DB00BFA4F8DC500025FF
:10A8F0000EE0A088A84205DD1AF8051004F10D004D
:10A90000415503E0002104F10D004155681CC5B21A
:10A91000C82DEEDB84F80C9000202081E0802046DA
:10A9200000F084F9BDE8F0872DE9F04704460F46B2
:10A9300016469846A4F83A710120A4F83C0100207C
:10A94000E08084F80C800025C4F8D8600DE006B9DA
:10A950000DE0D4F8D80050F8250090F80090B9F137
:10A96000000F00D103E0681CC5B2C82DEFDB00BFAB
:10A97000A4F8DC50642084F83801642201212046C8
:10A98000FDF7F0FBBDE8F0872DE9FF4106460F46D5
:10A990000A2E01DA012409E0642E01DA022405E01E
:10A9A000B6F57A7F01DA032400E004240A2F01DAE5
:10A9B000012509E0642F01DA022505E0B7F57A7F69
:10A9C00001DA032500E00425334610A20B2101A87B
:10A9D00000970CF0D7FE60190E490988884208D00C
:10A9E00060190C4908801023382201215020FEF7FD
:10A9F00049FA6119891CC900C1F1A00188B201237B
:10AA000001AA1946FEF73AFDBDE8FF8125647C25C1
:10AA1000640000009204002070B50446A08810B9BC
:10AA20003648006870BD354800683549084480B331
:10AA3000B0F5001F5CD13348007838B132488078D7
:10AA400008B9012000E000202F498870204600F05E
:10AA50004DF9E08830B92B48007818B9A088401E1D
:10AA6000E08005E02748007810B9E088401EE080CB
:10AA7000257AE088052190FBF1F020812089A84209
:10AA800003D0204600F0D2F802E0204600F02EF974
:10AA900031E0FFE71B48007838B11B48807808B9DF
:10AAA000012000E0002018498870204600F01EF9BF
:10AAB0001448007810B9E088401CE080E088A18844
:10AAC000884204DB0F48007808B90020E080257A2E
:10AAD000E088052190FBF1F020812089A84203D075
:10AAE000204600F0A3F802E0204600F0FFF802E064
:10AAF0000248006896E700BF002093E7B8000020F6
:10AB0000D6FB43FF89020020AB56002010B5044657
:10AB1000A08810B94348006810BD42480068424907
:10AB2000084400283CD0B0F5001F03D0B0F5601FEA
:10AB300072D16DE0204600F043F9B4F83C01401EAC
:10AB4000A4F83C01B4F83C0118B9B4F83A01A4F8EF
:10AB50003C01E08880B9B4F83A01052808DD752287
:10AB600000212046FDF7FEFA012084F83E0106E0B0
:10AB7000A088401EE08002E0E088401EE08094F85B
:10AB80003E0118B1002084F83E0102E0204600F0AA
:10AB900017F9B4F83A11B4F83C01FFF7F5FE3EE0BE
:10ABA000204600F00DF9E088401CE080B4F83C013C
:10ABB000401CA4F83C01B4F83C01B4F83A118842B6
:10ABC00002DD0120A4F83C01E088A18888420EDB68
:10ABD000B4F83A01052808DD642200212046FDF77B
:10ABE000C1FA012084F83E0101E00020E08094F8E1
:10ABF0003E0118B1002084F83E0102E0204600F03A
:10AC0000DFF8B4F83A11B4F83C01FFF7BDFE06E0F6
:10AC10000448006880E7FFE7024800687CE700BF5F
:10AC2000002079E7B8000020D6FB43FF2DE9F04172
:10AC30000446A08808B9BDE8F081207A00EB8000C6
:10AC4000C7B23D4619E0A088A84210DC052095FB5C
:10AC5000F0F100FB1150182101EB00101FFA80F8F1
:10AC60001023902241460020FEF70CF903E029460C
:10AC7000204600F0BCF8681CC5B2781D8542E2DBB6
:10AC8000204600F033F81848007820282AD08F2674
:10AC90002089002808DD06F1080188B20323082274
:10ACA0001821FEF7EFFA05E008231022182130469C
:10ACB000FEF7E8F84FF0680821896089401E81425C
:10ACC00008DA06F1080188B2042308224146FEF79B
:10ACD000D9FA07E0A8F1080081B208231022304613
:10ACE000FEF7D0F800BFA6E7540100202DE9F0419F
:10ACF00006460024D6F8D80010B104F11000C4B202
:10AD0000F088052190FBF1F201FB1200C5B218207A
:10AD100000EB0510C7B22348007820282CD15DBB7A
:10AD200004F14800C4B22048007830B91023402212
:10AD300039462046FEF732FA32E0102340223946E7
:10AD40002046FEF79FF81948807838B9012318A2E9
:10AD5000394604F11000FEF791FB06E0012316A22C
:10AD6000394604F11000FEF789FB102340223946D2
:10AD70002046FEF713FA13E00A480078202809D18C
:10AD800004F12000C4B210237E2239462046FEF78B
:10AD900005FA05E010237E2239462046FEF7FEF92B
:10ADA000BDE8F0815401002089020020AB5600204C
:10ADB000B9D8B1D500000000BFAAC6F40000000059
:10ADC0002DE9F04104460026D4F8D80010B106F170
:10ADD0001000C6B2A579182000EB0510C7B21023E9
:10ADE0007E2239463046FEF7D9F9BDE8F0812DE9DB
:10ADF000F0438BB004460D46052095FBF0F100FBB7
:10AE0000115087B20026182000EB07101FFA80F9B6
:10AE100010238E2249463046FEF734F8142106A846
:10AE2000F9F775FA207B50B1206850F825201421DD
:10AE300006A808F06AFD00208DF82B0009E02068C4
:10AE400050F82510142206A8F9F78AFA00208DF888
:10AE50002B00112206A901A808F024FDD4F8D8007F
:10AE6000A0B104F10D0010F80580D4F8D80050F816
:10AE7000282049463046FEF78DFA06F1100188B2C7
:10AE8000012301AA4946FEF7F9FA05E0012301AAC8
:10AE900049463046FEF7F2FA0BB0BDE8F0830000F9
:10AEA0002DE9F0438BB004460D46052095FBF0F1EB
:10AEB00000FB11501FFA80F80027182000EB081043
:10AEC0001FFA80F910238E2249463846FDF7DAFF33
:10AED000142106A8F9F71BFA207B68B105EBC50120
:10AEE00004F1DE0000EB4102142106A808F00DFD7C
:10AEF00000208DF82B000CE005EBC50204F1DE000C
:10AF000000EB4201142206A8F9F72AFA00208DF876
:10AF10002B00112206A901A808F0C4FCD4F8D8001F
:10AF200048B305EBC50104F1DE0000EB4100407CB5
:10AF3000B4F8DC10884206DB012213A1002008F0DF
:10AF4000B3FA002606E005EBC50104F1DE0000EBD4
:10AF50004100467CD4F8D80050F8262049463846AF
:10AF6000FEF718FA07F1100188B2012301AA494639
:10AF7000FEF784FA05E0012301AA49463846FEF7A8
:10AF80007DFA0BB0BDE8F0834C4231002DE9F04171
:10AF90000446A08808B9BDE8F081002512E0A08829
:10AFA000A84209DC182000EB05171023902239462F
:10AFB0000020FDF767FF03E029462046FFF770FFFA
:10AFC000681CC5B2052DEADB94F83801752802D15A
:10AFD000A088401EE0802046FFF7F2FE8F26B4F8DE
:10AFE0003A01052808DD06F1080188B2032308228A
:10AFF0001821FEF747F905E00823102218213046F2
:10B00000FDF740FF6827B4F83A01052808DD06F18E
:10B01000080188B2042308223946FEF733F907E015
:10B02000A7F1080081B2082310223046FDF72AFF5D
:10B0300000BFB0E710B586B01B4C1C48007808B9BB
:10B0400006B010BDDFF868C000DF1A490968884201
:10B0500027D919A002F0BCF81E20DFF86CC000DF71
:10B06000002012490870012008F036FB0F48437891
:10B0700016A2142101A80CF085FB01A802F0A8F883
:10B080000A48D0F8660020B90848801C02F0A0F8F1
:10B0900004E00649D1F8660002F09AF80FA002F029
:10B0A00097F800BFCCE70000CE090020F85500203B
:10B0B000B19901081C04002041542B4C53485454AE
:10B0C0005354500D0A0000004993010841542B4C81
:10B0D00053485454533D25642C220000220D0A008D
:10B0E00070B586B005460E4614462B4608A21421BC
:10B0F00001A800940CF046FB01A802F069F8214673
:10B10000304602F074F807A002F062F806B070BD95
:10B1100041542B54435053454E443D25642C2564E3
:10B120002C0000000D0A000070B504460D461646BE
:10B13000324629462046FFF7D3FF3146284604F021
:10B140006DFB012C08D109480078FF2804DA074874
:10B150000078401C05490870012C06D1044800788D
:10B1600020F00400001D0249087070BD000000209E
:10B17000041F00202DE9F04F93B004468846414655
:10B18000204604F04BFB6178A07861F31F208246D3
:10B190004FF0010B5346B9A2322106A80CF0F2FA87
:10B1A000012206A9002008F07FF9504648F2071254
:10B1B000AAEB020192457DD00BDCA0F602700028BC
:10B1C00079D0A0F5E040FF38002875D0FF2874D171
:10B1D00006E0A1F2F91100295BD00129F7D196E030
:10B1E000E57B2B46A8A2322106A80CF0CBFA01225F
:10B1F00006A9002008F058F9052D33D2DFE805F044
:10B20000031A20262C00072204F11001A248F9F7A6
:10B21000C8F848B1A04821690160A18A8180A17D58
:10B220008171002002F0C0FB9CA20A2103A80CF04F
:10B23000A9FA1DE09AA20A2103A80CF0A3FA17E0CC
:10B240009AA2012103A80CF09DFA11E099A20A210B
:10B2500003A80CF097FA0BE09AA20A2103A80CF0BD
:10B2600091FA05E09AA20A2103A80CF08BFA00BF1C
:10B2700000BF03A82B4698A23221009006A80CF02C
:10B2800081FA012206A9002008F00EF9FAF7D0F998
:10B29000EAE0E6784FF6FF7000EA062606F47F46FD
:10B2A00020790643701E86B2B6F5C87F01DB4FF4E5
:10B2B000C87603E0A8E0ABE032E0D2E040F29111C2
:10B2C0008A48F9F724F8324604F10E018748F9F765
:10B2D00005F88648001FA0F8966148F203108449DB
:10B2E000A1F80100E07A8DF80800207B8DF80900B4
:10B2F000BDF80800A1F80300022048717B48001F38
:10B30000B0F89601002801DD05F02CFDACE0657B6E
:10B31000052D03D1262009F073FE00BF00BFA3E076
:10B320000FFA88F7F81E215CB81E14F8009061F33C
:10B330001F29781E255C43466EA2322106A8CDE95E
:10B3400000950CF01FFA012206A9002008F0ACF8C5
:10B3500040F20711A9EB0100894549D006DCB9F19B
:10B36000020F31D0B9F5817F4CD106E0F92825D004
:10B37000A0F6FA50002845D12CE075B9664800784F
:10B3800020F0100010306449087064A2322106A831
:10B390000CF0F8F90DF014F80AE05F48007820F09E
:10B3A00010005D49087060A2322106A80CF0EAF98D
:10B3B000012206A9002008F077F823E001225EA10F
:10B3C000002008F071F81DE001225FA1002008F0C4
:10B3D0006BF817E0012260A1002008F065F86148D1
:10B3E00090F8BA02401CC1B25E4880F8BA1209E077
:10B3F0003DB901205C49087001225CA1002008F0E1
:10B4000053F800BF00BF2FE00020574908702BE021
:10B4100001225CA1002008F047F8607B8DF808004D
:10B42000A07B8DF80900BDF80800A0F5FA60584926
:10B430000870E07B57490870207C57490870607C91
:10B4400056490870A07C56490870E07C5549087040
:10B4500008460278524801785048007806F082FE8B
:10B4600002E04FF0000B00BF00BFBBF1000F02D0A5
:10B4700000204D49087013B0BDE8F08F0D0A636DD0
:10B48000643D2530347800000D0A726573756C7464
:10B490003D25303278000000A45900204F6B000099
:10B4A0004361722045786973740000004E6F206319
:10B4B000617200004465766963652045786973743C
:10B4C000000000004E6F205265636F726400000040
:10B4D0004661696C650000000D0A5B52656769731F
:10B4E0007465725D25642025730000006E3D0020A8
:10B4F000380100200D0A4C656E3D25642C61636B9C
:10B50000436D643D253034782C726573756C743DE1
:10B510002530327800000000041F00200D0A5B4136
:10B5200054485D4F6B0000000D0A5B4154485D4676
:10B5300061696C65000000000D0A4C6F63617469FD
:10B540006F6E2041434B00000D0A486561725469DB
:10B55000636B2041434B00000D0A534F532041437E
:10B560004B000000403900200F0100205465726D2F
:10B57000696E616C496E666F2053656E64204F4B37
:10B580000D0A00000D0A54696D6541636B000000EF
:10B590000400002005000020060000200300002019
:10B5A0000100002002000020000000202DE9F041F1
:10B5B00090B0044620680E9060680F902088C0F319
:10B5C000C507382F02DAC7F1380001E0C7F178006B
:10B5D000804642462849204600F062F800260025B1
:10B5E00018E004F11800E91C405C020604F11800A0
:10B5F000A91C405C42EA004204F11800691C405C4E
:10B6000042EA002004F11801495D08434DF8260084
:10B61000761C2D1D0E2EE4D3694604F1080008F0B7
:10B62000A7FF0026002521E004F1080010F82610ED
:10B6300050304155503830F82600C0F3072204F14D
:10B640005800691C4254503850F82600C0F3074295
:10B6500004F15800A91C4254503850F82600000E3E
:10B6600004F15801EA1C8854761C2D1D042EDBD3EE
:10B6700010B0BDE8F081000088B1010800214160F0
:10B68000016005498160054AC260CA430261034AFC
:10B69000D2434261704700000123456789ABCDEF7B
:10B6A0002DE9F04391B004460F4615462088C0F3BB
:10B6B000C509206800EBC5002168884202D2606895
:10B6C000401C6060206800EBC5002060606800EBF3
:10B6D0005570606033E017F8012B484609F1010905
:10B6E00004F118010A54B9F1400F28D14FF00008B5
:10B6F00000261AE004F11800F11C405C020604F177
:10B700001800B11C405C42EA004204F11800711CB0
:10B71000405C42EA002004F11801895D084301A958
:10B7200041F8280008F10108361DB8F1100FE1D3E7
:10B7300001A904F1080008F01BFF4FF00009281EC2
:10B74000A5F10105C7D111B0BDE8F08308B54FF4EC
:10B75000A06002F0EFFA3121012004F025FE25203F
:10B760008DF8000001208DF801008DF802008DF8A1
:10B770000300684602F0A6FA3821012004F014FE06
:10B7800026208DF8000001208DF801008DF80200C0
:10B790008DF80300684602F095FA3F21012004F07D
:10B7A00003FE27208DF8000001208DF801008DF8A0
:10B7B00002008DF80300684602F084FA4621012059
:10B7C00004F0F2FD17208DF8000001208DF8010033
:10B7D0008DF802008DF80300684602F073FA4E21DE
:10B7E000012004F0E1FD4FF4C06002F0A3FA032051
:10B7F0008DF8000001208DF8010000208DF8020076
:10B8000001208DF80300684602F05CFA08BD0000D4
:10B8100008B500BF00BF002640F2B341082004F085
:10B82000C3FDDFF8E0C100DF774908604FF49651AF
:10B830007648F8F76CFD07F05DFF0A20DFF8D0C10D
:10B8400000DF64214FF47A7005F02EF84FF4807019
:10B850007049486104F0B6FB002000906E48B0F8D3
:10B860002F20012300F121016CA00BF07BFF6A481F
:10B87000D0F81D1070A00BF075FF012271A10020FF
:10B8800007F012FE00207449088005F08BFDFEF7DA
:10B89000B1FE012271A1002007F006FE00207249CE
:10B8A0000860DFF8C8C100DF00F5FA607049086081
:10B8B0000023704A70497148DFF8C4C100DF714944
:10B8C00008600023704A6C497048DFF8B4C100DF9B
:10B8D0006F4908604FF49A61082004F065FD0AF092
:10B8E0001FFA8EE06B48007860B9DFF880C100DF96
:10B8F0005F490968884202D84448407810B1012065
:10B900006449087003F072FF62480078012801D191
:10B910000AF0B2FC0120DFF8F8C000DFFDF76CFF91
:10B92000FFF788FB40F2E141082004F03DFD5A4852
:10B93000008838B1594802F021FE0020564908809D
:10B9400057490880FCF742FB051E0CD0012D08D199
:10B95000FEF7A8F90020FEF73DFC00203E490880D4
:10B9600001E0FEF70BF80020FEF780FEFBF78AFFF0
:10B970000DF024F9DFF8F4C000DF4A490968884275
:10B9800000D23EE0DFF8E4C000DF643045490860E3
:10B99000FDF7DCFFFCF7D6FE0446002C01DD424833
:10B9A0000460032E02DA701CC6B204E000263E4892
:10B9B0000068FAF7FBFAFBF77DFA07F0F1FF3B4866
:10B9C00090F89A10903000EB41000088002817DDB5
:10B9D00021480088401C81B21F480180334890F8FC
:10B9E0009A20903000EB42000088814208DB002062
:10B9F0001949088005484078012801D1FEF7EAFB83
:10BA000000BF6FE7499C0108380000204029002052
:10BA10004993010800100140C41500200D0A257348
:10BA20005F5625642E25642E25642053746172743C
:10BA30002E2E2E0D0A00000050534E3A256C750D27
:10BA40000A0000004D61696E205461736B205374CD
:10BA50006172742100000000A40200204C65642083
:10BA6000496E69742E2E2E0054000020B1990108F1
:10BA700074000020084300200300040039D90008A6
:10BA80004D9A010828010020083F002081D40008B9
:10BA9000240100207800002012000020D00E002099
:10BAA000100000208000002040000020AB56002045
:10BAB00010B5124C10212046F8F729FC1048806977
:10BAC000000E20700E488069000C60700C48008BDE
:10BAD000000AA0700A48007EE07009484069000E24
:10BAE000207107484069000C60710548808A000A8F
:10BAF000A0710348007DE07110BD000010540020CB
:10BB0000041F002070B50546002407E0285D0D28BD
:10BB100002D10020285570BD601C84B22846F8F779
:10BB20002BFCA042F2D800BFF5E700002DE9F04160
:10BB300006460D4617462846F8F71EFC84B2642CCC
:10BB400000DD64247FB9224629461148F8F7C6FB78
:10BB5000642C02DA00210E48015500200C49891E90
:10BB6000C1F8660003E00A48801EC0F86650084825
:10BB7000801E46700078401C0549891E0870DFF859
:10BB800014C000DF283004490860BDE8F0810000DF
:10BB9000FA550020B19901081C04002004480268ED
:10BBA0000448018804A00BF0DDFD00BFFEE70000A3
:10BBB00068000020640000200D0A5B4D4D485D4682
:10BBC0003D25642C4C3D2564000000002DE9F0412A
:10BBD00004460E462660002500BF206850F8250068
:10BBE000077807B902E0681CC5B2F6E700BF681E17
:10BBF000C5B2681C2071052095FBF0F0E071E0797A
:10BC0000052190FBF1F201FB120010B1E079401C1C
:10BC1000E0710020A0716071204600F051F8BDE88D
:10BC2000F081000070B504462348006823490844A9
:10BC3000F8B1B0F5001F39D1204600F09AF86079CC
:10BC400018B92079401E607102E06079401E607171
:10BC5000A5796079052190FBF1F0A071A079A84247
:10BC600003D0204600F02CF802E0204600F081F8D6
:10BC70001FE0204600F07DF86079401C607160791B
:10BC80002179884201DB00206071A5796079052166
:10BC900090FBF1F0A071A079A84203D0204600F0FB
:10BCA0000FF802E0204600F064F802E00248006865
:10BCB00070BD00BF0020FBE7B8000020D6FB43FFAB
:10BCC0002DE9F0410446A07900EB800000F0FF0868
:10BCD00045461BE02079A84212DC052095FBF0F1D7
:10BCE00000FB115000EB8000182101EB800087B2AF
:10BCF000781E81B2122378221420FDF7C3F803E0E6
:10BD00002946204600F04FF8681CC5B208F105002E
:10BD10008542DFDB204600F02CF88C26A079002835
:10BD200008DD06F10A0188B2032308221821FDF775
:10BD3000A9FA05E00823122218213046FDF7A2F8DF
:10BD40007C27A179E079401E814208DA06F10A01D8
:10BD500088B2042308223946FDF794FA07E0A7F1D8
:10BD6000080081B2082312223046FDF78BF8BDE8A7
:10BD7000F0812DE9F041044614256079052190FBFE
:10BD8000F1F201FB1200C7B207EB8700182101EBAB
:10BD90008000C6B2701E81B2122378222846FDF7B9
:10BDA000FDF9BDE8F0812DE9F04105460C4605207E
:10BDB00094FBF0F100FB1140C7B207EB870018219C
:10BDC00001EB8000C6B2701E81B2122378221420CB
:10BDD000FDF758F8296851F82400314606F00CFEAA
:10BDE000BDE8F08110B50B4800680B49884208D1C6
:10BDF0000A484088012801DBFAF778FC052009F0A1
:10BE0000FFF8044800680649884202D1052009F07D
:10BE1000F7F810BDB80000202A04EC0054520020AE
:10BE20002A04F40010B50446D4B1FDF717F8012137
:10BE30000CA006F0E1FD012314229F210020FDF754
:10BE4000B1F80BA006F014FF012368229F21002007
:10BE5000FDF7A8F8012309A26E210020FDF70EFBD3
:10BE600010BD0000CFFBCFA2C9BEB3FD0000000093
:10BE7000C8B7B6A8C9BEB3FD3F0000005B4D5DC8A2
:10BE8000B7B6A820205B455849545DC8A1CFFB0038
:10BE90002DE9F04104460F4615461E462780A57041
:10BEA0003046F8F769FA84F87500102084F87700B6
:10BEB000002084F87400BDE8F0812DE9F05F0446AD
:10BEC00089464FF0000A4E4694F802C094F877E095
:10BED0000CEB0E03B4F800C094F876E0F4441FFABB
:10BEE0008CF2A1782088FCF7CDFF142104F16000CA
:10BEF000F8F70DFA2088C0F19F0087B23846F9178D
:10BF000007EB5171C1F3C70184F87410D0460025C6
:10BF1000AB4644E030789F2810DD94F87400401B55
:10BF2000022808DB04F16000284431880180A81C45
:10BF3000C5B2B61C11E04FF0010B0EE094F874008E
:10BF4000401B012807DB317804F160004155681C73
:10BF5000C5B2761C01E04FF0010BBBF1000F1ED003
:10BF60004FF0000B002104F16000415594F802C02D
:10BF70004246531C03F0FF080CEB021120880123FA
:10BF800004F16002FDF77AFA0AEB05001FFA80FA65
:10BF90000025B8F1050F02DB5046BDE8F09F307870
:10BFA0000028B7D1002104F16000415594F802C087
:10BFB0004246531C03F0FF080CEB021120880123BA
:10BFC00004F16002FDF75AFA0020E6E710B50948CF
:10BFD00000680949884204D1FBF712F8052009F0EE
:10BFE0000FF8044800680549884202D1052009F08D
:10BFF00007F810BDB80000202A04EC002A04F40061
:10C0000010B50446D4B1FCF729FF01210CA006F0BD
:10C01000F3FC012314229F210020FCF7C3FF0BA097
:10C0200006F026FE012368229F210020FCF7BAFFBC
:10C0300001230AA26E210020FDF720FA10BD0000A6
:10C04000CFFBCFA2B8F1CABDBBAF0000C8B7B6A83E
:10C05000C9BEB3FDCBF9D3D0A3BF00005B4D5DC813
:10C06000B7B6A820205B455849545DC8A1CFFB0056
:10C0700010B51048FFF7D6FD04460F4884420ED194
:10C080000C48407910B1012808D103E00F2008F0D6
:10C09000B7FF03E0102008F0B3FF00BF08E0074837
:10C0A00000680749884203D10649487808F0A8FF8C
:10C0B00010BD0000800200202A04EC00B80000201F
:10C0C0002A04F4005401002010B504460CB3FCF718
:10C0D000C5FE01210FA006F08FFC012314229F2131
:10C0E0000020FCF75FFF012368229F210020FCF75E
:10C0F00059FF0B490B48FFF769FD012368229F2177
:10C100000020FCF74FFF012307A26E210020FDF75E
:10C11000B5F910BDCEC4B1BED1A1CFEE0000000074
:10C1200068020020800200205B4D5DC8B7B6A820E1
:10C13000205B455849545DCDCBB3F60010B51C4883
:10C1400000681C49884203D1052008F059FF2EE001
:10C15000174800681849884229D0154800681749CF
:10C16000884224D11648F8F707F916490988884209
:10C170001DD967239F2218210020FCF7C9FE104B10
:10C18000182208211048FFF783FE0D480D4A128837
:10C1900081180D48FFF791FE04462CB1094800882C
:10C1A00020440849088002E000200649088010BDAC
:10C1B000B80000202A04F4002A04EC002A04BC0081
:10C1C0007E52002064020020DC51002010B504469D
:10C1D000002C32D000201A4908804FF4C871194849
:10C1E000F8F795F8FCF73AFE012117A006F004FCD9
:10C1F000012314229F210020FCF7D4FE114803F0F4
:10C2000035FF104B182208211248FFF741FE0D4858
:10C210000B4A128881180F48FFF74FFE0849088023
:10C22000012368229F210020FCF7BCFE01230AA203
:10C230006E210020FDF722F910BD00BFFCE70000D1
:10C24000640200207E520020CFFBCFA2D4C4B6C12E
:10C2500000000000DC5100205BCFC25DB7ADD2B35F
:10C26000205B455849545DB7B5BBD80010B512489E
:10C27000408810B11148FEF749FC11480068114987
:10C28000084450B1B0F5002F03D0B0F5402F0FD1C6
:10C290000AE0022008F0B4FE0BE00748408810B125
:10C2A0000E2008F0ADFE04E00D2008F0A9FE00E02D
:10C2B00000BF00BF10BD00005452002058470020AE
:10C2C000B8000020D6FB13FF18B10121034A5161C9
:10C2D00002E00121014A1161704700000010014095
:10C2E00008B50120ADF8000010208DF803000320F0
:10C2F0008DF8020069460548FBF7C2F90020FFF7F8
:10C30000E3FF7A21072004F04FF808BD0010014038
:10C310002DE9F041B0B0002600275A4890F8DD0121
:10C32000C0EB4011584800EB4105564890F8DD013C
:10C33000C0EB4011544800EB410000F11F04DFF84E
:10C340004C8153A2642117A80BF01CFA4D4890F8B9
:10C35000DF0120B952A117A8F7F7E4FF14E04A4B18
:10C360001F3B53A2502103A80BF00CFA03A800F0C6
:10C370002FFF454B1F3B54A2502103A80BF002FA9C
:10C3800003A917A8F7F7CEFF002217A9104607F058
:10C390008BF84EA2642117A80BF0F4F9287808B1A5
:10C3A000207820B93EA117A8F7F7BCFF15E02B466F
:10C3B00049A2502103A800940BF0E4F903A800F06F
:10C3C00007FF2B464AA2502103A800940BF0DAF98C
:10C3D00003A917A8F7F7A6FF0126012217A9002035
:10C3E00007F062F8002E4AD043A2642117A80BF090
:10C3F000C9F9244890F89B00C0B1012802D0022856
:10C4000019D10EE03FA117A8F7F78CFF1D48CDE921
:10C41000004590F89B303CA2502103A80BF0B2F9E4
:10C4200016E03FA117A8F7F77DFF00BF3EA117A8B0
:10C43000F7F778FF00BF3EA117A8F7F773FF114881
:10C4400090F89B303DA2502103A80BF09BF900BF50
:10C4500000BF012217A9002007F026F803A800F06A
:10C46000B7FE002203A9104607F01EF81420DFF8DB
:10C47000E0C000DF012237A1002007F015F830B03E
:10C48000BDE8F081AB560020A9580020CE0900205D
:10C490005B31315D416363657373703A0000000086
:10C4A000756E737570706F72742D456D7074790050
:10C4B00041542B4D495050524F46494C453D312C2B
:10C4C000222573220D0A0000257300002C4E616D99
:10C4D000652D506173733A0041545E50505043468D
:10C4E000473D222573222C222573220D0A000000CD
:10C4F00025732C2573000000415554482D4C4F479F
:10C50000494E3A0050415000415424514350445048
:10C51000503D312C25642C25732C25730D0A000009
:10C5200043484150000000004E4F4E4500000000BF
:10C5300020446F206E6F7468696E67004154245107
:10C5400043504450503D312C25640D0A000000003A
:10C5500049930108417574684C6F67696E20446F98
:10C560006E650000002070472DE9F04FA5B04FF038
:10C570000009CA46CB460020019001268B4C0025BD
:10C580000EE18BA000F024FE322703E14FF4A061FE
:10C59000A01C01F091FA80B2208000287ED088A1F2
:10C5A000A01C00F059FF0028EFD100222088C01EF7
:10C5B000A11C0A5404F10F00F8F726FC8046002164
:10C5C000A01C00F808101BAA7FA1FBF763FF8046A0
:10C5D0007E48D0F81D307EA2642102A80BF0D2F86C
:10C5E0001BA902A8F7F7CFFE08B14FF001091BAA5B
:10C5F00078A1A01CFBF74EFF8046774B77A2642101
:10C6000002A80BF0BFF81BA902A8F7F7BCFE08B1FF
:10C610004FF0010B724890F89C0005282FD2DFE8FC
:10C6200000F003040607050000BF00BF27E000BFBD
:10C630006B4890F89C00022806D16A4B67A26421DF
:10C6400002A80BF09FF80BE0654890F89C000328C7
:10C6500006D1644B283361A2642102A80BF092F842
:10C660001BAA61A1A01CFBF715FF80461BA902A80D
:10C67000F7F789FE08B101200190002600BF00BF36
:10C68000BEB11BAA5AA1A01CFBF704FF80460BF009
:10C6900075FF034651A26421009000E076E002A8F5
:10C6A0000BF070F81BA902A8F7F76DFE08B14FF068
:10C6B000010AB9F1000F0BD1BAF1000F08D1BBF19B
:10C6C000000F05D1019818B9002025B0BDE8F08F02
:10C6D00048A000F07DFD3D48D0F81D3049A228213A
:10C6E0001BA80BF04FF802A91BA8F8F741FB02A802
:10C6F00000F06EFD7EB10BF041FF034643A22821FE
:10C7000000901BA80BF03EF802A91BA8F8F730FB1D
:10C7100002A800F05DFD304B3EA228211BA80BF0C3
:10C7200031F802A91BA8F8F723FB02A800F050FD7E
:10C730002B4890F89C00022806D12A4B37A22821CA
:10C740001BA80BF01FF815E0254890F89C00032863
:10C7500007D1244B283331A228211BA80BF012F853
:10C7600008E031A228211BA80BF00CF802A91BA895
:10C77000F8F7FEFA02A91BA8F8F7FAFA02A800F0E7
:10C7800027FD2CA000F024FD01209EE70120DFF80A
:10C79000A8C000DF381EA7F101077FF4F7AE6D1CBB
:10C7A000052DFFF6EEAE00208FE70000CE09002039
:10C7B00041542B504F433D3032303030300D0A0061
:10C7C0002B504F433A30320069640000C4150020FA
:10C7D000256C750070776400F61500202573000045
:10C7E000AB56002038580020646F6D61696E000000
:10C7F0006970000041542B504F433D303130303090
:10C800003000000069643D256C753B0069703D2572
:10C81000733B00007077643D25733B00646F6D616E
:10C82000696E3D25733B0000646F6D61696E3D3B31
:10C83000000000000D0A0000499301082DE9FE43A5
:10C840000025214CA846002639E032274DB90125A4
:10C850001EA000F0BDFC20A20A2168460AF092FF4B
:10C8600008E000251EA000F0B3FC20A20A216846C3
:10C870000AF088FF1DE04FF4A061A01C01F01CF934
:10C8800080B2208088B16946A01C00F0E5FD80B927
:10C89000E81DA11C085C52280BD105F10900085CB9
:10C8A000412806D10120BDE8FE830120DFF844C005
:10C8B00000DF381EA7F10101CFB2DCD1761C1E2E9D
:10C8C000C3DB0020EFE70000CE09002041542B51CC
:10C8D0004350494E3F0D0A002B514350494E3A00F8
:10C8E00041542B4350494E3F0D0A00002B43504901
:10C8F0004E3A000049930108F0B595B0424C00272C
:10C90000002578E0642641A000F062FC6CE042481B
:10C910000078012802D1801E15B0F0BD4FF4A0614F
:10C92000A01C01F0C9F880B22080002858D03BA19B
:10C93000A01C00F091FD002856D1152204F1090138
:10C940003848F7F7CBFC0020364908750B4636A26D
:10C95000502101A80AF016FF324800798DF8000036
:10C96000304840798DF8010000208DF802006846BB
:10C97000F7F774FD0C2826D2DFE800F01006111B33
:10C98000122507131C08251D00BF00BF02202B49DC
:10C9900008702BA101A8F7F7C5FC19E000BF00BF84
:10C9A00000BF01202549087029A101A8F7F7BAFCAA
:10C9B0000EE000BF00BF00202049087028A101A898
:10C9C000F7F7B0FC04E02AA101A8F7F7ABFC00BF21
:10C9D00000BF012201A9002006F066FD01209BE7AF
:10C9E0000120DFF89CC000DF301EA6F101010EB26D
:10C9F0008DD1681C05B2052D84DB012221A1002008
:10CA000006F052FD002087E7CE09002041542B4953
:10CA1000434349440D0A0000350100205E53434959
:10CA2000443A0000965600205B4D696E69745D497A
:10CA3000434349443A25735B000000003F01002056
:10CA40004348494E415F554E49434F4D5D000000FC
:10CA50004348494E415F4D4F42494C455D000000FF
:10CA60004348494E415F54454C45434F4D5D00009E
:10CA7000554E4B4E4F572D49434349445D000000EE
:10CA8000499301085B4D696E69745D476574204385
:10CA9000434944206661696C6564000070B58AB0E2
:10CAA000224C23480078012801D00AB070BD00252F
:10CAB0002AE032261FA000F08BFB1DE04FF4A0619E
:10CAC000A01C00F0F9FF80B2208088B11EA1A01C3C
:10CAD00000F0C2FC80B9207C302804D100211E481F
:10CAE00080F8BC1203E001211B4880F8BC1208E06A
:10CAF0000120DFF868C000DF301EA6F101010EB290
:10CB0000DCD100BF681C05B2052DD2DB124890F8BD
:10CB1000BC3213A2282168460AF034FE012269467D
:10CB2000002006F0C1FC00BFBFE70000CE090020D6
:10CB30002800002041542B504F433D3430303030DA
:10CB40003030300D0A0000002B504F433A34303063
:10CB50003030303030300000403900204993010837
:10CB60000D0A47657420636F6465747970653A25B2
:10CB7000640000002DE9F0478CB0724C40F2612156
:10CB8000022003F011FC4FF0000A01226EA10020E8
:10CB900006F08AFC01264FF00008CDE01EB96EA019
:10CBA00000F016FB02E06EA000F012FB4FF032091D
:10CBB000B9E04FF4A061A01C00F07EFF80B220809D
:10CBC00000287BD0002E40D168A1A01C00F044FCBE
:10CBD00028B90022A11C104606F066FCA3E067A15C
:10CBE000A01C00F039FC0028E2D166A1A01C00F0D6
:10CBF00033FC20B168A1A01C00F02EFC18B9012064
:10CC00006A49087019E06AA1A01C00F025FC20B157
:10CC10006CA1A01C00F020FC18B902206349087028
:10CC20000BE06DA1A01C00F017FC18B903205F49B0
:10CC3000087002E000205D4908700022A11C104627
:10CC400006F032FC701CC6B273E068A1A01C00F0B4
:10CC500003FC28B90022A11C104606F025FC62E066
:10CC600067A1A01C00F0F8FB38B90022A11C1046F7
:10CC700006F01AFC0CB0BDE8F08762A1A01C00F021
:10CC8000EBFB00284FD10022A11C104606F00CFC43
:10CC9000002700253DE0A01C405D5F2838D1781CAE
:10CCA000C7B2012F0BD1A01CE91C405C8DF8040019
:10CCB000A01C291D405C8DF8050029E02FE0032F02
:10CCC00026D1A01CA91C405C8DF80600A01CE91C04
:10CCD000405C8DF80700A01C291D405C8DF8080001
:10CCE000A01C691D405C8DF8090000208DF80A0029
:10CCF00001AB48A21E2104A80AF044FD012204A9A8
:10CD0000002006F0D1FB01A8F7F7A8FB4549086011
:10CD10006D1CA01CF7F730FBA84204D9BBE701202B
:10CD2000DFF804C100DFB9F10000A9F101097FF4C7
:10CD300040AF00BF08F10108B8F10A0FFFF62EAFAF
:10CD400000BF97E7CE0900205B30335D4D6F64650F
:10CD50006D496E666F3A00004154490D0A000000AB
:10CD600041542B4C435453570D0A00004D616E75CE
:10CD700066616374757265723A0000004D6F646598
:10CD80006C3A00004D6F64656C3A20553935303788
:10CD900043205633000000004D6F64656C3A205507
:10CDA00039353037432053584E5400003E0100209F
:10CDB0004D6F64656C3A205539353037435F5358B1
:10CDC0004E4D00004D6F64656C3A20553935303753
:10CDD000432053584E4D00004D6F64656C3A20550A
:10CDE000393530374320504F43430000536F66744A
:10CDF0007761726556657273696F6E3A0000000064
:10CE000041503A00496E6E657256657273696F6E75
:10CE10003A0000005B30335D4D6F64656D5665729E
:10CE20003A257300F40000204993010810B5B4219D
:10CE3000022003F0B9FA00F025FF00201149087024
:10CE4000B821022003F0B0FA02200F4908606420E4
:10CE5000DFF838C000DF02200B49091D08600120FF
:10CE6000091F08606420DFF824C000DF01200649A4
:10CE7000091D08600AF090FB08B1002010BD0120D8
:10CE8000FCE7000000000020100C0140499301085D
:10CE900070B52E4C01222EA1002006F005FB0025C6
:10CEA0004AE032262FA000F093F940E04FF4A06151
:10CEB000A01C00F001FE80B22080002833D02DA1FC
:10CEC000A01C00F0C9FA30B901222CA1002006F004
:10CED000EBFA002070BD34A1A01C00F0BDFA0028C0
:10CEE00025D1E07B312806D1012232A1002006F0B5
:10CEF000DBFA0020EEE7012234A1002006F0D4FA8C
:10CF00003AA000F065F93EA005F0B2FE002604E06C
:10CF10000220F9F7B3FBFCF795FB701C064632289C
:10CF2000F6DB0120D6E70120DFF8E4C000DF301E89
:10CF3000A6F10106BAD16D1C642DB2DB012235A128
:10CF4000002006F0B1FA0020C4E70000CE0900205E
:10CF5000636865636B2076657273696F6E207479A0
:10CF60007065000041542B4C53504F4350463F0DC9
:10CF70000A0000004552524F5200000049742069D7
:10CF800073206E6F74203320696E203120766572B5
:10CF900073696F6E2071756974207468697320639A
:10CFA0006865636B000000002B4C53504F435046A4
:10CFB0003A00000049742069732068677320766521
:10CFC0007273696F6E206E6F770000005265736533
:10CFD0007420746F206867732076657273696F6E52
:10CFE00020616E64207265626F6F740041542B4C37
:10CFF00053504F4350463D6867730D0A00000000D0
:10D00000C7D0BBBBBAA3B8DFCBBCB0E6B1BE000093
:10D010004993010854696D654F75740010B5074850
:10D020000078012800D010BD05A000F0D1F8022042
:10D03000DFF820C000DF00BFF5E700002800002077
:10D0400041542B504F433D3330303030303031304D
:10D05000300D0A004993010808B501211C2002F097
:10D0600019FD10208DF8030003208DF80200022026
:10D07000ADF8000069460948FAF702FB0120ADF857
:10D08000000069460548FAF7FBFA0220034910310F
:10D0900008600120091D086008BD0000000C014067
:10D0A0002DE9F0438BB0374C00255CE04FF032099E
:10D0B00035A000F08DF84DE04FF4A061A01C00F009
:10D0C000FBFC80B22080002840D033A1A01C00F0DF
:10D0D000C3F900283ED1A01CF7F74EF907B24FF074
:10D0E000000800252FE0A01C405D0D2819D100206C
:10D0F00001A901F8080001A8F7F7B0F90646A01C3D
:10D10000334628A22821009001A80AF03BFB002208
:10D1100001A9104606F0C8F9274806600BB0BDE823
:10D12000F083A01C405D30280BDBA01C405D39283B
:10D1300007DCA01C425D4046411C0FFA81F801A9A2
:10D140000A54681C05B2BD4204DACCE70120DFF8BE
:10D150006CC000DFB9F10000A9F101010FFA81F9FB
:10D16000AAD1681C05B2052DA0DB334614A22821E4
:10D1700001A80AF007FB012201A9002006F094F99A
:10D1800000BFCBE7CE09002041542B504F435F56E0
:10D1900045523F0D0A0000002B504F435F56455249
:10D1A0003A0000005B30345D504F437665723A259B
:10D1B000643C2D3E25730000F800002049930108CF
:10D1C0005B30345D506F635665723D25640000002E
:10D1D00070B504462046F7F7CFF885B22521022026
:10D1E00003F0E2F82946204609F0F0FD70BD70B565
:10D1F00004460D462946204609F0E8FD70BD0000B2
:10D200002DE9F0438DB005460E46194C00272AE063
:10D210004FF0320833462A4616A168460AF0C6FA8D
:10D220006846FFF7D5FF18E04FF4A061A01C00F09E
:10D2300043FC80B2208060B1A01CF7F79DF88146C6
:10D2400012A1A01C00F008F938B900200DB0BDE80B
:10D25000F0830120DFF838C000DFB8F10000A8F14A
:10D260000108E1D17F1C0A2FD2DB2846EEE700003F
:10D27000CE09002041542B434F4445433D332C25D8
:10D2800032782C2534780D0A000000004F4B000046
:10D290004993010808B501211C2002F0FBFB102076
:10D2A0008DF8030001208DF80200C003ADF80000E6
:10D2B00069460448FAF7E4F94FF400400149143193
:10D2C000086008BD000C014070B58AB0064656B132
:10D2D000012E02D0022E09D102E00524192507E013
:10D2E0000524372504E00524052501E00AB070BDBA
:10D2F00000BF234607A21E2102A800950AF042FAA9
:10D3000002A8FFF765FF002202A9104606F0CCF83C
:10D3100000BFEBE741542B5544503D25642C256458
:10D320000D0A000008B501211C2002F0B3FB1020FB
:10D330008DF8030001208DF80200C002ADF8000056
:10D3400069460448FAF79CF94FF40060014914312A
:10D35000086008BD000801402DE9F041214C00267D
:10D3600036E0322700BF20A0FFF732FF29E04FF45C
:10D37000A061A01C00F0A0FB80B2208000281CD07F
:10D380001EA1A01C00F068F8D8B904F10F00F7F74F
:10D3900065F8054641F65830854207D01BA0FFF7D7
:10D3A00017FF0120DFF880C000DFDCE701221FA1AA
:10D3B000002006F079F8BDE8F0810120DFF868C0B0
:10D3C00000DF381EA7F10101CFB2D0D1701CC6B268
:10D3D000052EC6DB01221AA1002006F065F800BF69
:10D3E000E9E70000CE09002041542B4C5348545427
:10D3F0005353504545443F0D0A0000002B4C534801
:10D4000054545353504545443A00000041542B4C6A
:10D41000534854545353504545443D2D312C3730D7
:10D4200030300D0A00000000499301085B30365D82
:10D43000536574545453205370656564204F6B00DA
:10D440005B30365D53657454545320537065656486
:10D45000204661696C65640030B502460B4619468A
:10D46000144607E008782578A84201D0012030BD95
:10D47000491C641C08780028F4D100BFF7E70000BD
:10D480008AB000BF00BFD14C0120D14908700122F1
:10D49000D0A1002006F008F80120FBF707FB0020D0
:10D4A000D0490870D04948708870C8700122CFA157
:10D4B00005F0FAFF00BF0122D1A1002005F0F4FF22
:10D4C000012003F0ABFE0420D14908610021D148BE
:10D4D00080F8B91280F8BB120020CF490870CF49FC
:10D4E0000870CF490860DFF83CC300DFCE49086709
:10D4F000CE48FBF7CDF801280AD1CC4BCCA228218D
:10D5000068460AF03FF901226946002005F0CCFF89
:10D51000FFF78CFCA8B90120C94908700420BC4958
:10D5200048610122C7A1002005F0BEFFF9F74AFAC1
:10D5300006E00020B84908726420DFF824C300DF49
:10D54000F7E7FFF7A5FC00B1B5E74FF40071C54858
:10D55000FAF76AF9012802D1C349087002E00420F1
:10D56000AB4948610120AD490870C0A0FFF730FE0B
:10D57000C2A0FFF72DFE0122C2A1002005F094FFFA
:10D58000FA20DFF8DCC200DFFFF7F4FAFFF788FDCE
:10D59000F8F7E4FCFFF742FDFFF780FAFFF7DCFE47
:10D5A0003220DFF8BCC200DF09F0F4FD09F006FF0D
:10D5B00009F07CFEF8F790FD06F058F8FFF73EF909
:10D5C00030BB0421934880F8BB1200BFFAF73AF948
:10D5D0001DE04FF4A061A01C00F06EFA80B2208024
:10D5E00000B114E00120DFF878C200DF00208A4992
:10D5F00008727748007800B909E0A548008828B18A
:10D60000A4480BF075FD0020A149088000BFE0E7A9
:10D610000122A1A1002005F047FFFFF76DF902F0FC
:10D62000A3FDFEF7A1FF28B101229FA1002005F074
:10D630003BFF04E00122A0A1002005F035FF0120FE
:10D6400075494871FEF764FE01229FA1002005F094
:10D650002BFFFAF7F7F8FBF7AFFB03F0D1FF01223E
:10D660009EA1002005F020FFFEF77CFF28B10122DB
:10D670009EA1002005F018FF04E00122A0A10020D7
:10D6800005F012FFA4A0FFF7A3FD9EE0504800782C
:10D69000F8B94FF4A061A01C00F00EFA2080208899
:10D6A000002808DD0022A11C104605F0FDFEA01C8C
:10D6B000F7F70CFC89E02088002805DA01229AA1FE
:10D6C000002005F0F1FE80E00120DFF894C100DFCA
:10D6D0007BE04FF4A061A01C00F0EEF920802088D0
:10D6E000002824DDA0780D2803D1E0780A2800D195
:10D6F0006BE08F48007820B10022A11C104605F095
:10D70000D3FEA01CF9F7D0FC002043490872A07892
:10D710002B2802D0A0785E2808D1A01C01F080FC44
:10D72000012800D151E0A01CF7F7D0FB4DE0208884
:10D73000002805DA01227CA1002005F0B5FE44E0B6
:10D740000120DFF81CC100DF3348007818B9012040
:10D7500003F064FD16E030488078002803DD0320E4
:10D7600003F05CFD0EE02C480079002807DD2A4814
:10D770008079002803DD042003F050FD02E0022040
:10D7800003F04CFD0020FBF791F917484078012881
:10D7900001D102F013FE05F031FF09F057FF1D48DB
:10D7A00090F8B90200B186E6DFF878C000DF614981
:10D7B0000968884200D208E0DFF868C000DF643002
:10D7C0005C490860F7F7D2FE00BF5FE7CE09002092
:10D7D00034010020506F63205461736B20737461B7
:10D7E0007274210000000020000100204D6F64656C
:10D7F0006D205461736B207374617274210000009A
:10D800004D6F64656D496E69742E2E2E0000000008
:10D810000010014040390020402900203C00002039
:10D82000F8000020B1990108041F0020F61500201F
:10D830005B30315D6861726449443A2573000000D1
:10D84000780000205B30315D4661696C65640D0ACB
:10D85000456E746572204754204D6F646521000049
:10D8600049930108000C01403D00002041542B5019
:10D870004F433D3035303030300D0A004154453093
:10D880000D0A00005B30325D41544530204F4B00A3
:10D8900018000020980F00205B30385D43617264EF
:10D8A00020726561647900005B31305D5273745F92
:10D8B000504F4350617261005B31305D504F4320E7
:10D8C0007374696C6C0000005B31325D4869676F8E
:10D8D00073536572496E6974000000004D6F646592
:10D8E0006D4C6F6F70537461727400005B31355D05
:10D8F0005273745F466F7461446F6D61696E0000AE
:10D900005B31355D466F7461446F6D61696E207384
:10D9100074696C6C0000000041542B504F433D3043
:10D9200033303030300D0A00517565756546310071
:10D93000400400204C01002000210748DFF81CC0F3
:10D9400000DF07E04FF6FF710348DFF814C000DF87
:10D9500009F04EF8F6E700002C010020519701086D
:10D9600091970108042009494861012208A100207B
:10D9700005F09AFDF9F726F806E00020084908723C
:10D980006420DFF820C000DFF7E70000001001404E
:10D99000676F2047545F4D6F64650D0A00000000FB
:10D9A00040290020499301082DE9F047054600274A
:10D9B00034480468002640F23338DFF8CC90042065
:10D9C00032490861002C00DA55E031484068A04235
:10D9D00000D850E015B100200CF090FA06EB0801D9
:10D9E00004EB440000EBC4022948083000EB82003D
:10D9F000406A81420AD904EB440000EBC401244888
:10DA0000083000EB8100406A871B00E04746FBF7C7
:10DA100019FE04EB440101EBC4021D49083101EB7E
:10DA200082000021F7F72CFE04EB440101EBC40255
:10DA30001749083101EB82004B463A46314600F067
:10DA400029F804EB440101EBC4021149083101EB50
:10DA5000820009F05DFA04EB440101EBC4020C49B9
:10DA6000083101EB82000121F7F70AFE15B1012010
:10DA70000CF044FA00BF0420044948613846BDE870
:10DA8000F08700003C040020AB560020001001404D
:10DA900040B200202DE9F04180460C4615461E4656
:10DAA00004482718AAB2394630460CF06DF9BDE893
:10DAB000F081000000F01F002DE9F84380460E467B
:10DAC000304C3148007820B930A009F04BFEFFF708
:10DAD00049FFA08810B90020BDE8F8836188A01D27
:10DAE00030F82100ADF800006188A01D00EB810036
:10DAF0004088ADF802000027002522E0B4F8D000ED
:10DB000000B922E0CE34D4F80A00E18810F8019080
:10DB1000E088401CE080E08834F8CE19884202DBBF
:10DB20000020A4F8D400B4F8D000401EA4F8D0001F
:10DB3000B74204DA3846791C8FB208F80090681CA6
:10DB400085B2BDF80000A842D8DC00BF6088401C48
:10DB500060806088322801DB00206080A088401E41
:10DB6000A080BDF80000A84202D06FF00100B3E72A
:10DB7000BDF80000B04202DD4FF0FF30ACE7BDF869
:10DB80000000A9E7C0ED00203401002053544F509D
:10DB900020474F2047540D0A0000000030B50346CF
:10DBA0000A4612480024048084804480002108E052
:10DBB0000025841D04EB81046580841D24F8215018
:10DBC000491C3229F4DBC0F8D830002104E00024DD
:10DBD000D0F8D8506C54491C9142F8DB20F8CE2F75
:10DBE00000248480C4804480CE3830BDC0ED002045
:10DBF00070B504460A4622498888322802DB4FF075
:10DC0000FF3070BDB1F8D0001044B1F8CE50A8423A
:10DC100002DD6FF00100F4E7B1F8D2500E88881DE4
:10DC200000EB860045800D88881D20F82520002304
:10DC300017E0E05CD231D1F806500E88A85508886C
:10DC4000401C088031F8D209B0F5C05F02DB00202B
:10DC5000A1F8D200B1F8D000401CA1F8D000581CA7
:10DC600083B29342E5DB0888401C0880088832288C
:10DC700001DB002008808888401C88800020C0E7E5
:10DC8000C0ED002000B54FF4C0510248FFF786FFF9
:10DC900000BD0000C0D5002010B50120F9F714FC2C
:10DCA00048210548F6F733FB122000F04DF800201C
:10DCB0000249087010BD0000E05900204C0400200B
:10DCC0007047000070B5002100230F22C47804B310
:10DCD000154C246804F4E064C4F5E064210AC1F141
:10DCE0000403CA40447804FA03F1847814402143C1
:10DCF00009010E4C0678A155047804F01F05012493
:10DD0000AC4005786D11AD0005F1E025C5F8004186
:10DD100009E0047804F01F050124AC40044D0678A6
:10DD2000761145F8264070BD0CED00E000E400E0FF
:10DD300080E100E002490143024A1160704700009F
:10DD40000000FA050CED00E0024948710121014A8A
:10DD500011717047E05900202DE9F04104460D464D
:10DD600016461F462580A67014223946E01CF6F799
:10DD7000F7FAE01CF6F700FB6076607EC006000E46
:10DD8000A0761020E07600202076BDE8F08100002B
:10DD900070B50446217EE01C455C164800681649B3
:10DDA000084498B1B0F5001F03D0B0F5601F1ED134
:10DDB0001BE0392D02DA681CC5B200E03025217E57
:10DDC000E01C4554204600F019F810E0217E607EEA
:10DDD000401E814203DA207E401C207601E00020B4
:10DDE0002076204600F00AF801E0022070BD00BF56
:10DDF0000020FBE7B8000020D6FB43FF2DE9F041EF
:10DE00000446A678E77E3E44103EB3B22688A77E3D
:10DE10003E44B2B2A1782088FBF77AF8207EC50094
:10DE2000A17820880123E21CFBF728FB20882844E6
:10DE300085B2A178102308222846FBF7AFF9BDE888
:10DE4000F0812DE9F0410446A678E77EF319268893
:10DE5000A77E3E44B2B2A1782088FBF713F8207E5B
:10DE6000C500A17820880123E21CFBF707FB20886E
:10DE7000284485B2BDE8F0810B48016801F40070C8
:10DE8000B0F5007F0BD109480078052805DA07486E
:10DE90000078401C054A107004E001207047002003
:10DEA000024A10700020F9E7080C014079000020B8
:10DEB0000EB50121084601F0EDFD04208DF80300A8
:10DEC00003208DF802004FF40070ADF800006946A1
:10DED0000B48F9F7D5FB09210120F9F7B1FB4FF405
:10DEE0000070019000208DF8080008208DF80900CE
:10DEF00001208DF80A0001A8F8F71AFD0EBD0000F8
:10DF0000000C014070B50446002506E00120DFF852
:10DF100010C000DFFBF796FB6D1CA542F6DB70BD61
:10DF20004993010810B51248FFF732FF1148006805
:10DF30001149884213D1062210490D48C01CF6F73A
:10DF400030FA18B9172007F05BF808E00CA004F0CD
:10DF50008FFE6420FFF7D6FF062007F051F8054832
:10DF600000680A49884202D1062007F049F810BD2E
:10DF70001C4B0020B80000202A04EC005E000020AA
:10DF8000C3DCC2EBB4EDCEF3000000002A04F400C1
:10DF9000F0B5A7B000273148FCF73EFD06463048F3
:10DFA000864203D1062007F02BF855E02D48864223
:10DFB00052D12A4884792C480078012803D0022CB9
:10DFC00001DBA01CC4B2294890F89C00A04240D0BC
:10DFD000264880F89C4026A004F04AFE0020FFF767
:10DFE000E3FC0AF09BFA0AF0C9FA05460AF07CFA4B
:10DFF0000746F8F71FF81C480078012807D12B4680
:10E000001EA232211AA8009709F0BCFB08E02048A4
:10E010000095D0F81D301FA232211AA809F0B2FBDA
:10E0200001A91AA8F6F7A4FE1EA0FFF7D1F801A8CF
:10E03000FFF7CEF81FA0FFF7CBF8FBF703FB142088
:10E04000DFF874C000DF1DA0FFF7C2F86420FFF7FF
:10E0500059FF012006F0D4FF27B0F0BD584700203B
:10E060002A04F4002A04EC0028000020AB5600200B
:10E07000C5E4D6C3CDEAB3C90000000069703D25F0
:10E08000733B646F6D61696E3D25733B000000005A
:10E09000C415002069643D256C643B69703D25739F
:10E0A0003B00000041542B504F433D303130303065
:10E0B000300000000D0A00004993010841542B5024
:10E0C0004F433D3034303030300D0A000149086292
:10E0D0007047000000000E420349096841EA8001D0
:10E0E000014A1160704700000070004001460020A6
:10E0F000034A52680A400AB1012000E0002070473C
:10E10000007000402DE9FC470446884691460025F2
:10E1100023212046F6F7FBF8AB2229466D1C6254FA
:10E120007A2229466D1C6254002229466D1C6254D5
:10E130001F2229466D1C62542D48D0F81D00019005
:10E140009DF8072029466D1C62549DF8062029463B
:10E150006D1C62549DF8052029466D1C62549DF883
:10E16000042029466D1C6254002607E02148825D88
:10E170002946681C85B26254701C86B2142EF5DBE9
:10E18000CDF804809DF807202846691C8DB22254E2
:10E190009DF806202846691C8DB222549DF8052062
:10E1A0002846691C8DB222549DF804202846691C1B
:10E1B0008DB22254CDF800909DF801202846691CAC
:10E1C0008DB222549DF800202846691C8DB222543D
:10E1D0000027002603E0A05D4740701C86B2AE42D7
:10E1E000F9DB2846691C8DB227542846BDE8FC8718
:10E1F000C4150020085A00202DE9FC4104460025E2
:10E200001D212046F6F783F8AB2229466D1C625487
:10E210006A2229466D1C6254002229466D1C6254F4
:10E22000192229466D1C62542048D0F81D00019027
:10E230009DF8072029466D1C62549DF8062029464A
:10E240006D1C62549DF8052029466D1C62549DF892
:10E25000042029466D1C625414211548F6F757F81E
:10E2600014480088114B213313A214210090104848
:10E2700009F088FA002607E00D48825D2846691CEF
:10E280008DB22254701C86B2142EF5DB00270026B6
:10E2900003E0A05D4740701C86B2AE42F9DB284621
:10E2A000691C8DB227542846BDE8FC81C4150020A6
:10E2B000085A00204404002025735F5625642E620E
:10E2C000696E00002DE9F04F89B004460D461646F0
:10E2D0001F46A02C01DA802D02DB09B0BDE8F08FCB
:10E2E000A019A02802DDC4F19F0086B2E819802899
:10E2F00002DDC5F17F0087B2FBF7A4F9E819401EE3
:10E3000083B2A019401E82B229462046FBF77AFF4D
:10E310004FF000083FE005EB080008904FF0000ABE
:10E3200035E0089800EB80001D4901EB401004EB3C
:10E330000A01405C079007984FEA8009194810F8D5
:10E3400009000490174909F10100085C059009F1E2
:10E350000200085C06900698C01003900598801093
:10E3600002900498C01001900398C102029801EB3A
:10E370004011019808441FFA80FB4FEA2B20FCF75C
:10E3800001F90BF0FF00FCF7FDF80AF1010AB245B4
:10E39000C7DB08F10108B845BDDB00BF9DE7000001
:10E3A00040620020405E00202DE9FF4F8DB01A989A
:10E3B00000F0F00009901A9800F00F000890002576
:10E3C0000F9810BB099838B94FF0080910264FF084
:10E3D00001084D4F4D4C06E04FF0100918264FF044
:10E3E00002084B4F4B4C07E021781098814200D136
:10E3F00005E0641C681C85B220780028F4D100BFB9
:10E4000005FB08F000FB06772EE0099880B94FF075
:10E41000100910264FF002086F46002400256A46B6
:10E42000DDE90F01F9F792FD20281DD03A4F1BE0DE
:10E430004FF0180918264FF00308384F384C0BE0FE
:10E4400021780F98814204D161781098814200D1DF
:10E4500005E0A41C681C85B220780028F0D100BF1C
:10E4600005FB08F000FB06770E983044802802DB9D
:10E4700011B0BDE8F08F0D984844A02800DBF7E705
:10E480004FF0000B3CE00E98584480B20C904FF0D7
:10E49000000A2FE00D9800EBCA0080B20B9017F82D
:10E4A000010B0A9000251FE0802028410A990840AE
:10E4B00058B11C4801780C9800EB80001A4A02EB16
:10E4C00040120B98284411540CE0089850B117489A
:10E4D00001780C9800EB8000134A02EB40120B9875
:10E4E00028441154681C85B2082DDDDB0AF10100B7
:10E4F0001FFA80FAC245CDDB0BF101001FFA80FB49
:10E50000B345C0DB00BFB3E714A60108B4A50108FA
:10E5100041AC010827AC010804AC0108F8B00108BF
:10E52000F1B0010887040020406200208804002028
:10E530002DE9F04704460D46DDF820C0002116E025
:10E540006F1801FB02F600200EE006EB00081CF835
:10E55000088007EB8709DFF820A00AEB491904EBD4
:10E56000000A09F80A80401C9042EEDB491C9942DF
:10E57000E6DBBDE8F0870000406200202DE9F04FA7
:10E58000EBB082467C22FC494CA8F5F7A7FE4FF081
:10E59000000800200590049040F20311082001F0CB
:10E5A00003FF00BF404608F101084CA951F82000C4
:10E5B00000780028F6D1A8F101084FF483710820F3
:10E5C00001F0F2FE002621E04CA850F826900AF156
:10E5D000030B0020069007900FE099F800009BF8CD
:10E5E0000010884202D0012006900AE009F10109DA
:10E5F0000BF1010B0798401C079099F800000028C8
:10E60000EBD100BF069800B902E0761C4645DBDB83
:10E6100000BF4FF48D71082001F0C6FE464502D1BF
:10E620006BB0BDE8F08F1E2E2DD2DFE816F01E0075
:10E630002D003B0065006600C80036019001A9026C
:10E64000D102E202EF0247035403850395039603C8
:10E65000970398039903C303D003DC032C00DD0365
:10E66000DE03DF03E003E1030E04092002F006FEEF
:10E670000122C2A1002004F017FF0220F7F756FE86
:10E680000120C1490870EEE3092002F0F7FD0122E4
:10E69000BEA1002004F008FFF9F7D4F80120F7F735
:10E6A00045FEE0E3092002F0E9FD0122BAA10020C5
:10E6B00004F0FAFE0220F7F739FE4FF40050B94992
:10E6C00048610420B8490860C001B6490861FEF7F6
:10E6D000E1FDFEF727FE0120B44908600220086032
:10E6E000091D086007E0FAF7ADFFFFF7C5FB10B1A1
:10E6F0000420AC494861F6E7B5E326AAACA1504630
:10E70000F9F7C8FE0446012C01DB282C05DB0122A9
:10E71000A8A1002004F0C8FEA5E326A91CA8F5F7CF
:10E720004DFE26AAA9A15046F9F7B4FE04460CB93D
:10E7300000250BE0052C05DD0122A6A1002004F038
:10E74000B3FE90E326A8F5F789FE85B226AAA8A114
:10E750005046F9F79FFE0446012C01DB142C05DB23
:10E760000122A5A1002004F09FFE7CE326A912A8A7
:10E77000F5F724FE26AAA8A15046F9F78BFE044619
:10E78000012C01DB142C05DB0122A6A1002004F0E2
:10E790008BFE68E326A908A8F5F710FE08A812A9C1
:10E7A0001CABA8A2CDE900510290962126A808F042
:10E7B000E9FF012226A9002004F076FE53E326AAF1
:10E7C0007BA15046F9F766FE0446012C01DB282C9C
:10E7D00005DB0122A6A1002004F066FE43E326A982
:10E7E0001CA8F5F7EBFD26AA78A15046F9F752FED2
:10E7F00004460CB900250BE0052C05DD0122A2A181
:10E80000002004F051FE2EE326A8F5F727FE85B27E
:10E8100026AAA4A15046F9F73DFE0446012C01DBCF
:10E820000A2C05DD0122A0A1002004F03DFE1AE320
:10E8300026A8F5F720FE0746A248D0F81D00B842EA
:10E8400004D0A048C0F81D70012005909E4890F8A3
:10E850009C00042805D004209B4981F89C000120DD
:10E8600004901CA99948F5F78EFD28B11CA997487A
:10E87000F5F7A4FD012004909248D0F81D00934BB9
:10E8800093A29621CDE9005026A808F07BFF012233
:10E8900026A9002004F008FEE5E226AA44A150467D
:10E8A000F9F7F8FD0446012C01DB282C05DB0122D9
:10E8B0008FA1002004F0F8FDD5E226A91CA8F5F7E9
:10E8C0007DFD26AA41A15046F9F7E4FD04460CB9A6
:10E8D00000250BE0052C05DD01228BA1002004F0B2
:10E8E000E3FDC0E226A8F5F7B9FD85B2764890F8B9
:10E8F0009C00042805D00420734981F89C00012065
:10E9000004901CA971482830F5F73DFD20B96E48E8
:10E91000B0F82D03A84209D01CA96C482830F5F79F
:10E920004DFD6948A0F82D53012004906648B0F8C9
:10E930002D03664B28337BA29621009026A808F071
:10E9400021FF012226A9002004F0AEFD8BE209F090
:10E9500015FE7A490390CDE900105A48D0F81D30D1
:10E9600077A2962126A808F00DFF012226A90020F3
:10E9700004F09AFD77E2000090A0010847542B5460
:10E980004D3A4F4B000000004800002047542B54E4
:10E99000473A4F4B0000000047542B444D3A4F4B31
:10E9A000000000000010014010140140100C014054
:10E9B0004950000047542B5354503A4641494C5B50
:10E9C000495020496E76616C69645D00506F7274C5
:10E9D0000000000047542B5354503A4641494C5BC9
:10E9E000506F727420496E76616C69645D0000003E
:10E9F0004163636F756E740047542B5354503A460D
:10EA000041494C5B4163636F756E7420496E76615A
:10EA10006C69645D0000000050617373776F72640D
:10EA20000000000047542B5354503A4641494C5B78
:10EA300050617373776F726420496E76616C69649C
:10EA40005D00000047542B5354503A49503D257304
:10EA50003B506F72743D25753B4163636F756E74F7
:10EA60003D25733B50617373776F72643D2573006E
:10EA700047542B534D503A4641494C5B495020492D
:10EA80006E76616C69645D0047542B534D503A4675
:10EA900041494C5B506F727420496E76616C6964B9
:10EAA0005D00000050534E0047542B534D503A46E2
:10EAB00041494C5B50534E20496E76616C69645DF0
:10EAC00000000000C4150020AB560020E8570020CD
:10EAD00047542B534D503A49503D25733B506F726C
:10EAE000743D25753B50534E3D256C753B00000031
:10EAF00047542B5347503A4641494C5B49502049B3
:10EB00006E76616C69645D0047542B5347503A46FA
:10EB100041494C5B506F727420496E76616C696438
:10EB20005D00000047542B5347503A49503D257330
:10EB30003B506F72743D25753B000000F6150020B8
:10EB400047542B524D503A50534E3D256C753B4D1A
:10EB50004549443D25733B434E554D3D30303030A3
:10EB60003030303030303B55494D49443D30303005
:10EB7000303030303030303B49503D25733B000061
:10EB8000092002F07BFB0122BFA1002004F08CFCD5
:10EB90000120DFF800C300DF0220F7F7C7FBFEF714
:10EBA00079FB0120BC4908600220091F086005208C
:10EBB000DFF8E0C200DF0220B749086007E0FAF79B
:10EBC00041FDFFF759F910B10420B4494861F6E757
:10EBD000B348B0F82F00B24B2133B2A29621009077
:10EBE00026A808F0CFFD012226A9002004F05CFC35
:10EBF00039E1B048B0A29621036826A808F0C2FD0A
:10EC0000012226A9002004F04FFC2CE126AAAFF235
:10EC100020215046F9F73EFC0446012C01DB1E2C56
:10EC200005DD0122A8A1002004F03EFCF8E426A99D
:10EC300012A8F5F7C3FB26AAAFF224215046F9F734
:10EC400029FC0446012C01DB1E2C05DD0122A6A1B6
:10EC5000002004F029FCE3E426A908A8F5F7AEFBA0
:10EC600008A812ABA8A29621009026A808F08AFD59
:10EC7000012226A9002004F017FCAB4800680028F8
:10EC800000DAF0E0A94912A8F5F77DFB30B9A749F1
:10EC90001F3108A8F5F777FB00B9E4E012A9A348F3
:10ECA000F5F78CFB08A9A1481F30F5F787FB032077
:10ECB0009F4981F8DD0101200490D4E09B4B1F3374
:10ECC0009A4A9CA126A808F071FD012226A90020DD
:10ECD00004F0EAFBC7E026AA9EA15046F9F7DAFB4A
:10ECE000044624B126A8F5F7B9FB064601E040F238
:10ECF0006E3626AA98A15046F9F7CCFB044624B1FB
:10ED000026A8F5F7ABFB85B200E0082504F0F2FC7D
:10ED10002946304601F09EFD05EB85004000334654
:10ED20008EA29621009026A808F02CFD012226A98B
:10ED3000002004F0B9FB96E07D48B0F82D038B4B22
:10ED40008BA29621009026A808F01CFD012226A97E
:10ED5000002004F0A9FB86E085E084E083E082E007
:10ED600026AA89A15046F9F795FB0446002C01DB41
:10ED70001E2C05DD012286A1002004F095FB4FE446
:10ED800024B900216A4880F8DF1104E026A97748F9
:10ED90007A30F5F713FB754B7A3385A2962126A8B6
:10EDA00008F0F0FC012226A9002004F07DFB0120E0
:10EDB000049058E06D4B7A3382A2962126A808F081
:10EDC000E1FC012226A9002004F06EFB4BE0642246
:10EDD0004FF4601126A80AF061FF012226A9002045
:10EDE00004F062FB3FE03EE03DE03CE03BE03AE027
:10EDF00026AAAFF250315046F9F74CFB0446012CDD
:10EE000001DB0A2C05DD012273A1002004F04CFB7C
:10EE100029E026A8F5F72FFB07462148D0F81D006A
:10EE2000B84204D01E48C0F81D70012005901C484F
:10EE3000D0F81D306FA2962126A808F0A3FC01226D
:10EE400026A9002004F030FB0DE01548D0F81D3055
:10EE50006DA2962126A808F095FC012226A9002083
:10EE600004F022FB00BF00BF059808B101F0A2FB2F
:10EE7000049810B10020FEF797FD40F2D22108203F
:10EE800001F092FA00BFD1E647542B5053543A4F49
:10EE90004B00000049930108140C01400010014090
:10EEA000C415002047542B5645523A25735F56250A
:10EEB000640000004000002047542B4241543A2097
:10EEC000256420560000000047542B41504E3A461E
:10EED00041494C5B4163636F756E7420496E766186
:10EEE0006C69645D0000000047542B41504E3A4667
:10EEF00041494C5B50617373776F726420496E7641
:10EF0000616C69645D00000047542B41504E3A41EA
:10EF100063636F756E743D25733B50617373776FD8
:10EF200072643D25733B00003C04002063590020BF
:10EF3000AB56002047542B5241504E3A4163636F09
:10EF4000756E743D25733B50617373776F72643DCA
:10EF500025733B0046000000540000004245455028
:10EF60003D2564487A2C25646D73000010580020FC
:10EF700047542B5247503A49503D25733B504F520E
:10EF8000543D25643B00000041636365737370006A
:10EF900047542B534143433A4641494C5B416363D9
:10EFA0006573737020496E76616C69645D00000062
:10EFB00047542B534143433A416363657373703D38
:10EFC00025733B0047542B524143433A41636365E9
:10EFD0007373703D25733B0047542B535049443A9B
:10EFE0004641494C5B50534E20496E76616C6964D2
:10EFF0005D00000047542B535049443A50534E3D56
:10F00000256C753B0000000047542B525049443A90
:10F0100050534E3D256C753B0000000070470000CA
:10F02000F0B5BBB0044648210BA8F5F770F960783D
:10F030004C2818D1A078532815D1E078482812D14F
:10F04000207954280FD1607A45280CD10020FE4940
:10F05000C8700846807818B94FF48070FB49486141
:10F0600001203BB0F0BD6079302827D1A07942283B
:10F0700024D1E07946280DD1207A46280AD10020F3
:10F08000F349087004F036FB0A214FF47A7001F05E
:10F09000E1FB11E0E07930280ED1207A30280BD145
:10F0A0000120E9490871EA49087004F023FB0A21AC
:10F0B0004FF4FA7001F0CEFB0120D2E760793828D6
:10F0C0007ED1A0794228FBD1E07930287DD1207A09
:10F0D000312816D109F074F90120DB490871DB49A8
:10F0E00048610020D849887001208871D84800788C
:10F0F00018B94FF48070D54948610120D249087091
:10F1000009E0207A302806D10020CF4908718871A3
:10F110000120CE490861607A30281CD1A07A3028BD
:10F1200019D1CB48007801280AD10020C8490870BD
:10F13000C548807810B10020C3498870012090E74D
:10F140000020C149887004F0D5FA0A214FF4FA7002
:10F1500001F080FB37E0607A30281AD1A07A31289C
:10F1600017D109F02DF90020FBF734F80020B94938
:10F1700008800120B4490870887004F0BBFAB648D2
:10F1800090F8F702F8B10A214FF4FA7001F062FB2F
:10F1900019E0607A312816D1A07A332813D1AC480F
:10F1A0000078012802D10020A94908700121AB484C
:10F1B00080F8B81204F09EFA0A214FF47A7000E049
:10F1C00003E001F047FB01204BE76079382870D15C
:10F1D000A0793228FBD1E0798DF87800207A8DF87B
:10F1E000790000208DF87A001EA8F5F737F9C7B22C
:10F1F00037B1012F73D0022F72D0032F71D1AFE03E
:10F200000021964880F8B71200208F490870944872
:10F21000007820F010009249087092A266211EA882
:10F2200008F0B0FA607C422814D1A07C352811D1B6
:10F23000607E43280ED1A07E41280BD105208B494A
:10F2400008700121854880F8BB1289A11EA8F5F736
:10F2500069F84BE0607C432816D1A07C452813D187
:10F26000607E432810D1A07E32280DD17B4890F8D3
:10F27000BB02012803D00221784880F8BB1280A18C
:10F280001EA8F5F74FF831E0607C432812D1A07C2E
:10F2900045280FD1607E43280CD1A07E312809D1AA
:10F2A00005216E4880F8BB1278A11EA8F5F73AF840
:10F2B0001CE05EE0607C432814D1A07C332811D18F
:10F2C000607E42280ED1A07E37280BD106216348EC
:10F2D00080F8BB1270A11EA8F5F724F806E00BE039
:10F2E00010E043E06FA11EA8F5F71CF801221EA94B
:10F2F000002004F0D9F839E001226DA1002004F0CB
:10F30000D3F833E004F11100F5F736F8801EC5B2EA
:10F31000242D00DB24252A4604F111016748F4F767
:10F32000DDFF00206549485547491531634804F021
:10F3300067FA0020607410221DA904F10900F5F796
:10F3400055F84149086101225DA1002004F0ACF8A4
:10F3500001205E4908700321404880F8BB1205E097
:10F3600001225BA1002004F09FF800BF00BF012034
:10F3700077E62046F8F7BAFA08B1012071E660791D
:10F3800038285FD1A07936285CD101202E49087039
:10F390001E2036490870207A30284ED104F1110021
:10F3A000F4F7EAFF801EC5B2242D00DB24252A468F
:10F3B00004F1110101A8F4F791FF002001A94855BB
:10F3C000607410221DA904F10900F5F70FF81E4919
:10F3D000C863423101A804F013FA1B484078D0B941
:10F3E0003A48007830B901AB3CA266211EA808F06B
:10F3F000C9F90AE000203549087001A82F4B38A24E
:10F40000662100901EA808F0BDF900221EA9012067
:10F41000FCF78CFB11E03848007801280DD1002062
:10F420003549087001AB35A266211EA808F0AAF97B
:10F4300000221EA90120FCF779FB0021074880F873
:10F44000B71263E066E00000402900200010014090
:10F45000FD000020A4020020AB560020403900200F
:10F46000041F00205B6D73675D0000005D000020DD
:10F47000D5CBBAC5D0C5CFA2B4EDCEF30000000005
:10F48000CEDECDF8C2E7C1ACBDD30000CEDEB7A85A
:10F49000C1ACBDD300000000C3BBD3D0B7FECEF1DA
:10F4A000000000004E6F206C6F67696E0000000066
:10F4B0006C6F67696E20696E67000000443D002034
:10F4C0006C6F67696E206F6B00000000FC0000200D
:10F4D0006C6F676F757420696E670000257300009C
:10F4E0002573324344324431423543374332424438
:10F4F00032432573000000005C000020424446387F
:10F5000043384542324325730000000001209A49E8
:10F510004870A6E5607938282BD1A079332828D106
:10F52000E079302825D1207A302822D104F1110049
:10F5300000F0ECFD04F11100F4F71EFF0646242E46
:10F5400001DB242600E0761C8B49743104F11100A4
:10F5500004F056F90020607410221DA904F109007E
:10F56000F4F744FF8449C1F89C0000206074012036
:10F5700077E5607938280AD1A079332807D1E07976
:10F58000302804D1207A312801D1012069E5607941
:10F59000392807D1A079312804D1E01DFFF73EFDBD
:10F5A00001205EE56079302824D1A079452821D159
:10F5B000002060743AA904F10D0004F021F99DF8CF
:10F5C000E9008DF8E4009DF8EA008DF8E500BDF84B
:10F5D000E40069498881012081F86C00084683892C
:10F5E00066A266211EA808F0CDF801221EA90020FF
:10F5F00003F05AFF6079382830D1A07934282DD112
:10F600002046FCF77FFA002204F109010120FCF7F3
:10F610008DFA08225CA104F10900F4F7C2FE20B9BA
:10F6200001215C4880F8B71216E008225AA104F1C3
:10F630000900F4F7B6FE20B90021564880F8B71249
:10F640000AE0102257A104F10900F4F7AAFE18B944
:10F650000121504880F8B712012002E56079322874
:10F6600069D1A079312866D12046FCF74BFA42488F
:10F6700090F86B0000EB400101EBC0013E48A03068
:10F6800000EB81000021C0F805104172607D68B96F
:10F690002021394890F86B0000EB400202EBC002D9
:10F6A0003548A03000EB820041710FE0324890F8FD
:10F6B0006B0000EB400202EBC0022F48A03000EBD1
:10F6C0008200411D04F1150004F09AF800206075D5
:10F6D0003AA904F10D0004F093F89DF8E8008DF8C4
:10F6E000E3009DF8E9008DF8E2009DF8EA008DF84E
:10F6F000E1009DF8EB008DF8E0001F4890F86B00EA
:10F7000000EB400202EBC0021B48A030389940F8E1
:10F7100022100321A03890F86B0000EB400202EBAE
:10F72000C0021548A03000EB82000171012012498F
:10F7300081F86A0095E4607931281BD1E07930289E
:10F7400018D1A07B372802D0A07B382812D11A48C4
:10F75000D4F81310C162D4F81710016304F11F002C
:10F76000FCF7D0F9002204F11F010120FCF7DEF9BB
:10F77000012076E400BF74E4402900206F6E654CE0
:10F78000696E653A25640000433144394341423192
:10F7900000000000403900204344434242334636D3
:10F7A0000000000042414634424444304233433971
:10F7B0004239413600000000C03B002008B501215D
:10F7C0001C2000F067F910208DF8030003208DF84D
:10F7D00002000420ADF8000069460348F7F750FF27
:10F7E00004200149486108BD0010014010B50948D6
:10F7F000007800B910BD0020FAF7ECFC4FF400705F
:10F8000005490861002008F055FD042002494861BF
:10F8100000BFFEE73D0000200010014070B5054626
:10F820000E46314608A007F09DFF002405E0295D43
:10F8300008A007F097FF601C84B2B442F7DB07A072
:10F8400007F090FF70BD0000446174615B25645D4A
:10F850003A0D0A0025303278000000000D0A000041
:10F8600070B59AB006460C4604F078FB072000906D
:10F870000848D0F81D10084B4FF4817201A804F01D
:10F880007FFA85B22A4601A90020FBF74DFC2046ED
:10F890001AB070BDC4150020AC03002070B59AB03A
:10F8A00004460D46607AA17AC8B21249088108461A
:10F8B000038911A2642101A807F064FF012201A9B4
:10F8C000002003F0F1FD04F049FB1C2000900E48DD
:10F8D000D0F81D100D4B40F2013201A804F050FA8F
:10F8E00086B2324601A90020FBF71EFC28461AB05A
:10F8F00070BD0000041F00205B47707354696D6584
:10F900003D25645D00000000C41500203454002033
:10F9100070B59AB005460E4604F020FB1C200090FE
:10F920000848D0F81D10084B48F2012201A804F045
:10F9300027FA84B2224601A90020FBF7F5FB00203C
:10F940001AB070BDC41500203454002070B50446B0
:10F950000D4609480078C0F3800058B90648007881
:10F9600020F00400001D04490870012203A10020BA
:10F9700003F09AFD002070BD041F00205B477073E8
:10F98000204C6F67696E65645D00000070B59AB0C9
:10F9900005460E4604F0E2FA1C2000900848D0F814
:10F9A0001D10084B48F2010201A804F0E9F984B2E5
:10F9B000224601A90020FBF7B7FB00201AB070BD5A
:10F9C000C41500203454002070B59AB006460C4689
:10F9D0000E480078012802D104F052FB01E004F047
:10F9E000EFFB2E2000900A48D0F81D10094B4FF471
:10F9F000807201A804F0C4F985B22A4601A900204A
:10FA0000FBF792FB20461AB070BD0000F00000200A
:10FA1000C41500205054002070B59AB005460E461B
:10FA200004F09CFA1C2000900848D0F81D10084BE8
:10FA3000022201A804F0A4F984B2224601A9002000
:10FA4000FBF772FB00201AB070BD0000C415002047
:10FA50003454002029B1064A52690243044B5A61CA
:10FA600004E0034A52698243014B5A617047000027
:10FA70000010024029B1064AD2690243044BDA6100
:10FA800004E0034AD2698243014BDA617047000007
:10FA90000010024029B1064A92690243044B9A6160
:10FAA00004E0034A92698243014B9A617047000067
:10FAB000001002400348406A40F0807001494862EB
:10FAC00070470000001002402DE9F04100210022A3
:10FAD000002500230026002400278C46DFF86081E3
:10FAE000D8F8048008F00C0121B1042907D00829B6
:10FAF00059D109E0DFF84C81C0F8008058E0DFF808
:10FB00004481C0F8008053E0DFF83481D8F80480E5
:10FB100008F47012DFF82881D8F8048008F48035E2
:10FB2000920C0D2A01D0921C00E0062235B9DFF8B4
:10FB3000188102FB08F8C0F8008033E0DFF800818C
:10FB4000D8F82C8008F48036DFF8F480D8F82C80C0
:10FB500008F00F0808F1010446B9DFF8E880B8FBA7
:10FB6000F4F808FB02F8C0F800801BE0DFF8D08052
:10FB7000D8F82C80C8F3031808F10107DFF8C0801B
:10FB8000D8F82C80C8F3032808F1020CDFF8B48001
:10FB9000B8FBF7F808FB0CF8B8FBF4F808FB02F820
:10FBA000C0F8008004E0DFF89C80C0F8008000BF4F
:10FBB00000BFDFF88C80D8F8048008F0F001090954
:10FBC000DFF8888018F80130D0F8008028FA03F8B0
:10FBD000C0F80480DFF86880D8F8048008F4E06199
:10FBE000090ADFF8688018F80130D0F8048028FA94
:10FBF00003F8C0F80880DFF84880D8F8048008F4DB
:10FC00006051C90ADFF8448018F80130D0F8048048
:10FC100028FA03F8C0F80C80DFF82480D8F80480B4
:10FC200008F44041890BDFF8288018F80130D0F83B
:10FC30000C80B8FBF3F8C0F81080BDE8F08100003C
:10FC400000100240001BB700808D5B0051040020B3
:10FC50006104002010B501460022002300204A1153
:10FC6000012A02D1094C236806E0022A02D1074C7E
:10FC7000236A01E0054C636A01F01F0201249440ED
:10FC80001C400CB1012000E0002010BD001002401B
:10FC900001490860704700003C0442420249096A79
:10FCA0000143014A116270470010024010B5022062
:10FCB00000F062F898B10120094908704004F6F795
:10FCC00025FE0120FEF712FA10B10120FEF704FA1A
:10FCD00000F0B6F8022000F005F800F0B1F810BD11
:10FCE00020040020024909888143014A118070479D
:10FCF0000428004010B501214FF0C050FFF7BAFEB4
:10FD00000120FEF7E3F910BD10B54FF40070FFF7C6
:10FD1000C5FF0120FFF7BCFF00F09CF800F090F851
:10FD20000121084600F05EF800F08AF847F6FD7001
:10FD300000F076F800F084F810BD00000348008859
:10FD400040F010000149088070470000042800407E
:10FD5000034800884FF6EF7108400149088070475A
:10FD600004280040002103480188001F008841EA60
:10FD7000004070471C28004001460020064A1288B7
:10FD80000A40D0B2044A121F12880A4012B108B1C8
:10FD9000012000E0002070470428004010B5012039
:10FDA000FFF7EAFF10B10120FFF79CFF0220FFF7E9
:10FDB000E3FF98B101200A4908704004F6F7A6FD58
:10FDC0000120FEF793F910B10120FEF785F900F04C
:10FDD00037F80220FFF786FF00F032F810BD000070
:10FDE0002004002029B1064A12880243044B1A80DD
:10FDF00004E0034A12888243014B1A8070470000D6
:10FE00000028004000B50246FFF798FF100C034998
:10FE10000880091D0A80FFF79BFF00BD18280040DD
:10FE200000B50246FFF78AFFC2F30340034908808A
:10FE3000091D0A80FFF78CFF00BD00000828004064
:10FE400000BF0348008800F020000028F9D0704768
:10FE500004280040074800884FF6F771084005491C
:10FE6000088000BF0348008800F008000028F9D08F
:10FE7000704700000428004038B5002407E01E4801
:10FE80001E4941F8240000201D490855641C052C1A
:10FE9000F5DD002416E004EB440000EBC401194832
:10FEA00000EB81000079401E1549085504EB440021
:10FEB00000EBC401134800EB8100401D0F4941F8DD
:10FEC0002400641C0F48A03890F86B00A042E2DCCC
:10FED0000C48A038808928B90BA008490860002088
:10FEE000074908550648094B002204490090084874
:10FEF000FAF7C0FC38BD0000E8010020044B0020E8
:10FF0000E9010020E0290020BFD50000D801002031
:10FF1000584700202DE9F04704460D4617469846FD
:10FF2000002C02DA0020BDE8F08719484068A042A2
:10FF300001D80020F7E7E91904EB440000EBC40204
:10FF40001348083000EB8200406A81420AD904EB72
:10FF5000440000EBC4010E48083000EB8100406A09
:10FF6000461B00E03E4604EB440000EBC401084899
:10FF7000083000EB8100806A00EB050909F5805923
:10FF8000B2B24946404609F089FE3046CBE7000050
:10FF900040B20020F0B505460B4616460027002467
:10FFA0000DE0281900F003FB024638467F1C1A5466
:10FFB0004FEA122C38467F1C03F800C0A41CB44240
:10FFC000EFDBF0BD10B50024F9F73CFB32221C49F1
:10FFD0001C48FFF7DFFF1A48D0F81D001A49884275
:10FFE00008D31748D0F81D100022184B591A72EB8D
:10FFF000020009DA1248D0F81D1015A007F0B2FB74
:020000040801F1
:1000000000200F49C1F81D000D48B0F82F00B0F5D1
:10001000D87F05D04FF4D8700949A1F82F000124EA
:1000200010A107482130F4F7AEF928B10DA104481A
:100030002130F4F7C3F901240CB100F0BBFA10BD74
:10004000C415002000F8010840420F0000EA56FAEB
:1000500050534E20696E76616C69643A25780D0ABA
:100060000000000048533139314C00007FB5044690
:100070006D461C48C2881C4800EB8200006800F1F5
:1000800010014FF4C872204609F008FE1548C288D6
:10009000154800EB820001680222284609F0FEFDA7
:1000A00000208DF801000F48C2880F4800EB820045
:1000B00001680222284609F067FE0B48163880883E
:1000C00070B1094816388088401E07491639888063
:1000D0000846808820B90846007820F001000870A2
:1000E0007FBD0000584700206A52002010B5012251
:1000F00003A1002003F0D8F904F062F810BD00005D
:100100005472792D526567210000000002461146A5
:1001100007E00D2801D00A2802D100230B7003E06C
:10012000491C08780028F4D100BF704710B50220A0
:100130000B4908606420DFF82CC000DF022008496A
:10014000091D08600120091F08606420DFF814C041
:1001500000DF01200249091D086006F04DFE10BDB8
:10016000100C01404993010810B5F7F7C9FF10BD05
:100170002DE9F04786B00026764890F88B004E288F
:1001800002D0522812D10BE0012073494870714807
:10019000D0F88C00C1F80600012006B0BDE8F08759
:1001A00001226EA1002003F07FF909E001226EA177
:1001B000002003F079F90020674948700520ECE73A
:1001C00000BF01236BA20A210020F9F757F9012093
:1001D00074238022642100901D20F8F7FAFE4FF46A
:1001E000407A4FF4FA284FEA1837C8F30B0008B1E9
:1001F000781C87B200251BE00AEB050009F02CFDF6
:100200000A2095FBF0F100FB115008B1F9F71AFA3A
:100210006420684390FBF7F0C6B2FF2006F11D0290
:100220007223662100901D20F8F71AFF681C85B222
:10023000BD42E1DB012354A20A210020F9F71EF997
:1002400073237F2265211E20F8F762FE0DF1080955
:1002500000244DE000208DF808008DF80900ADF86D
:100260000E00CDF80A0044B94C4804904C48059063
:1002700039490498C1F80A0013E040F2E73084429B
:1002800005D1484804904FF44010059009E0601EE5
:100290004FF4401101EB40200490601C01EB402022
:1002A00005904FF4401000EB44211022484609F01D
:1002B0006BFD142094FBF0F100FB114008B1F9F73D
:1002C000C1F90A2094FBF0F100FB114078B96420D9
:1002D00060434FF47A7190FBF1F0C6B2012006F151
:1002E0001D020346722100906620F8F79EFE641CF2
:1002F000B4F57A7FAEDB4E20164981F88B004FF4BF
:100300004010C1F88C000020FDF74EFB4FF4401068
:100310001149C1F80600002048808880084600780E
:1003200020F0010008700846007820F002000870F4
:100330000846007820F0040008700120487003F09F
:10034000D7F810224FF44011484609F0A7FC0020CE
:1003500023E70000AB560020545200205B534D535E
:100360005D526573657400005B534D535D52457279
:10037000723300002020CFFBCFA2C4DAB4E6C5E47C
:10038000D6C3312F322000002020CFFBCFA2C4DA09
:10039000B4E6C5E4D6C3322F3220000000CE3700C9
:1003A0000002300000CC3700024A1080024A11607F
:1003B000704700006400002068000020F0B589B09C
:1003C0002F488078D0B1DFF8BCC000DF2E49096823
:1003D000884213D9DFF8ACC000DF64302A490860D6
:1003E0002748C078401CC0B22549C870142805DDD4
:1003F00000208870012225A103F056F820480078DB
:10040000012803D01E480078022836D11C48B0F8D5
:10041000961120A007F0A6F9194D083500240FE029
:10042000A01C2E5CE01C2F5C295DA01C2954601CC4
:10043000295CE01C29542E55601C2F54201D84B2C9
:100440000F48B0F89601A042EADC012003F044F91D
:10045000032314A21E2101A807F094F901A8FCF7B8
:10046000B7FE2846FCF7B4FE12A0FCF7B1FE01204F
:100470001149C87000200249087009B0F0BD0000A1
:100480006A3D0020B19901087802002054696D6529
:100490006F7574005454535F4C454E3A25640D0AF1
:1004A0000000000041542B4C53485454533D2564E4
:1004B0002C220000220D0A004029002021B10288D0
:1004C00042F04002028004E002884FF6BF731A40F7
:1004D000028070470246002013890B400BB10120B7
:1004E00000E000207047014688897047818170478D
:1004F00010B50022028802F441520B884C88234335
:100500008C882343CC8823430C8923434C89234381
:100510008C892343CC8923431A430280838B4FF277
:10052000FF74234083830B8A038210BD10B50446F9
:1005300000BF02210A48FFF7CDFF0028F9D021466D
:100540000748FFF7D3FF00BF01210548FFF7C2FFAF
:100550000028F9D00248FFF7C6FFC0B210BD000066
:100560000030014001461CE000BF00BF00BF00BFDB
:1005700000BF00BF00BF00BF00BF00BF00BF00BF83
:1005800000BF00BF00BF00BF00BF00BF00BF00BF73
:1005900000BF00BF00BF00BF00BF00BF00BF00BF63
:1005A00000BF0A1EA1F1010399B2DDD170470146D7
:1005B0000888704710B504200549086132220549B2
:1005C000054807F081F804200149486110BD00008A
:1005D00000100140C415002000F8010810B51948AA
:1005E000FAF71AFA0446184884421DD117A002F0FF
:1005F0003FFB1A4890F8DD011249C98888420FD0A4
:1006000010488079154981F8DD010020FDF7CCF90B
:10061000C820DFF84CC000DF01201249087010E04C
:10062000062004F0EDFC0CE00F48844203D11320B7
:1006300004F0E6FC05E00D48844202D1062004F0F7
:10064000DFFC10BD584700202A04EC00BCB4BDAB51
:10065000D6D8C6F4B8FCD0C22E2E2E00AB56002041
:10066000499301083D0000202A047C002A04F4007C
:1006700038B50446002C43D02248007801280AD01F
:1006800021A002F0F5FAC820DFF888C000DF0620BC
:1006900004F0B6FC38BD2048007801280AD11FA01C
:1006A00002F0E6FAC820DFF86CC000DF062004F094
:1006B000A7FCEFE7F8F7D2FB02211CA002F09CF99F
:1006C000012314229F210020F8F76CFC0120194916
:1006D00091F8DD11184A50541046184B0022184961
:1006E00000901848FAF7C6F8012368229F210020DD
:1006F000F8F758FC012314A26E210020F8F7BEFE83
:1007000000BFC7E780040020BDFBD6B9D0DEB8C467
:100710000000000049930108D5020020C5E4D6C3BB
:10072000CEC4BCFECEDE41504E000000C9E8D6C3A8
:1007300041504E00AB560020D7020020BC020020E2
:10074000A8020020584700205B4F4B5DC7D0BBBBC1
:1007500020205B50315DCFEAC7E9000010B51D488D
:1007600000681D49884212D11C480078401C1B4972
:100770000870084600781A490978884202DB002090
:10078000164908701548007801F00CFF21E0114867
:1007900000681449884214D11048007818B91048EC
:1007A00000780E4908700D480078002804DD0B48D9
:1007B0000078401E094908700848007801F0F2FEF0
:1007C00007E0044800680849884202D1122004F07A
:1007D00017FC10BDB80000202A04BC00C80200208D
:1007E000D50200202A04DC002A04F40010B50446D7
:1007F000F4B1F8F733FB02210EA002F0FDF801235B
:1008000014229F210020F8F7CDFB00200B4908702F
:100810000846007801F0C6FE012368229F210020CF
:10082000F8F7C0FB012306A26E210020F8F726FE90
:1008300010BD000041504ECFEAC7E900C8020020B9
:100840005B455849545DB7B5BBD8202020202020F7
:100850002020000070B505460C460F4890F8F702BE
:1008600020B94FF480700D49486170BD284608F0EA
:1008700013F8A0B20121DFF828C000DF09490860A1
:1008800004F1080188B20221DFF814C000DF054935
:10089000086000BFE9E70000AB56002000100140EF
:1008A000BD9901083000002070B505460C460C4883
:1008B00090F8F70200B970BD284607F0EDFF6821F7
:1008C0000720FFF771FD0121064803F003F9A0B2EC
:1008D000F5F7D4FE0021034803F0FCF800BFEAE777
:1008E000AB560020000C004043185A00FF2A00DDE0
:1008F0007047034B1870034B197000BFF8E70000F6
:10090000A2000020A300002000B589B0294800689B
:1009100029490844C0B1B0F5001F06D0B0F5401F0A
:1009200022D0B0F5601F41D13CE02448007818B9CE
:1009300002202249087004E020480078401E1F4928
:100940000870F5F793FB31E01C480078022803D1CA
:1009500000201A49087004E018480078401C174924
:100960000870F5F783FB21E0154890F8BC021349A5
:100970000978884212D011480178114880F8BC12D9
:100980000E4802780FA101A806F010FF01A8FCF79D
:100990001FFC012211A1002002F086FD012004F0BD
:1009A0002FFB03E0062004F02BFB00BF00BF09B0C3
:1009B00000BD0000B8000020D6FB43FF2404002047
:1009C0004039002041542B504F433D3430303030BB
:1009D000303031253032780D0A00000055706461E6
:1009E000746520636F6465747970650070B5044642
:1009F0000425012C28D1002023490880F8F72EFA7D
:100A0000012122A001F0F8FF012314229F210020E0
:100A1000F8F7C8FA012368229F210020F8F7C2FAEC
:100A20001D48007848B91DA002F022F96420FDF7A6
:100A300069FA062004F0E4FA06E01C4890F8BC02CB
:100A40001B490870F5F712FB0F48008830B90123E5
:100A500018A26E210020F8F711FD09E00A4800886D
:100A6000C82805D1012318A26E210020F8F706FD41
:100A700005480088401C80B203490880B0F5C87F53
:100A800001DB0020088070BD3A040020B1E0C2EB19
:100A9000C6F7C9E8D6C300003C000020C4A3BFE9E4
:100AA000D4DDCEB4C6F4B6AF00000000403900205B
:100AB000240400205BC9CF5DD1A1D4F1205BCFC25B
:100AC0005DD1A1D4F12020005B4D5DB1A3B4E6203F
:100AD000205B455849545DCDCBB3F60010B5334883
:100AE00000683349084450B1B0F5001F06D0B0F596
:100AF000401F28D0B0F5601F55D150E000BF2B48F3
:100B000000682C4988420DD12B48807A072805DAE5
:100B10002948807A401C284988720FE00020264925
:100B200088720BE02448807A18B90720224988721D
:100B300004E02148807A401E1F4988721E49887A45
:100B400000F0CEF82FE01C48807A1C4991F8F8128A
:100B5000884220D0194890F82F03002811DD16484C
:100B6000807A03280DDA1448807A50B114A002F07C
:100B70007FF86420DFF858C000DF012004F040FA5D
:100B800011E00D48807A0D4981F8F802F8F714F960
:100B90000120FCF709FF012004F032FA03E00620EF
:100BA00004F02EFA00BF00BF10BD0000B800002006
:100BB000D6FB43FF2A04DC00041F0020AB560020B4
:100BC000B5CDB9A6BAC4B7C7B7A8B2D9D7F7000090
:100BD0004993010810B5044614B3F8F73FF9012111
:100BE0002AA001F009FF01232BA258210020F8F7C9
:100BF00045FC012314229F210020F8F7D3F92B484C
:100C000090F8F8022A498872887A00F069F801237E
:100C10006A229F210020F8F7C5F9002025490880A5
:100C20002448008830B9012323A26E210020F8F760
:100C300025FC09E01F480088C82805D1012323A20C
:100C40006E210020F8F71AFC19480078C0F3400024
:100C500000B97CB11748008818B116480088C82828
:100C600008D14023A02218210020F8F70BF900201A
:100C7000F6F7C2FF0F480088401C80B20D4908807B
:100C8000B0F5C87F01DB0020088010BDB1B1B6B758
:100C9000C9E8D6C300000000B1B1B6B7C9CFB4AB44
:100CA000C9E8D6C33A202020C3EB0000AB56002091
:100CB000041F0020060300205BC9CF5DD1A1D4F141
:100CC00020205BCFC25DD1A1D4F120005B4D5DB18E
:100CD000A3B4E620205B455849545DCDCBB3F60064
:100CE0003EB50546194830F8154068239F22582123
:100CF0006420F8F70DF964B9012315A25821642086
:100D0000F8F7BCFB1023202258216C20F8F746FA94
:100D10001AE0234610A20A21684606F033FD01239B
:100D20006A4658216420F8F7A9FB632C06DD1023DE
:100D3000182258216C20F8F731FA05E010231A46E2
:100D400058216C20F8F72AFA3EBD000094A1010852
:100D500020B9D8B1D5200000202530326420C3EB63
:100D6000000000002DE9F041334804794579867987
:100D7000C779302C1AD1302D18D1322E16D1302F00
:100D800014D1B0F89601001F2B49A1F8960101205B
:100D9000087088700020C8704870012227A102F0F6
:100DA00083FB0220244981F898013BE0012C19D1F2
:100DB000022D17D12048B0F89601001F1E49A1F856
:100DC00096010220087081F898011F48007820F0F1
:100DD0000200801C1C49087001221CA1002002F0A6
:100DE00063FB1FE0202C1DD1202D1BD1202E19D1FB
:100DF000202F17D11048B0F89601001F0E49A1F816
:100E0000960100200870012081F898010E480078B2
:100E100020F00200801C0C49087001220EA1002065
:100E200002F042FB00200F4948710120087002F0D7
:100E300097FCBDE8F08100006A3D0020416C6172C2
:100E40006D537461727400005452002050757265C5
:100E500020545453000000005075726520545854BB
:100E6000000000003801002070B504460C25012C5C
:100E700021D1F7F7F3FF01211FA001F0BDFD0123F0
:100E800014229F210020F8F78DF8A8B201231EA29A
:100E90003821F8F7F3FA1F4890F8F7021E49087056
:100EA00007F010FC012368229F210020F8F77AF850
:100EB00000201A4908801948008830B9012318A277
:100EC0006E210020F8F7DAFA09E014480088C828F3
:100ED00005D1012317A26E210020F8F7CFFA0F48A1
:100EE0000088401C80B20D490880B0F5C87F01DB46
:100EF0000020088070BD0000505454CCE1CABED21E
:100F0000F4C9E8D6C3000000202020BFAAB9D83A0F
:100F100000000000AB560020D6020020780300201D
:100F20005BC9CF5DD1A1D4F12020205BCFC25DD1C0
:100F3000A1D4F1005B4D5DB1A3B4E620205B455820
:100F400049545DCDCBB3F60010B51B4800681B4972
:100F5000084450B1B0F5001F06D0B0F5401F11D0C5
:100F6000B0F5601F25D120E000BF1548007818B902
:100F700001201349087002E000201149087007F0B1
:100F8000A1FB16E00F4890F8F7020D490978884256
:100F900007D00B4800780B4981F8F7020120FCF7D5
:100FA00003FD062004F02CF803E0062004F028F8E6
:100FB00000BF00BF10BD0000B8000020D6FB43FFFB
:100FC000D6020020AB56002010B504242348006848
:100FD00023490844B8B1B0F5001F06D0B0F5401F52
:100FE00022D0B0F5601F36D131E01E480078401C99
:100FF000C0B21C490870052801DB002008700220DF
:1010000000F034F827E017480078002805DD15487F
:101010000078401E1349087002E00420114908704E
:10102000022000F023F816E00F4890F89A000D49CE
:101030000978884207D00B4800780B4981F89A005C
:101040000120FCF7B1FC062003F0DAFF03E00620E4
:1010500003F0D6FF00BF00BF10BD0000B8000020A5
:10106000D6FB43FFC9020020AB56002030B585B047
:1010700005460424012D52D1504890F89A00504959
:101080000870F7F7EBFE01214EA001F0B5FC01233B
:1010900014229F210020F7F785FFA0B201234BA265
:1010A0003821F8F7EBF946480078042805D14BA21F
:1010B0000A2102A806F066FB0BE040489030404948
:1010C000097800EB4100038846A20A2102A806F035
:1010D00059FB04F1500188B2012302AA3821F8F724
:1010E000CDF904F1500188B2102320223821F8F7FD
:1010F00055F8334803783DA20621684606F042FBC6
:1011000001226946002002F0CFF9012368229F21C5
:101110000020F7F747FF0020354908802DE0022D19
:101120002BD127480078042805D12CA20A2102A837
:1011300006F028FB0BE0214890302149097800EBAC
:101140004100038827A20A2102A806F01BFB04F134
:10115000500188B2012302AA3821F8F78FF904F16F
:10116000500188B2102320223821F8F717F8012304
:1011700068229F210020F7F715FF1D48008830B92D
:1011800001231CA26E210020F8F778F909E0184825
:101190000088C82805D101231BA26E210020F8F782
:1011A0006DF913480088401C80B211490880B0F5E1
:1011B000C87F01DB0020088005B030BDAB560020A1
:1011C000C90200204C4344C9E8D6C30020B1B3B9DA
:1011D000E2CAB1BCE43A202020200000B3A3C1C180
:1011E0002020000025336420C3EB00002533640079
:1011F000080300205BC9CF5DD1A1D4F1205BCFC231
:101200005DD1A1D4F12020005B4D5DB1A3B4E620F7
:10121000205B455849545DCDCBB3F60010B504466C
:10122000052C27D2DFE804F0030A11181F00002064
:1012300011490870012000F021F81BE001200E493F
:101240000870052000F01AF814E002200A4908701E
:10125000062000F013F80DE0032007490870042071
:1012600000F00CF806E0042003490870012000F0AB
:1012700005F800BF00BF10BDA500002010B5044652
:101280000A2C60D2DFE804F0050E172029323B4417
:101290004D560021084600F021FD00210846FFF7C9
:1012A00023FB50E00021012000F018FD002108463A
:1012B000FFF71AFB47E00121084600F00FFD00216F
:1012C0000846FFF711FB3EE00A21012000F006FD71
:1012D00000210846FFF708FB35E00021084600F032
:1012E000FDFC00210120FFF7FFFA2CE00021084659
:1012F00000F0F4FC01210846FFF7F6FA23E0002194
:10130000084600F0EBFC0A210120FFF7EDFA1AE095
:101310000021012000F0E2FC00210120FFF7E4FAA7
:1013200011E00121084600F0D9FC01210846FFF731
:10133000DBFA08E00A21012000F0D0FC0A2101209C
:10134000FFF7D2FA00BF00BF10BD000038B5054658
:10135000002407E0E00025FA00F0C0B20DF8040018
:10136000601CC4B2042CF5DB0A480BA109680160BB
:101370000B480069074988614FF40010486110224A
:10138000074918310348001DF2F7A8FFFFF712F9CB
:1013900038BD0000C4150020464F54410000000035
:1013A000E059002010B5FEF7E3FE044602F0A0F875
:1013B000012202A1002002F077F810BD5B534D53CB
:1013C0005D4F6B0010B586B0042429480068294998
:1013D0000844B8B1B0F5001F06D0B0F5401F22D0C8
:1013E000B0F5601F41D13CE023480078401CC0B2FA
:1013F00021490870072801DD00200870022000F054
:1014000047F832E01C480078002805DD1A480078CB
:10141000401E1949087002E0072017490870022091
:1014200000F036F821E0154890F8310312490978A8
:10143000884212D010480078104981F831030846DC
:1014400090F831330EA2142101A806F09BF901A8EF
:10145000FBF7BEFE0120FCF7A7FA062003F0D0FD43
:1014600003E0062003F0CCFD00BF00BF06B010BDB6
:10147000B8000020D6FB43FFCB020020AB56002073
:1014800041542B4D49433D322C25640D0A00000088
:1014900030B585B005460424012D44D1424890F86A
:1014A000310342490870F7F7D9FC012140A001F04F
:1014B000A3FA012314229F210020F7F773FDA0B2A5
:1014C00001233FA23821F7F7D9FF374890F831338D
:1014D0003EA20A2102A806F055F904F1500188B293
:1014E000012302AA3821F7F7C9FF04F1500188B29D
:1014F00010231A463821F7F751FE2C48037833A2FF
:101500000621684606F03EF901226946002001F0F6
:10151000CBFF012368229F210020F7F743FD002025
:101520002C4908801EE0022D1CD12048037827A2F8
:101530000A2102A806F026F904F1500188B201231D
:1015400002AA3821F7F79AFF04F1500188B210235C
:101550001A463821F7F722FE012368229F21002036
:10156000F7F720FD1B48008830B901231AA26E212D
:101570000020F7F783FF09E016480088C82805D146
:1015800001231AA26E210020F7F778FF1148008886
:10159000401C80B20F490880B0F5C87F01DB0020F5
:1015A000088005B030BD0000AB560020CB02002003
:1015B000C2F3BFCBB7E7D4F6D2E6C9E8D6C3000082
:1015C000D4F6D2E6D6B53A20202020002530326469
:1015D000000000000C0300205BC9CF5DD1A1D4F155
:1015E000205BCFC25DD1A1D4F12020005B4D5DB165
:1015F000A3B4E620205B455849545DCDCBB3F6003B
:1016000070B5174C002522E0322616A0FBF7E0FD4E
:1016100016E04FF4A061A01CFCF74EFA80B22080C7
:1016200050B115A1A01CFBF717FF48B9012216A164
:10163000002001F039FF70BD0120DFF860C000DF3D
:10164000301EA6F101010EB2E3D1681C05B2052DD2
:10165000DADB012212A1002001F026FF00BFEAE739
:10166000CE09002041542B504F433D3130303030B3
:101670003032300D0A0000002B504F433A313030E9
:1016800030303030300000005B31345D53696D70B4
:101690006C654D6F64655F4F6B00000049930108F6
:1016A0005B31345D53696D706C654D6F64655F547B
:1016B0006F75740010B52148006821490844B8B11D
:1016C000B0F5001F06D0B0F5401F22D0B0F5601F66
:1016D00031D12CE01B480078401CC0B21949087079
:1016E000042801DB00200870022000F02FF822E01F
:1016F00014480078002805DD12480078401E114982
:10170000087002E003200F490870022000F01EF864
:1017100011E00C4800780C4981F8F6020120FCF732
:1017200043F9F6F7EDFC062003F06AFC03E006201F
:1017300003F066FC00BF00BF10BD0000B800002031
:10174000D6FB43FF88020020AB560020F0B589B0DD
:10175000054600260C24012D49D1F7F77FFB012116
:1017600048A001F049F9012314229F210020F7F736
:1017700019FCA0B2012346A23821F7F77FFE4848A2
:101780000068F6F741F907463B4646A2142101A836
:1017900005F0F8FF562101A801F02EF9434890F812
:1017A000F602434951F8203042A20A2106A805F06A
:1017B000E9FF06A8F2F7E0FDC6B204F1500188B2D5
:1017C000012306AA3821F7F759FEF20004F150016F
:1017D00088B210233821F7F7E1FC012368229F210A
:1017E0000020F7F7DFFB00203349088029E0022DB5
:1017F00027D100200690079008902D482F4909789E
:1018000050F821302BA20A2106A805F0BBFF06A83C
:10181000F2F7B2FDC6B204F1500188B2012306AA64
:101820003821F7F72BFEF20004F1500188B21023A3
:101830003821F7F7B3FC012368229F210020F7F736
:10184000B1FB1D48008830B901231DA26E21002084
:10185000F7F714FE09E018480088C82805D10123CD
:101860001CA26E210020F7F709FE13480088401CD7
:1018700080B211490880B0F5C87F01DB00200880E4
:1018800009B0F0BDCDF8C2E7C9E8D6C3000000003A
:1018900020CDF8C2E7D1A1D4F13A202020200000C9
:1018A0008C0300204D4F44453A257300AB56002071
:1018B0008C020020257300000E0300208802002007
:1018C0005BC9CF5DD1A1D4F1205BCFC25DD1A1D4E2
:1018D000F12020005B4D5DB1A3B4E620205B4558AC
:1018E00049545DCDCBB3F600F8B504462046F6F773
:1018F000F7FA06463046F6F70FFB054605B9F8BD80
:101900006B4602221C213046FEF704FBBDF80000A6
:10191000082800D0F3E7044B4FF4806236213046AC
:10192000FEF7F8FA00BFEAE7405E002010B51B485A
:10193000F9F772F804461A48844228D11748C0883B
:10194000184991F82F1388421DD014488079154901
:1019500081F82F0391F82F03FBF7B6FC114890F89C
:101960002F0300280CDD0F4890F8F80240B10D4815
:1019700090F8F802032803DA03200A4981F8F802F4
:101980000120FCF711F8062003F03AFB05E00648B9
:10199000844202D1062003F033FB10BD58470020DB
:1019A0002A04EC00AB5600202A04F40010B586B0DF
:1019B0000446184B0FCBCDE90423CDE902010020EA
:1019C00001902CB3F7F74AFA022113A001F014F8A2
:1019D000012314229F210020F7F7E4FA0120114986
:1019E00091F82F1301AA505401A80F4B002202A90D
:1019F00000900E48F8F73EFF012368229F21002047
:101A0000F7F7D0FA01230AA26E210020F7F736FD7E
:101A100006B010BDBCA10108C4A3CABDC9E8D6C3A5
:101A200000000000AB560020BC02002058470020F8
:101A30005B4F4B5DC7D0BBBB205B455849545DCD68
:101A4000CBB3F60010B51A48F8F7E6FF044619487C
:101A5000844217D11648C08840B91748007808B9A1
:101A6000012000E000201449087020E00120134903
:101A700008700F488079401E11490870042003F057
:101A8000BFFA14E00F48844211D10B4800780128B6
:101A900003D100200849087009E0002006490870B9
:101AA00006490870FBF780FF062003F0A9FA10BD75
:101AB000584700202A04EC00890200208B020020F5
:101AC0008A0200202A04F4002DE9F041A0B0064665
:101AD000002400250027A04614211BA8F2F717FCBC
:101AE00064225B4902A8F2F7F9FB002001905948F3
:101AF0000078A8B958A001F0BBF84FF0320802E016
:101B00000120FCF7FFF9B8F10000A8F1010101F094
:101B1000FF08F5D1012003F073FA20B0BDE8F08191
:101B200038E0002420E0514800EB8500016804EB18
:101B3000440000EBC4024E4850F82200814211D10B
:101B400004EB440202EBC403494A02EB8302911DF9
:101B50006A1C02EB820202AB03EB8200F2F7E2FBAB
:101B6000012705E0601CC4B23A48006FA042DADCED
:101B700000BF3848006FA04209D147B9691C01EB8A
:101B8000810102AA02EB81003AA1F2F7CBFB002708
:101B9000681CC5B2032DC4DB3448C01E8078012800
:101BA00004D136A102A8F2F709FC03E037A102A88C
:101BB000F2F704FC002409E004EB840002A901EB25
:101BC00080001BA941F82400601CC4B2052CF3DB83
:101BD000E6B1F7F743F9022130A000F00DFF012331
:101BE00014229F210020F7F7DDF901A800231A46EF
:101BF0001BA900902D48F8F73DFE012368229F2184
:101C00000020F7F7CFF964202949086028480068C8
:101C1000642806D1012327A26E210020F7F72EFCAD
:101C20000AE023480068B0F5967F05D1012326A27B
:101C30006E210020F7F722FC1D480068401C1C495B
:101C40000860B0F5C87F01DB0020086000BF64E7D2
:101C5000CCA10108402900202020C7EBCFC8B5C780
:101C6000C2BC2E2E2E20202000000000AE560020E8
:101C7000BC2A0020CEB4C6F4D3C30000BFECBDDD47
:101C8000CAB9C4DC3A2020BFAAC6F400BFECBDDD4F
:101C9000CAB9C4DC3A2020B9D8B1D500BFECBDDD4B
:101CA000C8BAD7E9C9E8D6C30000000058470020E9
:101CB0007C0300205BC9CF5DD1A1D4F12020205B43
:101CC000CFC25DD1A1D4F1005B4D5DB1A3B4E620DC
:101CD000205B455849545DCDCBB3F60043185A00FC
:101CE000FF2A00DD7047034B1870034B197000BFCB
:101CF000F8E70000A0000020A100002030B587B068
:101D00000546184890FBF5F084B2ADF81440032066
:101D1000ADF810000020ADF81600ADF812008DF8F7
:101D2000180004A9104801F099FF7020ADF80000D8
:101D3000204604EBD0714910ADF806100120ADF833
:101D400002000220ADF808006946074801F0DEFEF7
:101D50000821054801F026FF0121034801F0BAFEE1
:101D600007B030BD002D3101000C004010B52848EF
:101D7000F9F758FF04462748844241D12448407966
:101D80000D283CD2DFE800F0070B0F13171B1F23B1
:101D9000272B2F333700122003F032F92FE01420C5
:101DA00003F02EF92BE0152003F02AF927E0162086
:101DB00003F026F923E0182003F022F91FE01C208D
:101DC00003F01EF91BE0242003F01AF917E0252088
:101DD00003F016F913E01A2003F012F90FE01E20A9
:101DE00003F00EF90BE0202003F00AF907E01F20B2
:101DF00003F006F903E0232003F002F900BF05E039
:101E00000548844202D1022003F0FAF810BD000018
:101E1000800200202A04EC002A04F4007047704776
:101E200010B586B004242948006829490844B8B18F
:101E3000B0F5001F06D0B0F5401F22D0B0F5601FEE
:101E400041D13CE023480078401CC0B221490870D1
:101E5000FF2801DD00200870022000F047F832E082
:101E60001C480078002805DD1A480078401E1949F2
:101E7000087002E0FF2017490870022000F036F8D1
:101E800021E0154890F8320312490978884212D0AF
:101E900010480078104981F83203084690F8323330
:101EA0000EA2142101A805F06DFC01A8FBF790F922
:101EB0000120FBF779FD062003F0A2F803E00620DD
:101EC00003F09EF800BF00BF06B010BDB8000020B0
:101ED000D6FB43FFCA020020AB56002041542B4CD6
:101EE000564C3D342C25640D0A00000030B585B0F9
:101EF00005460424012D44D1424890F8320342495A
:101F00000870F6F7ABFF012140A000F075FD01233A
:101F100014229F210020F7F745F8A0B201233FA229
:101F20003821F7F7ABFA374890F832333EA20A214E
:101F300002A805F027FC04F1500188B2012302AA8F
:101F40003821F7F79BFA04F1500188B210231822C8
:101F50003821F7F723F92C48037833A20621684685
:101F600005F010FC01226946002001F09DFA0123D2
:101F700068229F210020F7F715F800202C490880DF
:101F80001EE0022D1CD12048037827A20A2102A8B6
:101F900005F0F8FB04F1500188B2012302AA3821B0
:101FA000F7F76CFA04F1500188B210231822382197
:101FB000F7F7F4F8012368229F210020F6F7F2FFDB
:101FC0001B48008830B901231AA26E210020F7F7C0
:101FD00055FA09E016480088C82805D101231AA23D
:101FE0006E210020F7F74AFA11480088401C80B2A1
:101FF0000F490880B0F5C87F01DB0020088005B0DC
:1020000030BD0000AB560020CA020020C0AEB0C8F0
:10201000D4F6D2E6C9E8D6C300000000D4F6D2E672
:10202000D6B53A202020200025303364000000007F
:102030000A0300205BC9CF5DD1A1D4F1205BCFC2E0
:102040005DD1A1D4F12020005B4D5DB1A3B4E620A9
:10205000205B455849545DCDCBB3F60010B500F078
:1020600001F810BD0CB500200190009039480068BF
:1020700040F480303749086000BF3648006800F4FB
:10208000003000900198401C0190009820B94FF654
:10209000FF7101988842F0D12E48006800F40030AA
:1020A00010B10120009001E000200090009801286C
:1020B0004AD12948006840F01000274908600846C6
:1020C000006820F0030008600846006840F0020045
:1020D0000860204840681F494860084640684860DA
:1020E0000846C06A1D4908401A49C8620846C06AC5
:1020F00040F46360C8620846406820F47C10486081
:102100000846406840F4102048600846006840F0E7
:102110008070086000BF0F48006800F00070002861
:10212000F9D00C48406820F003000A49486008468E
:10213000406840F00200486000BF0648406800F078
:102140000C000828F9D104E000200549087000BF00
:10215000FEE70CBD001002400020024000F0FEFF30
:10216000680400202DE9F04104460D4616464FF460
:1021700061606043C5EB051100EB810087193846AB
:10218000FDF740FEBDE8F08110B510480068104929
:10219000884201D1F4F75AFC0E48407801280CD04F
:1021A00000220DA10120F9F7C1FCF4F74FFC002239
:1021B0000D49104601F078F910BD01F0E1FA02F086
:1021C000B9F804F013F900BFF6E70000B8000020EA
:1021D0002A04F400000100204345444543444638A6
:1021E000433245370000000088A2010810B586B0D0
:1021F000394800683949884223D1212002F000FF84
:102200001823A02238210020F6F73CFE0123344A8F
:1022100028210420F7F732F90123324A462104200D
:10222000F7F72CF90123304A6E210020F7F726F941
:10223000F7F708FAC820DFF8B4C000DFFBF72CFD81
:1022400048E0254800682A49884203D1062002F068
:10225000D7FE3FE0204800682649884204D01E4847
:102260000068254988422DD100241B480068214977
:10227000884207D121480088401C20490880601C02
:10228000C4B210E0144800681B4988420BD11B48B7
:102290000088B0F5D97F06DB18480088401E174932
:1022A0000880601CC4B2ACB11448038814A2132186
:1022B00001A805F067FA012301AA44210020F7F7DD
:1022C000DDF807E0044800681149884202D0002088
:1022D0001049087006B010BDB80000202A04EC00B8
:1022E000DAA4010802A5010816A50108499301080E
:1022F0002A04F4002A04DC002A04BC004404002060
:1023000020202020C9FDBCB6B5BD3A56256420006A
:102310002A04F8005004002010B588B00446002CB0
:1023200035D040F2B1101B490880F6F797FD002127
:10233000194800F061FB012314229F210020F6F7C9
:1023400031FE4FF4D87315A21E21684605F01AFA23
:1023500001236A462C210020F7F790F80D480388E6
:1023600013A21E21684605F00DFA01236A46442196
:102370000020F7F783F8012368229F210020F6F759
:1023800011FE01230E4A6E210020F7F777F808B0FE
:1023900010BD0000440400202AA50108202020B51B
:1023A000B1C7B0B0E6B1BE3A205625642020200067
:1023B00020202020C9FDBCB6B5BD3A5625642000BA
:1023C00037A5010810B50D480078022814D10C4833
:1023D00000680C49884206D10320084908700AA009
:1023E000FAF7F6FE07E0064800680A49884202D17B
:1023F000062002F005FE00BF00BF10BD2C04002027
:10240000B80000202A04EC0041542B464F54413DB3
:10241000310D0A002A04F40010B58AB00446002CDD
:1024200030D0F6F71BFD01213BA000F0E5FA0123B7
:1024300014229F210020F6F7B5FD3BA0F5F7E4F844
:10244000012368229F210020F6F7ACFD01233AA268
:102450006E210020F7F712F84FF0FF303B4908607B
:1024600000203B4908703BA0FAF7B2FEDFF8F0C04D
:1024700000DFC8303B49086001233BA26E210020E9
:10248000F6F7FCFF3248007810B1012840D134E063
:10249000DFF8CCC000DF33490968884220D22B48DE
:1024A000006860B901202A49087034A0F5F7ACF83B
:1024B000DFF8ACC000DF96302A4908601CE02348F2
:1024C0000068002818DD214830A10268684605F040
:1024D0006DF96846F5F798F802201D4908700BE081
:1024E00001201B4908702CA0F5F78EF8DFF870C0AA
:1024F00000DF96301B4908600AE0DFF864C000DFA7
:1025000018490968884202D9012002F079FD00BF0C
:1025100000BF0AB010BD0000C9FDBCB6B6D4BDB244
:10252000B0E6B1BE00000000D5FDD4DABCECB2E2EA
:10253000B0E6B1BE000000005B4D5DC9FDBCB62039
:10254000205B455849545DCDCBB3F60028040020EC
:102550002C04002041542B464F54413F0D0A0000EB
:10256000B1990108300400205B4D5DC8B7B6A820C2
:10257000205B455849545DCDCBB3F600C3BBD3D0E7
:10258000BFC9B8FCD0C2B0E6B1BE0000B8FCD0C232
:10259000B5BD562564203F00BCECB2E2B3ACCAB175
:1025A000000000002DE9F04194B080460026162579
:1025B0000E2467239F2229460020F6F7A9FC4E48E7
:1025C0004E49097850F821304DA228210AA805F07B
:1025D000D9F83246761C102000FB025101230AAACA
:1025E0001846F6F74BFF45490978C1EB41124549BA
:1025F00001EB4200F1F7C0FEC7B240480078C0EBE3
:102600004012404800EB420122466846F1F766FE60
:1026100000200DF804006B463BA228210AA805F013
:10262000B1F83246761C102000FB025101230AAAA1
:102630001846F6F723FFA74215DD30480078C0EBB7
:102640004012304800EB420001190AA8F1F7B6FE2B
:102650003046721CD6B2102202FB005101230AAA96
:102660001846F6F70BFF25490978C1EB41122549B9
:1026700001EB420101F11F00F1F77EFEC7B21F48D6
:102680000078C0EB40121F4800EB420000F11F0130
:1026900022466846F1F722FE00200DF804006B4642
:1026A0001BA228210AA805F06DF83046721CD6B28C
:1026B000102202FB005101230AAA1846F6F7DEFE9B
:1026C000A74216DD0D480078C0EB40120D4800EB24
:1026D00042001F3001190AA8F1F770FE3046721C43
:1026E000D6B2102202FB005101230AAA1846F6F7BF
:1026F000C5FE14B0BDE8F081A8020020C802002089
:1027000025733A00A95800204E616D653A25730083
:10271000506173733A25730038B505462E24B5F51C
:10272000A57F28DADFF86CC100DF5B4909688842C1
:1027300000D238BDDFF85CC100DF50305649086078
:102740005648007850B904F1290188B254A20321F7
:10275000F6F720FE01205149087098E000204F490B
:10276000087004F144018AB21B3988B20F23032197
:10277000F6F7CEFB8BE0B5F5B17F11DC04F1290152
:1027800088B247A20321F6F705FE0120009004F16C
:102790003E0082B204230C210520F6F746FC76E0C9
:1027A000B5F5BB7F1BDC04F1290188B23CA20321F3
:1027B000F6F7F0FD0120009004F1390082B2042305
:1027C0000C210520F6F731FC0120009004F13E00B9
:1027D00082B204230C210520F6F727FC57E0B5F55B
:1027E000C87F25DA04F1290188B22DA20321F6F76A
:1027F000D1FD0120009004F1340082B204230C21A9
:102800000520F6F712FC0120009004F1390082B295
:1028100004230C210520F6F708FC0120009004F1A8
:102820003E0082B204230C210520F6F7FEFB2EE0C9
:1028300004F1290188B21AA20321F6F7ABFD0120A9
:10284000009004F12F0082B204230C210520F6F73A
:10285000ECFB0120009004F1340082B204230C212F
:102860000520F6F7E2FB0120009004F1390082B266
:1028700004230C210520F6F7D8FB0120009004F179
:102880003E0082B204230C210520F6F7CEFB00BFE8
:102890004FE70000B1990108F4010020F801002081
:1028A00056424154312E626D700000002DE9F04116
:1028B0001E25222664274FF03B0880200E49086120
:1028C00041000E48F4F7BBFFF6F7C8FA0CA200214E
:1028D0000846F6F75FFD002408E0642094FBF0F161
:1028E00000FB114008B9F6F7ADFE641C07488442AE
:1028F000F3DBBDE8F081000000100140000C014056
:1029000077656C636F6D652E626D7000801A0600CE
:102910002DE9F04104460D4616463046F5F7A0FE77
:10292000074605F1140083B2E019083082B2294647
:102930002046F6F7EDFAAA1C91B2221D90B20123AF
:102940003246F6F79BFD05F1140083B2E01908301A
:1029500082B229462046F6F721FCBDE8F08100004E
:1029600030B589B004460D461F480078322190FBEF
:10297000F1F201FB120058B324221C491C48F1F764
:1029800026FD48B9282219491948F1F720FD18B940
:10299000184890F8B80270B122239F22122100201B
:1029A000F6F7B6FA282211491148F1F797FC0021F1
:1029B000104880F8B81224220D49684600F072FFD2
:1029C00004F1300188B20123084A2946F6F756FD82
:1029D00005480078401CC0B203490870322801DB6A
:1029E0000020087009B030BD65010020B429002026
:1029F000BC480020403900202DE9F04104460D4636
:102A00002046F5F72DFE0646C6F1A00707EBD77165
:102A1000C1F34F00012322462946F6F72FFDBDE8FA
:102A2000F081000010B51423322200212D20F6F78A
:102A30006FFA1C48007800F0010030B914234B22D3
:102A400000212D20F6F764FA2AE016480078C0F33A
:102A5000400080B913480078C0F3001028B912A2D2
:102A600000212D20F6F796FC1AE012A200212D205D
:102A7000F6F790FC14E00B480078C0F3001028B97A
:102A800009A200212D20F6F785FC04E009A200210F
:102A90002D20F6F77FFC0AA202213520F6F77AFCFA
:102AA00010BD0000041F0020475053312E626D708E
:102AB00000000000475053412E626D70000000007E
:102AC000475053322E626D7000000000F0B58DB09B
:102AD00006460D46144638A207CA01AB07C30027B5
:102AE00038480078401CC0B236490870062800DA21
:102AF00014B100203349087032480078032835DAD1
:102B0000314890F8B70260B930493148F1F73BFCE1
:102B100000B994B124222E492C48F1F7DFFB01279C
:102B20000BE02A4901A8F1F72EFC00B92CB10922CB
:102B300001A92648F1F7D2FB0127DFB305F1100008
:102B400083B29F2229463046F6F7E2F924221F4934
:102B500004A800F0A7FE012304AA29463046F6F790
:102B60008DFC0121184880F8B81223E01749184855
:102B70002D38F1F708FC00B9E4B1242214492D39AD
:102B80001248F1F7ABFB05F1100083B29F222946F2
:102B90003046F6F7BDF924220C4904A800F082FE65
:102BA000012304AA29463046F6F768FC01210648AD
:102BB00080F8B8120DB0F0BDB5A5BAF4C4A3CABD73
:102BC00000000000640100204039002098480020E7
:102BD0008229002030B587B002A8FCF775FF642277
:102BE0000298B0FBF2F1B1F1807F00D31DE021F03B
:102BF0007F40401E4FF0E022506150170F22002806
:102C000007DA13071D0E0E4B00F00F04241F1D558D
:102C100003E013071C0E0B4B1C5400BF00204FF0A9
:102C2000E02290610720106100BF0398009006A089
:102C3000DDE90423029904F095FD07B030BD0000E2
:102C400018ED00E000E400E0535953434C4B3D25A0
:102C5000642C50434C4B313D25642C50434C4B323B
:102C60003D25642C48434C4B3D25640D0A00000073
:102C7000F0B593B00546402404F11403A4F1140008
:102C800081B29F220020F6F743F9012004F11203DC
:102C90000090A4F1120081B29D220220F6F799F96A
:102CA0001222294601A800F0FDFD01A8F5F7D8FC85
:102CB00086B2C6F1A00000EBD071C1F34F07A4F1BA
:102CC000080081B2012301AA3846F6F7D7FB13B0FA
:102CD000F0BD000070B50446002534B118480078F6
:102CE00000F00100B0B1012514E01548007800F0B3
:102CF000010014490978884200D170BD104800785D
:102D000000F001000F4908700D48007800F0010044
:102D100000B10125012D02D0022D0DD105E00AA23E
:102D200003213C20F6F736FB07E0012309A203212B
:102D30003C20F6F7A3FB00E000BF00BF00BFDCE7CC
:102D400054520020750200204D61696C312E626D75
:102D5000700000002020000038B50446424840784A
:102D6000012805D141A202210020F6F713FB04E05F
:102D700042A202210020F6F70DFB012C01DB632C9F
:102D800006D10E23152204210720F6F7C1F86AE0C8
:102D9000082C0EDA0120022307220E2100900C20BD
:102DA000F6F743F90E23152204210B20F6F7B0F8AD
:102DB00059E0102C16DA0120022307220E21009080
:102DC0000C20F6F732F9012002230B220E2100908D
:102DD0000920F6F72AF90E23152204210F20F6F711
:102DE00097F840E0162C1EDA0120022307220E215C
:102DF00000900C20F6F719F9012002230B220E2176
:102E000000900920F6F711F9012002230F220E216C
:102E100000900720F6F709F90E231522042113204C
:102E2000F6F776F81FE00120022307220E2100901A
:102E30000C20F6F7FAF8012002230B220E21009055
:102E40000920F6F7F2F8012002230F220E2100904C
:102E50000720F6F7EAF80120022313220E21009042
:102E60000420F6F7E2F838BD0001002053696E67D0
:102E70006C654F4B2E626D700000000053696E67E9
:102E80006C652E626D70000070B50546002D39D05E
:102E90000F239F2200210846F6F73AF85A480068A7
:102EA0005A49086058480068FFF756FF58480068BC
:102EB00058490860584890F8B70240B2574908701E
:102EC0000846007828B956A26B217920FFF720FD2B
:102ED00004E055A26B217920FFF71AFDFFF7A2FD50
:102EE0004B480068FFF718FC0120FFF7F3FE00F0E5
:102EF000ADF84F4800684F4908600846006800F088
:102F00003FF970BD4B48006849490968884207D0BD
:102F100047480068474908600846006800F030F9F3
:102F20003A48006838490968884205D142484078E3
:102F30004249097888420BD03F4840783F490870A1
:102F400031480068314908602F480068FFF704FFE6
:102F50003B480078642808DA4FF4B4702C490860C4
:102F600037480078401C364908702A4800682849CC
:102F70000968884204D126480068B0F5A57F07DAC1
:102F8000234800682349086021480068FFF7C4FB14
:102F90000020FFF79FFE2B480078C0F3400029492E
:102FA000097801F0010140EA012026490978C1F3BE
:102FB000001140EA810424480088A04203D022483E
:102FC0000480FFF72FFD00F041F8134890F8B70296
:102FD000124991F90010884213D00F4890F8B702B7
:102FE00040B20E4908700846007828B90CA26B213F
:102FF0007920FFF78DFC04E00BA26B217920FFF70D
:1030000087FC00BF7DE700000801002004020020CB
:103010004000002008020020403900201402002057
:10302000CFFBCFA200000000B9D2B6CF0000000055
:103030009003002010020020000100200E0200205A
:1030400000020020041F00200C020020F0B589B00F
:103050004148407808B909B0F0BDFCF783FE04464A
:103060004FF4616094FBF0F0182190FBF1F201FB4A
:1030700012064FF4616094FBF0F100FB11403C211B
:1030800090FBF1F7002535480078002841D04FF437
:10309000616094FBF0F100FB11403C2190FBF1F2E8
:1030A00001FB12052E480068A8423DD02D4800784B
:1030B000401C2C490870084600783C2815DB00208D
:1030C000087029480078401C274908702248007879
:1030D00058B126480078401CC0B224490870052821
:1030E00003DB002008701D4908701F4800783C2849
:1030F00007DB00201C4908701D480078401C1C4953
:1031000008701B48007818280EDB0020184908704A
:103110000AE03C2094FBF0F100FB114514490E70CD
:1031200011490F700F490D700D480068A84211D069
:103130000B4805600C48007800900D4803780DA2FC
:103140001E2101A804F01EFB012301AA0021762004
:10315000F6F794F900BF7EE7402900200D0100201A
:10316000FC0100200200002001000020F9010020E5
:1031700003000020253032643A253032640000001C
:1031800010B50446022C01D0032C05D110A2022157
:103190001820F6F7FFF819E0042C03D0052C01D015
:1031A000082C05D10CA202211820F6F7F3F80DE047
:1031B000092C05D10AA202211820F6F7EBF805E048
:1031C00014232D2202211820F5F7A2FE10BD0000C5
:1031D00032672E626D70000033672E626D700000E2
:1031E00034672E626D7000002DE9F04788B080468C
:1031F00089464FF0000AB8F1000F03D000206A4959
:10320000A1F8680069A0FFF733FD0120DFF8A8C12D
:1032100000DF654869A21E21C36B684604F0B2FA5C
:103220006846F9F7D5FF00226946104600F03CF9E0
:103230004FF47A7600205C4981F86C00888112E0B6
:10324000701E86B20120FAF75DFE574890F86C00B8
:1032500000B10AE0C82096FBF0F100FB116010B944
:103260006846F9F7B5FF002EEAD100BF4E488089C5
:10327000002804DC00204C4981F86B008BE04A48B0
:103280008089052190FBF1F201FB120018B905209D
:103290004F49087008E044488089052190FBF1F20D
:1032A00001FB12004A490870B9F1010F0DD13E48E7
:1032B000B0F868508089401B052801DB05242AE00E
:1032C0003948007B401BC4B225E03748B0F868504D
:1032D000B0F86800052803DA00253348047B1AE0BB
:1032E00031488089401B3A490978884212DC2E48CF
:1032F0008089052190FBF1F201FB120008B9052439
:1033000009E029488089052190FBF1F201FB1200B8
:10331000C4B200E00524052C00DB0524002022496E
:1033200081F86B002F462BE000201F4981F86A00CE
:103330003B4628A21E21684604F024FA6846F9F7A5
:1033400047FF00226946104600F0AEF8C82613E099
:103350000120FAF7D7FD144890F86A0038B11248F6
:1033600090F86B00401C104981F86B0005E0701E5E
:1033700080B2061E00D100E0EAE700BF781C87B2E9
:103380002819B842D0DCB8F1000F03D0002006495C
:10339000A1F8680000BF60239F2228210020F5F7D4
:1033A000B7FD08B0BDE8F08740290020C7EBC9D4BD
:1033B000BAF22E2E2E0000004993010841542B50E2
:1033C0004F433D304530303030253038780D0A00DD
:1033D0000A00002041542B504F433D3130303030F3
:1033E000303231253034780D0A000000012223A14B
:1033F000002000F059F84FF40050234948610420A0
:10340000224908608001224908601F494861012063
:1034100008618020486102201D49091F08600120C1
:10342000091D086040021849086140F6B830F6F7F7
:10343000E5F8002144F21C00FCF72CFB00214FF4BE
:10344000C020FCF717FB00211248F1F7C1FB002157
:103450000120FCF7FFFA10480068DFF840C000DFE9
:103460000F480068DFF834C000DF06E04FF47A70E0
:10347000DFF830C000DFF6F7E5F8F7E7536C656575
:1034800070696E67000000000010014014140140D4
:10349000140C01400024014028010020DD9A01089D
:1034A00024010020499301082DE9F84380460C4689
:1034B00015460DA0006800900C48007808B1BDE8E2
:1034C000F8832046F0F758FF06463146204603F0C1
:1034D000BBF93DB16846F0F74FFF074639466846ED
:1034E00003F0B2F900BFEAE70D0A00000C0000206B
:1034F0002DE9FF410546022D01DDBDE8FF81002DCC
:103500005FD0012D2FD100202F49488088806F4641
:103510000846D0F80660E8464FF47A7421E010229D
:103520003146384606F0BAFB9DF80000012812D15A
:1035300025484088401C244948809DF80100012806
:1035400009D108468088401C88800846007820F011
:103550000100401C0870601E84B204B902E0D8F873
:103560000C60DCE72DE0022D2BD16F461648D0F819
:103570000660E8464FF47A7421E01022314638465E
:1035800006F08CFB9DF8000018B90F48C0F80A60DF
:1035900016E0601E84B28CB90B48007820F004005D
:1035A000001D09490870012208A10020FFF77CFFD7
:1035B00000F0A0F808A0F9F70BFE01E0029EDCE79E
:1035C00000BF00BF99E70000545200205B534D53E9
:1035D0005D46756C6C00000041542B4C53485454AC
:1035E000533D312C22434646424346413244324405
:1035F0003143324641220D0A0000000010B5174841
:1036000090F8BA02012826D1DFF854C000DF15492E
:103610000968884200D210BDDFF844C000DF0F30D7
:103620001049086010480078401CC0B20E4908706C
:10363000022807DC00F05EF80A214FF4FA70FDF76B
:1036400009F908E00021054880F8BA12002006496F
:1036500008700449086000BFDDE700004039002021
:10366000B199010848010020450100202DE9F041F1
:10367000174F0326174890F8340008B9BDE8F081C9
:1036800014483430F0F778FE0446E11704EB51712A
:10369000C910A4EBC101C1F108010C44E11704EB0E
:1036A0005171CD10642045430A4890F8840008B950
:1036B000032605E0074890F88400012800D1012680
:1036C0000022044934313046F8F730FA00BFD5E71C
:1036D000CE090020AB56002010B5044614B100F00E
:1036E00009F803E04FF480700149486110BD000003
:1036F0000010014030B5042500240FE04FF4807025
:103700000B4908610520FCF72DFF4FF48070084934
:1037100048610520FCF726FF601CC4B2AC42EDDB1B
:103720004FF48070024908610520FCF71BFF30BD93
:103730000010014008B54FF48070ADF80000102073
:103740008DF8030003208DF8020069460348F3F763
:1037500097FF0020FFF7C0FF08BD000000100140E8
:1037600010B50648007800F0010000B910BD00F067
:1037700093FB00200149087000BFF7E738010020E3
:1037800010B51B48007800B910BD1948007900B980
:10379000FAE700201649087108464079122806D039
:1037A00025280AD047280ED058281ED114E01048EA
:1037B000807908B9F5F7FEFF17E000220D491046A1
:1037C000FFF772FE11E000220B491046FFF76CFE76
:1037D0000220F5F79DFE08E0002208491046FFF799
:1037E00063FE0320F5F794FE00BF00BF00BFCBE7E8
:1037F000E0590020A4A2010881A40108C1A2010887
:10380000F8B506460D463046F0F7B6FD00F001006B
:1038100000B1F8BD40E0002429E016F8010B0DF8D6
:1038200004001DF8040030280ADB1DF804003928C4
:1038300006DC1DF804003038C0B20DF8040014E0B6
:103840001DF8040041280ADB1DF80400462806DCA8
:103850001DF804003738C0B20DF8040005E01DF86B
:1038600004005738C0B20DF80400601CC4B2022C2A
:10387000D3DB9DF800000007000E8DF800009DF8D6
:10388000000000F0F0008DF800009DF800009DF8A9
:103890000110084305F8010B30780028BBD12870CF
:1038A00000BFB6E72DE9F047064688461446404675
:1038B000F0F762FD81460021601E3154621E4146D0
:1038C0003046F0F74DFD601E48451CDC052C1ADD26
:1038D0002E21A01E3154E01E31543546002707E04A
:1038E00028789F2802DDAD1CBF1C01E06D1C7F1CE9
:1038F000201FB842F4DCB84205D128789F2802DDA9
:103900002E21201F3154BDE8F0872DE9FC470446E5
:103910008946154600272846F0F72EFD8046B8F167
:10392000040F02DA0020BDE8FC8749462046F0F784
:10393000EEFC2AE0A8788DF80000E8788DF8010008
:1039400028788DF8020068788DF8030000208DF843
:103950000400102200216846F0F748FD1FFA80FAA3
:10396000504603F0A5FA0646301220B904F8016B60
:10397000781C87B206E0301204F8010B04F8016BE2
:10398000B81C87B22D1DA8F10408781C484502DA3E
:10399000B8F1000FCEDC002004F8010B3846C2E776
:1039A00010B50D480078B0B10C480078401CC0B28A
:1039B0000A49087005280EDB09480078012803D160
:1039C00008A26B21FEF7A4FF002003490870012222
:1039D00006A1FFF769FD10BD6C0000206D000020FE
:1039E00054010020B2CBB5A50000000051756974E8
:1039F00047726F757053656C0000000010B506A229
:103A00006B210120FEF784FF01200549087000208A
:103A10000449087010BD0000C8B7B6A80000000037
:103A20006C0000206D00002010B5E6B00C4CA4F135
:103A3000080090F8980102280ED140F28D1221461C
:103A400001A8F0F74BFCA4F10800B0F8961101AA08
:103A50002046FFF75AFF00E000BF00BF66B010BD70
:103A6000723D002010B51648006840F0010014496E
:103A700008600846406813490840114948600846F4
:103A80000068114908400E4908600846006820F4A3
:103A9000802008600846406820F4FE004860084620
:103AA000006820F0A05008604FF47F00886000207C
:103AB000C862FEF7D3FA05480549086010BD00004A
:103AC000001002400000FFF0FFFFF6FE004000087B
:103AD00008ED00E021B1028842F00102028004E01A
:103AE00002884FF6FE731A400280704731B1B0F879
:103AF000442042F40042A0F8442005E0B0F84420FD
:103B0000C2F30E02A0F844207047000070B50024F4
:103B100000220023058C4FF6FE7635400584028C8A
:103B20008388048B4FF68F752C40B51E2C400D8872
:103B30002C43751E2A400D892A434D882A43144D73
:103B4000A8420BD0134DA84208D0134DA84205D06F
:103B5000124DA84202D0124DA84213D14FF6F7756C
:103B60002A404D892A434FF6FB752A408D882A4307
:103B70004FF6FF652B404FF6FF552B408D892B43A9
:103B8000CD892B4383800483CD888586028470BDD4
:103B9000002C01400034014000400140004401403D
:103BA000004801400A460021018B4FF6F773194087
:103BB000114301837047000070B5002400220023E8
:103BC000058C4FF6EF7635400584028C8388048B94
:103BD00048F6FF752C404FF6FF452C400D884FF6F8
:103BE000FF7606EA05252C434FF6DF752A400D893E
:103BF00006EA05152A434D8806EA05152A43154DA0
:103C0000A84202D0144DA8421DD14FF67F752A401C
:103C10004D894FF6FF7606EA05152A434FF6BF7524
:103C20002A408D8806EA05152A434FF6FF352B40BA
:103C30004FF2FF752B408D8906EA85052B43CD8910
:103C400006EA85052B4383800483CD88058702849B
:103C500070BD0000002C01400034014000220288A9
:103C60001D4B98420ED01D4B98420BD0B0F1804FA7
:103C700008D01B4B984205D01A4B984202D01A4BE1
:103C8000984204D14FF68F731A404B881A43174B52
:103C9000984207D0164B984204D04FF6FF431A4083
:103CA000CB881A4302808B8883850B8803850A4B57
:103CB00098420BD0094B984208D00E4B984205D041
:103CC0000D4B984202D00D4B984201D10B7A0386DE
:103CD0000123838270470000002C01400034014022
:103CE0000004004000080040000C004000100040AC
:103CF00000140040004001400044014000480140E1
:103D000010B502460B465078012103E04C1C145DAF
:103D10006040491C5C1E8C42F8DC10BD10B586B0BA
:103D2000104C1C212046F0F7F2FA0F4C7821204667
:103D3000F0F7EDFA0D4890F8F8020D4931F810301F
:103D40000CA2142101A803F01DFD012201A90020ED
:103D5000FFF7AAFB2046007820F0100021460870EB
:103D600006B010BD34540020041F0020AB560020C4
:103D700094A1010847707374696D653D2564000066
:103D80002DE9F04F89B006468B4691469A46DDF8FC
:103D9000488035460020079000240120069000202E
:103DA000059008F1060080B2019008F10C0080B285
:103DB00000905B4634A20C2102A803F0E3FC7E22B3
:103DC0002046641C2A544FEA19222046641C2A54B7
:103DD0002046641C05F8009000202D490871084613
:103DE000C0F8088002792046641C2A540846027AEA
:103DF0002046641C2A5400222046641C2A540027B2
:103E00000BE002A8C15D02AA781C105C61F31F10D0
:103E1000C2B22046641C2A54BF1C0A2FF1DB1D4885
:103E20000088020A2046641C2A541A480278204658
:103E3000641C2A5417480088401C16490880BAF1AF
:103E4000000F09D0002705E01AF807202046641C5F
:103E50002A547F1C4745F7DB21462846FFF750FFD1
:103E600008902146641C08986854611E681C04F080
:103E7000C3FA0446641C7E222046641C2A54204651
:103E800009B0BDE8F08F000025303130750000002A
:103E9000805400200C04002010B59EB0012215A112
:103EA0000020FFF701FB1648B0F80300ADF80C0046
:103EB0001348B0F8010002909DF809008DF80E003B
:103EC0009DF808008DF80F000D4840798DF810001E
:103ED000052000900B48D0F81D1003AB012205A867
:103EE000FFF74EFF0446A2B205A90120F7F71CF91F
:103EF0001EB010BD4465766963652041434B0000E8
:103F000038010020C415002010B59AB001220CA180
:103F10000020FFF7C9FA00F021F81C2000900D489E
:103F2000D0F81D100C4B4FF4007201A8FFF728FFCA
:103F300084B2224601A90120F7F7F6F81AB010BDA5
:103F4000545347707354696D696E6753656E64505E
:103F50006F730000C41500203454002010B546488B
:103F6000C07A464988754448017B4448C175424837
:103F7000417B424801764048817B404841763E483B
:103F8000C17B3E4881763C48017C3C48C17600209C
:103F90003A490860486038480078C0F3400020B3D0
:103FA0000846406840F0807048600846406840F02D
:103FB00000704860304890F86C00532804D10846DF
:103FC000406840F0806048602B4890F86D005728AA
:103FD00005D12A48406840F00060284948602748D9
:103FE000406840F08050254948602348808FC0F3E6
:103FF0000720214991F83C1040EA01201F4908821E
:104000001D48808BC0F307201B49097F40EA01202F
:104010001A4948821848008C88820120F3F7ECFD89
:104020001548806E000E154908721348806E010C09
:10403000124841721048B0F86800010A0F488172B6
:104040000D4890F868100D48C1720B48406E000E84
:104050000A4908730848406E010C08484173064835
:10406000B0F86400010A05488173034890F86410B1
:104070000248C17310BD0000041F0020345400200A
:1040800010B52E2202490348F0F728F910BD0000B0
:10409000AB590020505400202DE9F04792B006465D
:1040A0000F2700201090119014210BA8F0F72FF982
:1040B000002009900A900690079008904FF001099F
:1040C0004FF0010A18216846F0F721F938A110A82D
:1040D000F0F774F937A339A214210BA803F052FBAF
:1040E00004F048FA804600240FE018F81400F0218C
:1040F00001EA00106100491C18F8011001F00F01DD
:10410000084306A90855601CC4B20A2CEDDB002444
:104110002146641C7754C7F307222146641C72545D
:10412000002507E010A8425D2146601CC4B272540D
:10413000681CC5B2052DF5DB002507E00BA8425D24
:104140002046611CCCB23254681CC5B2142DF5DB7C
:10415000002507E009A8425D2146601CC4B27254E4
:10416000681CC5B2072DF5DB002507E006A8425DF7
:104170002046611CCCB23254681CC5B20A2DF5DB56
:104180002046611CCCB206F8009000222046611C3B
:10419000CCB232542046611CCCB206F800A02046B6
:1041A000611CCCB23254204612B0BDE8F08700004A
:1041B0004847530048533139314C00002573000003
:1041C00070B59AB02648D0F81D50002025490880C7
:1041D0004880002404E000212248001D0155641C91
:1041E000052CF8DB002404E000211E4809300155AD
:1041F000641C142CF8DB280E1A494877290C19483E
:104200008177290AC17780F82050002405E0002238
:1042100014481D30211D4254641C032CF7DB002080
:10422000104981F82400002404E000210D482530C5
:104230000155641C082CF8DB2E2000900848D0F8AB
:104240001D10084B4FF4807201A8FFF799FD86B24C
:10425000324601A90120F6F767FF1AB070BD0000D1
:10426000C41500205054002010B59AB001220BA1B3
:104270000020FFF719F9002000900B48D0F81D101E
:10428000002340F6027201A8FFF77AFD84B22246AD
:1042900001A90120F6F748FF1AB010BD526571520E
:1042A00065616C54696D6500C415002010B59AB045
:1042B00001220BA10020FFF7F7F8002000900B4827
:1042C000D0F81D100023022201A8FFF759FD84B287
:1042D000224601A90120F6F727FF1AB010BD000001
:1042E00048656172745469636B000000C415002056
:1042F00010B59AB001220BA10020FFF7D5F80020DD
:1043000000900B48D0F81D10002340F6017201A860
:10431000FFF736FD84B2224601A90120F6F704FF1B
:104320001AB010BD534F532053656E640000000057
:10433000C415002000B58DB076484088401C80B27E
:1043400074494880B0F5FA7F7EDD00204880084639
:104350004079472848D004DC122807D025281FD1EF
:104360001FE058285CD0C228F9D16EE069488079F6
:1043700098B96848407A401C664948720846407AB5
:10438000032803DA1220F9F7DFFC09E00120614974
:10439000C872C220F9F7D8FC02E01220F9F7D4FC69
:1043A00088E05C48807918B91220F9F7CDFC1AE052
:1043B0005848807A401C574988720846807A1428E9
:1043C0000BDA012254A10020FFF76EF85149486929
:1043D0004FF48061F5F7C8F905E002204D49C87235
:1043E000C220F9F7B1FC65E00022022149481830EB
:1043F000F5F74CF910B1012810D103E05820F9F776
:10440000A3FC0BE004204349C87200224549104632
:10441000FFF74AF8C220F9F797FC00BF00BF49E058
:104420004148FCF793FF002240491046FFF73CF853
:104430003F480068DFF8FCC000DF3F480068DFF855
:10444000F4C000DF00BFFEE735E001233B4A28212E
:104450000420F5F713F82F48C07A012806D0022867
:104460000BD0032810D004281CD114E00123344AB7
:1044700046210420F5F702F814E00123314A4621D1
:104480000420F4F7FBFF0DE001232F4A462104200E
:10449000F4F7F4FF06E001232C4A46210420F4F748
:1044A000EDFF00BF00BFC820DFF8A4C000DFF2F7B7
:1044B000CDFA00BF00BF27480078401C254908708E
:1044C000084601780078401C224A1070FE291EDB45
:1044D00000201146087020480078401C1E490870D2
:1044E00008460078032809DA03231CA23221684613
:1044F00003F048F96846F8F76BFE08E0002016491B
:1045000008700448007810B90120F2F7DDFF0DB003
:1045100000BD0000E05900205265712044617461C3
:1045200000000000D2A20108A9CBED9F2CA3010836
:1045300028010020DD9A0108240100204BA5010874
:1045400060A5010875A501088AA501089FA50108B5
:10455000499301084D0400204E04002041542B547F
:1045600043505354415455533D25640D0A000000F7
:10457000F0B505460C4628686968AA68EB6801EA48
:10458000020623EA01073E4327683E44FE4F3E44AD
:104590003044C60146EA5060084400EA010622EAB7
:1045A00000073E4367683E44F84F3E4433441E03D1
:1045B00046EA1353034403EA000621EA03073E4395
:1045C000A7683E44F24F3E443244560446EAD23293
:1045D0001A4402EA030620EA02073E43E7683E4423
:1045E000EC4F3E4431448E0546EA9121114401EAE4
:1045F000020623EA01073E4327693E44E64F3E4454
:104600003044C60146EA5060084400EA010622EA46
:1046100000073E4367693E44E04F3E4433441E0377
:1046200046EA1353034403EA000621EA03073E4324
:10463000A7693E44DA4F3E443244560446EAD23239
:104640001A4402EA030620EA02073E43E7693E44B1
:10465000D44F3E4431448E0546EA9121114401EA8B
:10466000020623EA01073E43276A3E44CE4F3E44FA
:104670003044C60146EA5060084400EA010622EAD6
:1046800000073E43676A3E44C84F3E4433441E031E
:1046900046EA1353034403EA000621EA03073E43B4
:1046A000A76A3E44A6F524464F3E3244560446EAE5
:1046B000D2321A4402EA030620EA02073E43E76ABE
:1046C0003E44BB4F3E4431448E0546EA912111449D
:1046D00001EA020623EA01073E43276B3E44B54F39
:1046E0003E443044C60146EA5060084400EA0106F0
:1046F00022EA00073E43676B3E44AF4F3E443344DB
:104700001E0346EA1353034403EA000621EA0307A3
:104710003E43A76B3E44A94F3E443244560446EA0A
:10472000D2321A4402EA030620EA02073E43E76B4C
:104730003E44A34F3E4431448E0546EA9121114444
:1047400001EA030622EA03073E4367683E449D4FA1
:104750003E443044460146EAD060084400EA02067E
:1047600021EA02073E43A7693E44974F3E44334443
:104770005E0246EAD353034403EA010620EA010736
:104780003E43E76A3E44914F3E443244960346EA34
:1047900092421A4402EA000623EA00073E432768D1
:1047A0003E448B4F3E4431440E0546EA11311144DC
:1047B00001EA030622EA03073E4367693E44854F48
:1047C0003E443044460146EAD060084400EA02060E
:1047D00021EA02073E43A76A3E447F4F3E443344EA
:1047E0005E0246EAD353034403EA010620EA0107C6
:1047F0003E43E76B3E44794F3E443244960346EADB
:1048000092421A4402EA000623EA00073E4327695F
:104810003E44734F3E4431440E0546EA1131114483
:1048200001EA030622EA03073E43676A3E446D4FEE
:104830003E443044460146EAD060084400EA02069D
:1048400021EA02073E43A76B3E44674F3E44334490
:104850005E0246EAD353034403EA010620EA010755
:104860003E43E7683E44614F3E443244960346EA85
:1048700092421A4402EA000623EA00073E43276AEE
:104880003E445B4F3E4431440E0546EA113111442B
:1048900001EA030622EA03073E43676B3E44554F95
:1048A0003E443044460146EAD060084400EA02062D
:1048B00021EA02073E43A7683E444F4F3E4433443B
:1048C0005E0246EAD353034403EA010620EA0107E5
:1048D0003E43E7693E44494F3E443244960346EA2C
:1048E00092421A4402EA000623EA00073E43276B7D
:1048F0003E44434F3E4431440E0546EA11311144D3
:1049000081EA02065E4067693E443E4F3E443044C1
:10491000060146EA1070084480EA01065640276AFC
:104920003E44394F3E443344DE0246EA5353034487
:1049300083EA00064E40E76A3E44344F3E44324428
:10494000160446EA12421A4482EA03064640A76B5E
:104950003E442F4F3E443144CE0546EA5121114496
:1049600081EA02065E4067683E442A4F3E44304476
:10497000060146EA1070084480EA0106564027699D
:104980003E44254F3E4449E078A46AD756B7C7E86D
:10499000DB702024EECEBDC1AF0F7CF52AC6874761
:1049A000134630A8019546FDD8988069AFF7448B2F
:1049B000BED75C892211906B937198FD8E4379A6C6
:1049C0002108B44962251EF640B340C0515A5E2604
:1049D000AAC7B6E95D102FD65314440281E6A1D8C8
:1049E000C8FBD3E7E6CDE121D60737C3870DD5F461
:1049F000ED145A4505E9E3A9F8A3EFFCD9026F6766
:104A00008A4C2A8D4239FAFF81F6718722619D6DA9
:104A10000C38E5FD44EABEA4A9CFDE4B3344DE02E8
:104A200046EA5353034483EA00064E40E7693E4496
:104A30009F4F3E443244160446EA12421A4482EA28
:104A400003064640A76A3E449A4F3E443144CE0591
:104A500046EA5121114481EA02065E40676B3E44FA
:104A6000954F3E443044060146EA1070084480EAFF
:104A70000106564027683E44904F3E443344DE02D0
:104A800046EA5353034483EA00064E40E7683E4437
:104A90008B4F3E443244160446EA12421A4482EADC
:104AA00003064640A7693E44864F3E443144CE0546
:104AB00046EA5121114481EA02065E40676A3E449B
:104AC000814F3E443044060146EA1070084480EAB3
:104AD00001065640276B3E447C4F3E443344DE0281
:104AE00046EA5353034483EA00064E40E76B3E44D4
:104AF000774F3E443244160446EA12421A4482EA90
:104B000003064640A7683E44724F3E443144CE05FA
:104B100046EA5121114461EA0306564027683E44A3
:104B20006D4F3E443044860146EA9060084460EA96
:104B300002064E40E7693E44684F3E4433449E02BD
:104B400046EA9353034463EA01064640A76B3E449A
:104B5000634F3E443244D60346EA52421A4462EA64
:104B600000065E4067693E445E4F3E4431444E0558
:104B700046EAD121114461EA03065640276B3E44C0
:104B8000594F3E443044860146EA9060084460EA4A
:104B900002064E40E7683E44544F3E4433449E0272
:104BA00046EA9353034463EA01064640A76A3E443B
:104BB0004F4F3E443244D60346EA52421A4462EA18
:104BC00000065E4067683E444A4F3E4431444E050D
:104BD00046EAD121114461EA03065640276A3E4461
:104BE000454F3E443044860146EA9060084460EAFE
:104BF00002064E40E76B3E44404F3E4433449E0223
:104C000046EA9353034463EA01064640A7693E44DB
:104C10003B4F3E443244D60346EA52421A4462EACB
:104C200000065E40676B3E44364F3E4431444E05BD
:104C300046EAD121114461EA0306564027693E4401
:104C4000314F3E443044860146EA9060084460EAB1
:104C500002064E40E76A3E442C4F3E4433449E02D7
:104C600046EA9353034463EA01064640A7683E447C
:104C7000274F3E443244D60346EA52421A4462EA7F
:104C800000065E40676A3E44224F3E4431444E0572
:104C900046EAD12111442E6806442E606E680E4407
:104CA0006E60AE681644AE60EE681E44EE60F0BD05
:104CB000604BBBF670BCBFBEC67E9B28FA27A1EA3C
:104CC0008530EFD4051D880439D0D4D9E599DBE6C9
:104CD000F87CA21F6556ACC4442229F497FF2A43EE
:104CE000A72394AB39A093FCC3595B6592CC0C8F7E
:104CF0007DF4EFFFD15D84854F7EA86FE0E62CFE4A
:104D0000144301A3A111084E827E53F735F23ABD38
:104D1000BBD2D72A91D386EB38B5002440F2255177
:104D20003A4801F035FC00285CD0384801F0ECFC32
:104D3000C0B2009040F22551344801F0F8FB3448ED
:104D40000078022805D19DF80010324801F0E1FCFE
:104D500048E02F480078012805D19DF800102E4822
:104D600001F0D7FC3EE02A48007800283AD12B48D1
:104D7000008828B100202A4908802A49087038BDD7
:104D80009DF80010264802880088401C244B18809B
:104D900024488154244800780D281AD19DF8000039
:104DA0000A2816D11F48007847280DD11D484078A1
:104DB000542809D11846008818490880002019494C
:104DC0001A461288885404E00020154908801549C5
:104DD000087013480088C72804DB002010490880A9
:104DE0000E4908809DF800000F4908700821074807
:104DF00001F0C1FB012806D1044801F085FC08211F
:104E0000024801F08BFB00BFB9E700000038014009
:104E10000C00002000440040004800401200002028
:104E200010000020D00E00202500002008B540F220
:104E30002551254801F0ACFBB0B3234801F064FCD8
:104E4000C0B200902148007802280AD19DF80010D5
:104E50001F4801F05EFC40F225511B4801F067FB42
:104E600008BD1C480088B0F5A06F15DA9DF8000059
:104E700019491A4A1288885418480088401C80B280
:104E800016490880B0F5A06F01DB002008801148AA
:104E90000088401C0F490880114803F00BFC40F2C9
:104EA0002551094801F043FB0821074801F063FB45
:104EB000012806D1044801F027FC0821024801F02E
:104EC0002DFB00BFCCE70000004400400C00002098
:104ED000003801401E000020C410002020000020E7
:104EE0002C01002038B5002440F225513D4801F046
:104EF0004FFB002868D03B4801F006FCC0B2009090
:104F000039480078012805D19DF80010374801F094
:104F100000FC50E036480088002849D19DF8000088
:104F20003449354A1288885408460078242803D02A
:104F300000203149088004E02F480088401C2E4999
:104F400008802D480088B0F5957F02DD00202A49B1
:104F500008802A4800780D282DD19DF800000A28E5
:104F600029D124484078472807D12248C0785228C0
:104F700003D12048407943280BD01E484078472869
:104F800012D11C48007947280ED11A48407941288F
:104F90000AD1002118480088401E164A11541648AC
:104FA00000881349088006E000201349088002E0C9
:104FB00000201149088040F225510A4801F0B7FA53
:104FC0009DF800000D4908700821064801F0D3FA49
:104FD000012806D1034801F097FB0821014801F0A0
:104FE0009DFA38BD004800400C0000200038014008
:104FF00018000020980F0020160000202700002035
:1050000003498978024A5170114688707047000040
:105010005401002030B589B005467648007880B943
:1050200075A0FDF725FE322402E00120F8F76AFFA3
:10503000201EA4F10104F8D10120FFF7E1FF09B01F
:1050400030BD002D7ED000206A4981F86D006FA030
:10505000FDF70EFE002072490880F3F7FFFE0121E4
:1050600070A0FDF7C9FC012314229F210020F3F753
:1050700099FF002407E06E486E4941F824000020A3
:105080006D490855641C642CF5DD5A486BA21E213D
:10509000036F01A802F076FB002201A91046FEF77B
:1050A00003FA00244BE004EB440000EBC401664823
:1050B00050F821004F49C96B88423FD1E4B32346E1
:1050C00062A21E2101A802F05DFB012201A90020BD
:1050D000FEF7EAF94748D0F87C1104EB440000EBF6
:1050E000C402594840F8221004EB440101EBC40209
:1050F000014601EB8201881D24225349891DEFF7E7
:10510000EDF83C48B0F8801104EB440000EBC40219
:105110004D4800EB820081803648C06B3549C1F8AC
:105120007C012422423101F5A070EFF7D7F8314815
:10513000B0F84010A0F880112E48046F641C2D4870
:10514000006F00E034E0A04201DD642CABDB002402
:1051500019E004EB440000EBC4013B4850F8210087
:105160002449C96B884202D101203349085504EB18
:10517000440000EBC401344800EB8100801D2D4940
:1051800041F82400641C1B48006FA04201DD642C20
:10519000DFDB2948304B0022264900902F48F5F7E5
:1051A00069FB012368229F210020F3F7FBFE46E7FD
:1051B0001B48008830B9012329A26E210020F4F792
:1051C0005DF909E016480088C82805D1012329A205
:1051D0006E210020F4F752F911480088401C80B27B
:1051E0000F490880B0F5C87F01DB0020088000BFB0
:1051F00025E70000402900202020C7EBCFC8B5C715
:10520000C2BC2E2E2E20202000000000D5FDD4DAB6
:10521000BBF1C8A12CC7EBC9D4BAF22E2E2E0000C8
:10522000C4010020C8BAD7E9D1A1D4F10000000020
:10523000D4010020084900209C4A0020476E756D6B
:105240003D25640D0A000000BC2A0020693A25644F
:105250002A2A2A2A00000000C801002058470020FE
:105260005BC9CF5DD1A1D4F1205BCFC25DD1A1D408
:10527000F12020005B4D5DC8B7B6A820205B4558E3
:1052800049545DCDCBB3F60070B592B0054675B10B
:1052900000208B490870F3F7E1FD012189A0FDF79B
:1052A000ABFB012314229F210020F3F77BFE022693
:1052B0001624874800688749884206D084480068D9
:1052C0008549884201D0002D73D0002080490860B4
:1052D0007B48007818B17A48007802286BD17F2388
:1052E0009F2221460020F3F713FE7C4B7CA2322143
:1052F00002A802F047FA012302AA21463046F4F739
:10530000BDF804F1140084B274482138D0F81D307F
:1053100076A2322102A802F035FA012302AA214620
:105320003046F4F7ABF804F1140084B2734890F8F7
:1053300030030121CDE9001068482138B0F82F3042
:105340006FA2322102A802F01DFA012302AA21460F
:105350003046F4F793F804F1140084B26D486EA25D
:105360003221036802A802F00DFA012302AA2146A5
:105370003046F4F783F804F1140084B200208DF86D
:105380003C0056482138D0F81D10674A0FA8F2F7A4
:1053900043FB0FAB65A2322102A802F0F3F901230F
:1053A00002AA21463046F4F769F801204449087002
:1053B00084E02CE0FFE74248007801287ED17F237B
:1053C0009F2221460020F3F7A3FD5B485BA2322118
:1053D000036802A802F0D6F9012302AA214630464A
:1053E000F4F74CF804F1140084B20020302357A2E3
:1053F0003221009002A802F0C5F9012302AA214639
:105400003046F4F73BF802202D49087056E030484A
:1054100000685349884251D100202D49086028482E
:105420000078012803D026480078022846D17F233F
:105430009F2221460020F3F76BFD012349A221465C
:105440003046F4F71BF804F1140084B2484B49A22B
:10545000322102A802F096F9012302AA2146304621
:10546000F4F70CF804F1140084B2012342A221469F
:105470003046F4F703F804F1140084B2414B3DA226
:10548000322102A802F07EF9012302AA2146304609
:10549000F3F7F4FF04F1140084B21848B0F82D3388
:1054A00039A2322102A802F06DF9012302AA214695
:1054B0003046F3F7E3FF00200149087012B070BDD9
:1054C000F2010020D6D5B6CBD0C5CFA20000000097
:1054D000B80000202A04DC002A04BC00E5150020E6
:1054E000D6D5B6CBD0CDBAC53A257300D6D5B6CB76
:1054F000B1E0C2EB3A256C7500000000AB5600200D
:10550000D3A6D3C3B0E6B1BE3A5625642E25642E89
:1055100025640000F4000020C4A3BFE9B0E6B1BEDA
:105520003A4C256400000000F6150020D0A3D1E914
:10553000C2EB3A2573000000F8000020B6D4BDB2DB
:10554000B0E6B1BE3A562564000000004D4355D682
:10555000F7C6B53A25642E2564204D687A00000010
:105560002A04AC00BDBBBBBBB7FECEF1C6F73A0008
:105570000847002025730000B1B1B6B7B7FECEF1E1
:10558000C6F73A0030470020504F52543A25640085
:1055900010B50446002C29D0F3F760FC012314A2B7
:1055A00019460020F3F76AFF012314229F210020EF
:1055B000F3F7F8FC11484088012807DB0F484188C1
:1055C00000230F4A0F48F5F7AFF903E00021084622
:1055D000F5F7DAF901230CA26E210020F3F74EFF54
:1055E000012368229F210020F3F7DCFC10BD00009E
:1055F0002020CEC4B1BECFFBCFA200005452002069
:1056000058020020584700205B4D5DB2E9D4C42009
:105610002020205B535DD1A1CFEE200030B585B0B6
:10562000054695B1F3F71AFCB6A26B210120FDF7F0
:105630006FF94FF0FF30B54908600020B4490860A9
:105640002846FDF721FC05B030BD2846FDF71CFCBF
:10565000B048007808B9002424E0AE48807838B912
:10566000AC48807920B901240020AB49086019E0DA
:10567000A848807828B9A7488079002801DD02244D
:1056800010E0A448807800280CDD0324A2480068BC
:1056900040B90120A049086022239F221221002046
:1056A000F3F736FC34B1012C14D0022C26D0032C95
:1056B00076D14AE09548006884420AD061239F224F
:1056C00026210020F3F724FC94A226210020F3F7E2
:1056D00061FE65E08D48006884420ED061239F2200
:1056E00026210020F3F714FC8CA226210020F3F7DA
:1056F00051FE01218C4880F8B81251E083480068BF
:10570000844205D061239F2226210020F3F700FC6C
:105710007F48006828B985A228213420F3F73AFE93
:1057200012E07B480068642805D183A22821342038
:10573000F3F730FE08E076480068C82804D181A25B
:1057400028213420F3F726FE2AE0704800688442BE
:1057500005D061239F2226210020F3F7D9FB6C4856
:10576000006828B97AA226213620F3F713FE12E04A
:1057700067480068642805D178A226213620F3F70F
:1057800009FE08E062480068C82804D177A22621F3
:105790003620F3F7FFFD12210020FDF7E1F800BFEE
:1057A00000BF002C1CDD5A48006838B1584800681A
:1057B000642803D056480068C8280AD1032C08D0B2
:1057C00052480068844205D0012212210020FDF7D2
:1057D0007DF980E0002212211046FDF777F97AE08A
:1057E000202214216846EEF78BFD092263A168464A
:1057F000EEF774FD4648006830B901236A4612216D
:105800000020F3F73BFE1CE041480068642809D102
:105810002E208DF8090001236A4612210020F3F79B
:105820002DFE0EE03A480068C8280AD12E208DF8D7
:1058300009008DF80A0001236A4612210020F3F7BF
:105840001DFE394890F8BB024F490978884203D1C0
:105850002E480068401CB0BB334890F8BB024A4950
:10586000087008460078012805D148A2142168462E
:1058700001F088FF29E044480078022805D147A2BA
:105880001421684601F07EFF1FE03F48007804289D
:1058900005D146A21421684601F074FF15E03A488C
:1058A0000078052805D145A21421684601F06AFF59
:1058B0000BE035480078062806D143A2142168463B
:1058C00001F060FF01E006E006E001236A462621C0
:1058D0000020F3F7D3FD00BF0D480068401C0C49C1
:1058E0000860B0F5967F01DB00200860074800687B
:1058F000844204D00548046000200549086000BFC8
:10590000A1E60000B2CBB5A50000000068010020B0
:105910006C01002040290020580100206C6F676F47
:105920002E626D7000000000403900205069636BEA
:1059300075702E626D7000005069636B7570312E4A
:10594000626D70005069636B7570322E626D70000D
:10595000737065616B65722E626D70007370656146
:105960006B6572312E626D700000000073706561AE
:105970006B6572322E626D7000000000D5FDD4DAC6
:10598000B5C7C2BD2E00000070010020D5CBBAC53E
:10599000D0C5CFA2B4EDCEF300000000CEDECDF82E
:1059A000C2E7C1ACBDD3202000000000C7EBB2E5C8
:1059B000BFA820202020202000000000CEDEB7A8B5
:1059C000C1ACBDD300000000C3BBD3D0B7FECEF145
:1059D0000000000010B5044684B1F3F73FFA01213E
:1059E00007A0FDF709F8012314229F210020F3F7F7
:1059F000D9FA05490548F6F7E9F810BD00BFFCE7FC
:105A0000D6F7B2CBB5A50000740100205C010020E0
:105A100070B50646002500BF2846691CCDB21B495B
:105A200051F8200000780028F6D1681EC5B256B3A0
:105A3000F3F714FA012116A0FCF7DEFF012314226C
:105A40009F210020F3F7AEFA14480078012815D002
:105A5000002407E00D4850F82400114941F82400C3
:105A6000601CC4B2072CF5DB084850F825000C492F
:105A700041F824000B48F6F7A9F803E00349094868
:105A8000F6F7A4F870BD00BFFCE700008C01002011
:105A9000CFB5CDB3C9E8D6C3000000002800002070
:105AA000E048002080020020F8B50646002E5DD0B8
:105AB000F3F7D4F902212EA0FCF79EFF0123142254
:105AC0009F210020F3F76EFA012368229F21002016
:105AD000F3F768FA012329A26E210020F3F7CEFC28
:105AE0002B4890F89C502B480078012803D0022DB9
:105AF00001DBA81EC5B2002409E0AC4203D101209D
:105B00002549085502E0002023490855641C042C4F
:105B1000F3DD20480078012808D11F481F4B0022E0
:105B20001F4900901F48F4F7A5FE1EE0002406E080
:105B30001B4850F824001C4941F82400641C022C26
:105B4000F6DB174802692046641C174941F82020FB
:105B5000134842692046641C41F820200E480F4B30
:105B6000002200900F48F4F785FEF8BD00BFFCE767
:105B7000B7FECEF1C6F7C1D0B1ED00005B4D5DC8F8
:105B8000B7B6A820205B455849545DCDCBB3F6008D
:105B9000AB5600202800002000030020DC0200207B
:105BA000E8020020584700202054002010B5044689
:105BB00004B3F3F753F901210FA0FCF71DFF0123F4
:105BC0001422A0210020F3F7EDF90EA3382211468C
:105BD0000E48F8F7C1F80D48F8F710F901236822CC
:105BE000A0210020F3F7DEF9012309A26E21002095
:105BF000F3F744FC10BD0000C3DCC2EBD1E9D6A42E
